:100000000C9471070C9488550C94B5550C94E255DA
:100010000C9499070C9499070C9499070C949907E0
:100020000C9412140C9499070C9499070C9499074A
:100030000C9499070C9499070C9499070C949907C0
:100040000C9499070C9499070C9491560C94990769
:100050000C946C580C94FA580C9499070C949907CA
:100060000C9499070C9499070C942E730C9499078F
:100070000C94A1580C9435590C9499074E54502067
:1000800053796E63696E672E2E2E002020007273E6
:1000900000726400776C00666C00005D0D0A002C35
:1000A00000222C002C22002C002C005B002E7478E7
:1000B0007400302E2054657374202831206D696ED1
:1000C00029002E20002000486F6C642042332074E9
:1000D0006F20737461727400436C69636B204233E8
:1000E00020746F206C6973740052756E206120500B
:1000F000726F6772616D3A00286C7377632900280C
:10010000656970290020286F73697029003A0028FA
:1001100067776970290077746F7074732E747874C0
:100120000073746E732E64617400667776000074D9
:100130007A0000006E74700000646863700069707B
:10014000310000697032000069703300006970345A
:10015000000067773100006777320000677733006F
:10016000006777340000687030000068703100006C
:10017000687776000065787400007365710000731D
:10018000647400006D617300006D746F6E006D74B7
:100190006F6600757273000072736F0000776C00F9
:1001A000000064656E0000697061730064657669C3
:1001B00064636F6E00006C6974000064696D000018
:1001C000627374000075777400006E747031006E95
:1001D000747032006E747033006E747034006C672B
:1001E0000000006D617332006D746F6E326D746F5C
:1001F000663266776D00006670723000667072312C
:100200000072650000007265736574004669726D66
:10021000776172652076657273696F6E54696D657A
:10022000207A6F6E652028474D54293A456E6162E9
:100230006C65204E54502073796E633F456E616249
:100240006C6520444843503F202020205374617443
:1002500069632E6970313A20202020205374617424
:1002600069632E6970323A20202020205374617413
:1002700069632E6970333A20202020205374617402
:1002800069632E6970343A2020202020476174650C
:100290007761792E6970313A20202020476174659A
:1002A0007761792E6970323A202020204761746589
:1002B0007761792E6970333A202020204761746578
:1002C0007761792E6970343A2020202048545450A8
:1002D00020506F72743A2020202020202D2D2D2DAB
:1002E0002D2D2D2D2D2D2D2D2D2D2D2D4861726473
:1002F000776172652076657273696F6E23206F6611
:10030000206578702E20626F6172643A2D2D2D2D3C
:100310002D2D2D2D2D2D2D2D2D2D2D2D53746E2E5E
:100320002064656C61792028736563294D6173745D
:100330006572203120284D617331293A4D61733146
:1003400020206F6E2061646A7573743A4D61733159
:10035000206F66662061646A7573743A53656E73C4
:100360006F7220747970653A202020204E6F726D74
:10037000616C6C79206F70656E3F202057617465E9
:1003800072696E67206C6576656C3A2044657669A3
:10039000636520656E61626C65643F2049676E6FBE
:1003A00072652070617373776F72643F446576691C
:1003B00063652049443A2020202020204C434420DB
:1003C000636F6E74726173743A2020204C43442032
:1003D0006272696768746E6573733A204C43442097
:1003E00064696D6D696E673A202020204443206265
:1003F0006F6F73742074696D653A2020576561745E
:1004000068657220616C676F2E3A20204E54502030
:100410007365727665722E6970313A204E545020A1
:100420007365727665722E6970323A204E54502090
:100430007365727665722E6970333A204E5450207F
:100440007365727665722E6970343A20456E61620A
:100450006C65206C6F6767696E673F204D617374D0
:100460006572203220284D617332293A4D61733212
:1004700020206F6E2061646A7573743A4D61733227
:10048000206F66662061646A7573743A4669726D9E
:1004900077617265206D696E6F723A2050756C736A
:1004A0006520726174653A20202020202D2D2D2D8D
:1004B0002D2D2D2D2D2D2D2D2D2D2D2D41732072DA
:1004C000656D6F7465206578742E3F204661637496
:1004D0006F72792072657365743F202000006C0193
:1004E00001FFFFFFFFFFFFFFFFFFFF000501F730E8
:1004F0003C78FF01FA0101FFFFFFFFFAFFFFFFFF5A
:10050000FF01303C7800FFFF010120736563002587
:10051000004E6F00596573002E002B002B00303009
:10052000003A002D002B000020202020002D4469DF
:100530007361626C6564212D003A0045004D433AB9
:100540000020284D414329002D002E004D6F6E00E4
:1005500054756500576564005468750046726900FB
:100560005361740053756E00002D002000202000A0
:100570003A00200020414300204C41002044430029
:100580004857207600204F70656E537072696E6B0D
:100590006C657200486F6C6420423320746F207366
:1005A0006176650042312F42323A2B2F2D2C2042AA
:1005B000333A2D3E003D3D536574204F7074696F92
:1005C0006E733D3D00506C656173652057616974C1
:1005D0002E2E2E00526573657474696E672E2E2E52
:1005E000002A002F636D003F70773D244526736914
:1005F000643D244426656E3D244426743D24440015
:10060000436F6E6E656374696E672E2E2E00507296
:100610006F6772616D200063766A636470637063F4
:100620007275706A70636F6A6F73706A73636D63FB
:10063000736A6E6A656A6C646C737563756A61006F
:100640003C7363726970743E77696E646F772E6C69
:100650006F636174696F6E3D222F223B3C2F736381
:10066000726970743E0A0022726573756C74223A66
:1006700024447D0022726573756C74223A24447D93
:1006800000244600222446223A24447D007D002C8A
:100690002273746174696F6E73223A7B002C22732B
:1006A0007461747573223A7B002C226F7074696FC9
:1006B0006E73223A7B002C2270726F6772616D73C9
:1006C000223A7B002273657474696E6773223A7BE9
:1006D00000646179005D002453002C005B00747994
:1006E000706500656E64007374617274006869738C
:1006F00074007400656E00736964005D2C226E7373
:10070000746174696F6E73223A24447D002C002456
:10071000440022736E223A5B00637077006E70773C
:100720000077746F007474740077746B6579006C73
:100730006F6300777370006A737000726500726493
:1007400000656E007262740072736E003C6D6574B9
:1007500061206E616D653D2276696577706F727498
:100760002220636F6E74656E743D227769647468CD
:100770003D6465766963652D77696474682C696E7C
:10078000697469616C2D7363616C653D312E302C29
:100790006D696E696D756D2D7363616C653D312E8C
:1007A000302C757365722D7363616C61626C653D8D
:1007B0006E6F223E0D0A003C736372697074207381
:1007C00072633D2224452F686F6D652E6A73223E49
:1007D0003C2F7363726970743E0A3C2F626F6479B8
:1007E0003E0A3C2F68746D6C3E007661722076651F
:1007F000723D24442C697061733D24443B3C2F734B
:1008000063726970743E0A003C21444F435459504E
:10081000452068746D6C3E0A3C68746D6C3E0A3C01
:10082000686561643E0A24463C2F686561643E0A3F
:100830003C626F64793E0A3C7363726970743E0077
:100840007D002C2277746F223A7B24537D005D005B
:100850002C005B24442C244C2C244C5D00305D2C5B
:10086000227073223A5B0024442C00227362697464
:1008700073223A5B0022666C637274223A244C2C19
:1008800022666C777274223A24442C0022646576C6
:1008900074223A244C2C226E627264223A24442C34
:1008A00022656E223A24442C227264223A24442C7B
:1008B000227273223A24442C2272647374223A24E2
:1008C0004C2C226C6F63223A222445222C2277740E
:1008D0006B6579223A222445222C2273756E726947
:1008E0007365223A24442C2273756E736574223A20
:1008F00024442C22656970223A244C2C226C7763A4
:10090000223A244C2C226C737763223A244C2C22FA
:100910006C72756E223A5B24442C24442C24442CA3
:10092000244C5D2C003C666F726D206E616D653DE0
:100930006F6620616374696F6E3D6375206D6574C9
:10094000686F643D6765743E3C7461626C652063EA
:10095000656C6C73706163696E673D223132223E53
:100960003C74723E3C74643E3C623E4A6176615324
:1009700063726970743C2F623E3A3C2F74643E3C53
:1009800074643E3C696E70757420747970653D7452
:100990006578742073697A653D3430206D61786CB8
:1009A000656E6774683D34302076616C75653D22F4
:1009B000244522206E616D653D6A73703E3C2F7444
:1009C000643E3C2F74723E3C74723E3C74643E4400
:1009D000656661756C743A3C2F74643E3C74643E89
:1009E00024533C2F74643E3C2F74723E3C74723E20
:1009F0003C74643E3C623E576561746865723C2F8E
:100A0000623E3A3C2F74643E3C74643E3C696E70B6
:100A1000757420747970653D746578742073697A93
:100A2000653D3430206D61786C656E6774683D3467
:100A3000302076616C75653D22244522206E616D03
:100A4000653D7773703E3C2F74643E3C2F74723E5C
:100A50003C74723E3C74643E44656661756C743AE5
:100A60003C2F74643E3C74643E24533C2F74643EBB
:100A70003C2F74723E3C74723E3C74643E3C623E59
:100A800050617373776F72643C2F623E3A3C2F74EF
:100A9000643E3C74643E3C696E7075742074797079
:100AA000653D70617373776F72642073697A653D19
:100AB0003332206E616D653D70773E203C696E700B
:100AC000757420747970653D7375626D69743E3C10
:100AD0002F74643E3C2F74723E3C2F7461626C65CF
:100AE0003E3C2F666F726D3E3C736372697074207A
:100AF0007372633D68747470733A2F2F75692E6F2B
:100B000070656E737072696E6B6C65722E636F6D5B
:100B10002F6A732F6861736865722E6A733E3C2F6B
:100B20007363726970743E005D7D00225D00225D1A
:100B30002C00245300244C5D2C2200244C2C002437
:100B4000445D2C5B0024442C005B24442C24442C66
:100B500024442C5B00226E70726F6773223A244427
:100B60002C226E626F61726473223A24442C226DCF
:100B70006E70223A24442C226D6E7374223A2444FF
:100B80002C22706E73697A65223A24442C22706498
:100B9000223A5B002C2264657870223A24442C228D
:100BA0006D657870223A24442C22687774223A24A6
:100BB000447D002C00222453223A2444006E616DAF
:100BC0006500706964007069640070696400736432
:100BD00000737400736964007D00222444223A7B10
:100BE000227374223A24442C227364223A2224531E
:100BF000227D002C005D2C226D61786C656E223A9E
:100C000024447D002C00222453220022736E616D47
:100C10006573223A5B0073746E5F73706500737462
:100C20006E5F7365710073746E5F646973006D61EC
:100C3000736F70320069676E6F72655F7261696EA3
:100C4000006D61736F70005D2C002C002444002245
:100C50002446223A5B00707700485454502F312EBE
:100C60003120323030204F4B0D0A00436F6E7465D7
:100C70006E742D547970653A206170706C6963618F
:100C800074696F6E2F6A736F6E0D0A436F6E6E65B7
:100C90006374696F6E3A20636C6F73650D0A00416F
:100CA00063636573732D436F6E74726F6C2D416C4B
:100CB0006C6F772D4F726967696E3A202A0D0A00B2
:100CC00043616368652D436F6E74726F6C3A206D7B
:100CD00061782D6167653D302C206E6F2D636163F7
:100CE00068652C206E6F2D73746F72652C206D7586
:100CF00073742D726576616C69646174650D0A00A8
:100D00007B0024462446244624460D0A00436F6E89
:100D100074656E742D547970653A20746578742FFB
:100D200068746D6C0D0A0024462446244624460D42
:100D30000A000001080006040001450000820000CE
:100D400040002000504F5354202446204854545013
:100D50002F312E300D0A486F73743A2024460D0A45
:100D6000244624534163636570743A202A2F2A0D68
:100D70000A436F6E74656E742D4C656E6774683AC5
:100D80002024440D0A436F6E74656E742D5479707F
:100D9000653A206170706C69636174696F6E2F7859
:100DA0002D7777772D666F726D2D75726C656E631A
:100DB0006F6465640D0A0D0A2453004745542024CE
:100DC00046245320485454502F312E300D0A486F7A
:100DD00073743A2024460D0A24460D0A0D0A004178
:100DE00063636570743A20746578742F68746D6CF1
:100DF00000E30004FA0001000000012A002F7765DB
:100E000061746865720024442E70793F6C6F633D95
:100E10002445266B65793D2445266677763D244436
:100E20002677746F3D245300726400747A007363F4
:100E3000616C65006569700073756E73657400732D
:100E4000756E726973650000002100240027002A76
:100E50000000002200250028002B000000200023B5
:100E60000026002900020202020202020204040417
:100E70000404040404030303030303030301010143
:100E80000101010101010204081020408001020457
:100E9000081020408001020408102040808040207B
:100EA0001008040201000000010200000000000020
:100EB000000403070600000000000000000000001E
:100EC00000000000007C3C3E5E2B3D3F2F5B5D3B05
:100ED0002C2A225C0000780E56147C21155A145CD2
:100EE000EE6E11241FBECFEFD0E1DEBFCDBF12E00A
:100EF000A0E0B1E0E6E5FBEE02C005900D92A83857
:100F0000B107D9F71EE0A8E8B2E001C01D92A133F5
:100F1000B107E1F71EE0C2EEDEE004C02297FE0159
:100F20000E94A575C63DD107C9F70E94AB5A0C9423
:100F3000E0070C940000FC0188279927E894219190
:100F40002032E9F3293010F02E30C8F32B3241F073
:100F50002D3239F4689404C00E94C308820F911D99
:100F6000219120532A30C0F31EF4909581959F4F14
:100F700008951F93FC0199278827BC01E8941191DB
:100F80001032E9F3193010F01E30C8F31B3251F063
:100F90001D3249F4689406C00E94AE08610F711DAD
:100FA000811D911D119110531A30B0F33EF49095AC
:100FB0008095709561957F4F8F4F9F4F1F9108953A
:100FC000F8940C94A975FB01DC0102C005900D9208
:100FD00041505040D8F70895FB01DC010D900020EE
:100FE000E9F7119705900D920020E1F70895FB01B4
:100FF000DC0105900D920020E1F70895FB01DC0172
:1010000004C08D910190801921F441505040C8F7DF
:10101000881B990B0895FB01DC0102C001900D9221
:1010200041505040D8F70895DC0101C06D93415004
:101030005040E0F70895FB01DC010D900020E9F736
:10104000119701900D920020E1F70895FC01819124
:10105000861721F08823D9F7992708953197CF0172
:101060000895FB01DC0101900D920020E1F7089545
:10107000FB01DC014150504030F08D91019080190E
:1010800019F40020B9F7881B990B0895FB01DC01C6
:101090004150504048F001900D920020C9F701C026
:1010A0001D9241505040E0F70895A0E0B0E0EBE51C
:1010B000F8E00C9476757C01EB018A01690109C0A6
:1010C000CE012196F6010995F70181937F01015028
:1010D000104001151105A1F7CDB7DEB7E8E00C947B
:1010E0009275A0E0B0E0E7E7F8E00C947675EC01CB
:1010F0007B018A01690109C0CE012196F701619146
:101100007F01F60109950150104001151105A1F765
:10111000CDB7DEB7E8E00C949275FB019F01E8942F
:101120004230C4F04532B4F44A3029F497FB1EF43F
:10113000909581959F4F642F77270E940875805D59
:101140008A330CF0895D8193CB010097A1F716F4E7
:101150005DE251931082C9010C94F008592F482F79
:10116000372F262F660F771F881F991F660F771F4F
:10117000881F991F620F731F841F951F660F771FAB
:10118000881F991F08957AE0979F902D879F802D43
:10119000910D11240895FA01CF93FF93EF9322301C
:1011A000CCF02532BCF4C22F2C2F332744275527EF
:1011B000FF93EF930E942F75EF91FF91605D6A336B
:1011C0000CF0695D6193B901CA01605070408040C4
:1011D000904051F710828F919F91CF910C94F0081D
:1011E000DC01FC01672F71917723E1F7329704C08E
:1011F0007C916D9370836291AE17BF07C8F3089519
:10120000DF93CF9300D000D000D0CDB7DEB7DE01A2
:101210001196ECE1F2E086E001900D928150E1F749
:1012200086E191E0EEEEF2E0DF019C011D9221509B
:101230003040E1F780918802833019F46EED72E05E
:1012400003C0BE016F5F7F4F84E490E043E450E051
:101250000E94434880918802833039F08EEE92E0FC
:10126000BE016F5F7F4F0E943C5581E08093180361
:101270008093190386E080931A03809195029091E0
:101280009602A0919702B091980280931C039093CC
:101290001D03A0931E03B0931F0380918802833027
:1012A00039F488E193E00C966EEC72E00E944455AC
:1012B00084E393E068EC72E00E943C55A4E0B4E063
:1012C000E0EBF1E002C081918D9331E0E63BF30762
:1012D000D1F790918802992311F083E001C081E059
:1012E00080930A048DE380930B0487E080930C04C1
:1012F00081E080930D04AEE0B4E0E8ECF2E002C0DF
:1013000081918D9382E0EE3CF807D1F78CE08093D9
:10131000140485E080931504EAEAF1E0A6E1B4E064
:1013200002C081918D9321E0EF3AF207D1F72BE1D2
:1013300034E030939D0220939C02913069F582E362
:1013400080931B0484E080931C04D9011296EEEC78
:10135000F2E002C081918D9332E0E23DF307D1F7D4
:1013600086E38093210484E08093220483E294E066
:1013700090939D0280939C02DC01EEEDF2E002C0AE
:1013800081918D9382E0E23EF807D1F787E294E005
:1013900090939D0280939C0220919B02222311F046
:1013A00094E001C093E0A0919C02B0919D02FD01E8
:1013B00087E3819311969C93DF01119681E08183ED
:1013C000FD01319683E011968C93DF01119686E042
:1013D0008183CD01019690939D0280939C022223EC
:1013E00039F011962C93019690939D0280939C0264
:1013F000E0919C02F0919D028FEF8193F0939D020A
:10140000E0939C02CF01885193400E94294A26967E
:101410000FB6F894DEBF0FBECDBFCF91DF91089518
:10142000BF92CF92DF92EF92FF920F931F93CF93D1
:10143000DF938C0180918802823009F401C18330EE
:1014400030F4882351F1813009F076C14BC08330EC
:1014500021F0843009F070C1F3C00E94DD5020916A
:101460008D0230918E0240918F0250919002E09057
:101470008902F0908A0200918B0210918C022E0D4D
:101480003F1D401F511F261737074807590708F00F
:1014900053C10E94000984E018C00E94D95660938D
:1014A00095027093960280939702909398021092FF
:1014B000CE021092CF021092D0021092D1020E945E
:1014C000000981E00E941A0F81E0809388020E9447
:1014D000D9566093910270939202809393029093F5
:1014E00094022AC10634110508F4DEC0809111036C
:1014F000833409F0D9C020911C0330911D03409121
:101500001E0350911F038091950290919602A09125
:101510009702B0919802281739074A075B0709F02C
:10152000C3C0C8E0D4E0FE01A80142515D4FDF0115
:10153000119691819D012F5F3F4F8081853329F462
:1015400011968C91823009F4CEC0F901E90FF11D9A
:10155000E417F50760F3A8C0FE019191B980EF018F
:1015600021969333E1F0943340F4933091F0963028
:1015700099F0913009F04FC009C09A3381F09F3F34
:1015800009F45AC0963309F046C03FC082ED92E09C
:101590003EC08AED92E03BC082EE92E038C081818D
:1015A00090E0A0E0B0E0BA2FA92F982F88272981DA
:1015B000820F911DA11DB11DBA2FA92F982F882729
:1015C0002A81820F911DA11DB11DBA2FA92F982F1D
:1015D00088272B81820F911DA11DB11D80938D0243
:1015E00090938E02A0938F02B09390028158914500
:1015F000A140B04008F499C0C0928D02D0928E02F2
:10160000E0928F02F092900290C08EED92E0BE01C7
:101610000E9444558AC0E0919902F0919A02309755
:1016200009F483C080919B02981709F07EC0892F2E
:10163000BE014B2D099579C00E94000982E045CF7B
:101640000634110588F180911103833469F52091E6
:101650001C0330911D0340911E0350911F03809184
:10166000950290919602A0919702B0919802281746
:1016700039074A075B07C1F4E8E0F4E0A8014251EA
:101680005D4FDF01119691819D012F5F3F4F80815A
:10169000853321F411968C918530A9F1F901E90F78
:1016A000F11DE417F50768F30E94D95620919102C5
:1016B000309192024091930250919402205F384DF4
:1016C0004F4F5F4F261737074807590748F034C078
:1016D0008AED92E00E94A94883E0809388022CC0A2
:1016E0001092880229C08EEC92E068E273E00E94BA
:1016F000445580E8C82E81E5D82E81E0E82EF12CF3
:1017000002511D4F29CF81E00E94090F0E94DD5038
:101710006093890270938A0280938B0290938C026B
:101720008091DA028823C1F2D3CFCB0DD11DC0172F
:10173000D10708F411CF80CFDF91CF911F910F9186
:10174000FF90EF90DF90CF90BF900895CF93DF93FD
:1017500081E08093EA029091CD02892F82958F706B
:101760008F5B8093AD019F709F5B9093AE01109251
:1017700088020E94D956EB0104C00E946A0F0E94A1
:10178000100A80918802833061F00E94D9566C1B48
:101790007D0B6053754728F40E942B0F882389F333
:1017A000ECCF0E94BF471092ED021092EC0290E045
:1017B00080918802833009F491E0892FDF91CF91E5
:1017C0000895FF920F931F93CF93DF938C01F62E12
:1017D0000E94D956EB010CC00E946A0F0E94F64A83
:1017E0000E94D9566C1B7D0B6053754708F0EFC003
:1017F0000E942B0F882381F30E94D956EB010CC065
:101800000E946A0F0E94F64A0E94D9566C1B7D0BFB
:101810006053754708F0DBC00E94B947882381F701
:101820001092E6021092E7021092E8021092E9028A
:1018300080919E028F5F80939E028091E2028823B6
:1018400061F488E098E0A8E0B8E08093E202909329
:10185000E302A093E402B093E50280919E0290E03F
:10186000906E62EE72E045E350E00E944348E8E18A
:10187000F3E08CE0DF011D928A95E9F7DF011C9609
:1018800090E0FF2019F0F801808102C0F8018491F6
:101890000F5F1F4F8E3241F0882331F09F5FFD01B3
:1018A000E90FF11D8083EDCFFD019193DF01A90FB9
:1018B000B11D882329F7FD01119211961C92DF01B9
:1018C000119641E04183FD01319611961C924183AE
:1018D00086ED2EEE32E0821B32968E0F8093180337
:1018E00090919E029093190340931A0340931D0315
:1018F00090E00E94294A0E94D9568B0161C00E9443
:10190000D956601B710B6053754708F060C00E9488
:101910006A0FEC01009709F453C00E94F64A892B24
:1019200009F04EC0C634D10508F44AC080911103B5
:10193000853309F045C080911203803E09F040C014
:101940009091130380919E029817D1F5809119030D
:101950008917B1F580911B0390E08F709070892BEF
:10196000B1F580911803E82FF0E0E85EFC4F9E018E
:1019700022513D4F8081807C39F0329609C08081B0
:10198000882311F4319604C03196E217F307B8F3B7
:10199000CF010E962817390798F08181813051F4D4
:1019A0008185843039F43A9686EE92E0BF010E9438
:1019B000445506C0818590E00A96E80FF91FDACFFA
:1019C0008091E602882309F49ACF81E001C080E08B
:1019D000DF91CF911F910F91FF900895482F6AE0FA
:1019E0000E94FC74282F30E084E0220F331F8A9578
:1019F000E1F7842F0E94FC74892F820F0895CF9302
:101A0000DF93EC0180919F029091A00288369105AE
:101A100059F582EA9BE068E670E00E94DA5B82EAB0
:101A20009BE060E00E945C5C88810E94EE0C682F65
:101A300070E06F77707082EA9BE00E945C5C898145
:101A40000E94EE0C682F82EA9BE00E945C5C8A8117
:101A50000E94EE0C682F82EA9BE00E945C5C8B8106
:101A60000E94EE0C682F2DC08F36910509F04AC0F8
:101A700082EA9BE06FE670E00E94DA5B82EA9BE01C
:101A800060E00E945C5C88810E94EE0C682F6068B8
:101A900082EA9BE00E945C5C89810E94EE0C682FC8
:101AA00082EA9BE00E945C5C8A810E94EE0C682FB7
:101AB00082EA9BE00E945C5C8B810E94EE0C682FA6
:101AC000686082EA9BE00E945C5C8C810E94EE0C64
:101AD000682F82EA9BE00E945C5C8D810E94EE0C84
:101AE000682F82EA9BE00E945C5C8E818E510E948E
:101AF000EE0C682F82EA9BE00E945C5C82EA9BE02D
:101B00000E949F5CDF91CF91089588E690E09093CA
:101B1000A00280939F0282EA9BE068E670E00E9448
:101B2000DA5B82EA9BE060E00E945C5C82EA9BE018
:101B30000E949F5C8823D9F08FE690E09093A002EA
:101B400080939F0282EA9BE06FE670E00E94DA5B7E
:101B500082EA9BE060E00E945C5C82EA9BE00E947B
:101B60009F5C882321F01092A00210929F0208959A
:101B70001F93CF93DF93EC0160919F027091A002BD
:101B80006115710509F470C082EA9BE00E94DA5B7E
:101B900082EA9BE060E00E945C5C82EA9BE00E943B
:101BA0009F5C60919F027091A00282EA9BE047E0F7
:101BB00050E00E94B05C82EA9BE00E94ED5B282F1F
:101BC0002F7722952F701AE0219F900111248F709A
:101BD000820F888382EA9BE00E94ED5B282F22958A
:101BE0002F70219F900111248F70820F898382EAC8
:101BF0009BE00E94ED5B282F2F7322952F70219F71
:101C0000900111248F70820F8A8382EA9BE00E94E8
:101C1000ED5B87708B8382EA9BE00E94ED5B282F4F
:101C200022952F70219F900111248F70820F8C8339
:101C300082EA9BE00E94ED5B282F2F7122952F7086
:101C4000219F900111248F70820F8D8382EA9BE087
:101C50000E94ED5B282F2F70225E82958F70819FEE
:101C6000C0011124280F2E83DF91CF911F91089579
:101C70000F931F93DF93CF93CDB7DEB727970FB6A0
:101C8000F894DEBF0FBECDBF8E010F5F1F4FA801BE
:101C90000E948A4EC8010E94FF0C27960FB6F89446
:101CA000DEBF0FBECDBFCF91DF911F910F91089581
:101CB0000F931F93DF93CF93CDB7DEB727970FB660
:101CC000F894DEBF0FBECDBF8E010F5F1F4FC8015E
:101CD0000E94B80DC8010E94D04F27960FB6F89405
:101CE000DEBF0FBECDBFCF91DF911F910F91089541
:101CF00082EA9BE00E94B45C08958091A40261E0B6
:101D00000E94C45778940895FF920F931F93082F51
:101D1000162FF42EF8948091A40260E00E94C4571C
:101D20001F71102B1EBD0DB407FEFDCFFEBC0DB400
:101D300007FEFDCF0E947D0E1F910F91FF90089529
:101D40001F93182F282F30E0207630708091A50245
:101D500090E02817390799F080EA6FE143E00E948C
:101D6000840E412F40764093A50250E085E05595C2
:101D700047958A95E1F780E86FE10E94840E1F91F4
:101D800008950F931F93182F062F0E94A00E80E432
:101D9000612F402F0E94840E1F910F9108950F9381
:101DA0001F93182F072F0E94C10E812F8F5F602F66
:101DB0000E94C10E1F910F9108950F931F93182F2A
:101DC000062FF8948091A40260E00E94C457802FEF
:101DD0008F71812B8EBD0DB407FEFDCF1EBC0DB4DF
:101DE00007FEFDCF07FF04C01EBC0DB407FEFDCFEC
:101DF0001EB50E947D0E812F1F910F9108951F9394
:101E0000182F0E94A00E80E0612F0E94DD0E1F910E
:101E10000895882311F41092A3028091A3028823CD
:101E200041F488E30E94FF0E682F6E7F88E30E94D2
:101E3000C10E08951F93182F88E30E94FF0E682F8C
:101E4000616088E30E94C10E112319F481E0809340
:101E5000A3021F91089584ED61E10E94C10E82EDFD
:101E600061E00E94C10E8AEE0E94FF0E80FDFBCF52
:101E700082ED60E00E94C10E89ED0E94FF0E90E0AD
:101E80009695879596958795817008950F931F93E2
:101E9000CF93DF93EC018B01F8948091A40260E072
:101EA0000E94C4578AE38EBD0DB407FEFDCF09C062
:101EB0001EBC0DB407FEFDCF8EB5F80181938F01D6
:101EC00021972097A9F70E947D0EDF91CF911F9156
:101ED0000F9108950F931F93DF93CF9300D000D0FD
:101EE00000D0CDB7DEB789E30E94FF0E882319F436
:101EF00000E010E048C06091A6027091A70280E067
:101F00000E94CF0E86E090E0BE016F5F7F4F0E947F
:101F1000460F89819A819093A7028093A6022B8114
:101F20003C81E091A102F091A2028D8187FD03C066
:101F300000E010E00EC0245030408F0101501040EE
:101F40002017310708F48901C8016EEE72E00E9483
:101F5000460FF801E251FD4F10826091A602709188
:101F6000A7028CE06130780724F08CE06FEF7BE013
:101F700003C0615070408CE00E94CF0E80E86EE19B
:101F800040E40E94840EC80126960FB6F894DEBF86
:101F90000FBECDBFCF91DF911F910F9108950F9389
:101FA0001F93CF93DF938C01EB01F8948091A402EF
:101FB00060E00E94C4578AE78EBD0DB407FEFDCFD6
:101FC00008C088818EBD0DB407FEFDCF219601505B
:101FD000104001151105A9F70E947D0EDF91CF91E8
:101FE0001F910F910895CF93DF93EC018CE10E9434
:101FF000FF0E81FF0FC080E86FE140E80E94840E71
:1020000080EA6FE140E80E94840E80EA6CE142E0E1
:102010000E94840E82E060E07CE00E94CF0EBE0150
:102020006050744F86E00E94CF0E8AE760E040E087
:102030000E94840ECE016EEE72E00E94CF0F80E807
:102040006FE148E00E94840EDF91CF91089584E013
:1020500061E00E94855784E061E00E94C45785E0FA
:1020600061E00E94855787E061E00E94855786E025
:1020700060E00E94855785E061E00E94C45785E0DA
:1020800060E00E94C45787E060E00E94C45780E58A
:102090008CBD8DB581608DBD0895EF92FF920F9339
:1020A0001F93CF93DF93EB01142F9093A2028093A1
:1020B000A1020CB406FC02C00E9427101093A402D7
:1020C000812F61E00E9485570E947D0E8FEF60E0B6
:1020D0004FEF0E94840E62E070E080E090E00E948A
:1020E000E7560E94D9567B018C0180E395E7A0E07A
:1020F000B0E0E80EF91E0A1F1B1F09C00E94D95646
:10210000E616F7060807190710F480E084C080E09F
:102110006DE10E94DD0E882389F31092A7021092D0
:10212000A60288E060E070E00E94CF0E8CE060E0E4
:1021300070E00E94CF0E8AE06FEF7BE00E94CF0E2E
:1021400084E060E07CE00E94CF0E86E06FEF71E1FA
:102150000E94CF0E80E00E941A0F88E26FE370E3C6
:102160000E94CF0E80E369EF77EF0E94CF0E80ECE4
:102170006DE00E94C10E81EC60E00E94C10E80E81B
:1021800062EC42E30E94840E86EC62E17CE00E94F5
:10219000CF0E84EC62E10E94C10E8AEC6AEE75E01B
:1021A0000E94CF0E84EE68810E94C10E85EE698187
:1021B0000E94C10E82EE6A810E94C10E83EE6B8185
:1021C0000E94C10E80EE6C810E94C10E81EE6D8175
:1021D0000E94C10E84ED60E10E94C10E86ED60E0B8
:1021E00071E00E94CF0E8AEE0E94FF0E80FDFBCFB1
:1021F0008FE10E94A00E80E86BE140EC0E94840E0B
:1022000080E86FE144E00E94840E82E70E94FF0EA6
:10221000863008F08F5FDF91CF911F910F91FF9073
:10222000EF900895EF92FF920F931F93CF93DF9358
:10223000FC01EB018A0179011092EA02009729F072
:102240008EEC92E0BF010E944455209719F0CE0118
:102250000E94A9480115110529F082EE92E0B8010B
:102260000E944455E114F10429F082ED92E0B70197
:102270000E9444550E94BF471092ED021092EC025A
:1022800081E0DF91CF911F910F91FF90EF90089522
:10229000AF92BF92CF92DF92FF920F931F93CF9393
:1022A000DF938C01EB01F42E1092EA0238E341E057
:1022B00050E060E070E018C0832F90E0FC01B3E0D4
:1022C000F595E795BA95E1F7E855FD4F8770907061
:1022D0005A016B0104C0AA0CBB1CCC1CDD1C8A95E6
:1022E000D2F720812A292083315031F788EC92E0FF
:1022F000BE010E943C55C80168EC72E04F2D0E945F
:102300004D10DF91CF911F910F91FF90DF90CF90F3
:10231000BF90AF900895CF92DF92EF92FF920F930C
:102320001F93DF93CF93CDB7DEB7EB84FC84CD84CE
:10233000DE84DE011F9601C0D801F6018491882356
:1023400009F4BCC00894C11CD11C843209F099C0A6
:10235000F6010894C11CD11C8491863409F45FC035
:10236000873434F4843469F0853409F08AC06EC04F
:102370008C34C9F1833509F445C0883409F081C033
:102380000DC08D010E5F1F4FF701668177818D9122
:102390009C914AE050E00E948D087EC02C91822FD3
:1023A000992787FD909514E0959587951A95E1F703
:1023B0008F702F702A300CF0295F8A300CF0895F03
:1023C0008D010E5F1F4FF701A681B781805DFD0172
:1023D0008193205D11962C933196D7011796FC932B
:1023E000EE931697A9CF8D010C5F1F4F6D917D91D4
:1023F0008D919C91F701468157812AE030E00E943F
:10240000CB084AC08D010E5F1F4F6D917C91D701A3
:1024100016968D919C9117970E9431083DC08D01B1
:102420000E5F1F4F2D913C910AC0D7011696ED917A
:10243000FC91179781931796FC93EE931697F901E9
:102440002F5F3F4F8491882381F776CF8D010E5FF8
:102450001F4F2D913C910AC0D7011696ED91FC912A
:10246000179781931796FC93EE931697F999FECFE1
:1024700032BD21BDF89A80B52F5F3F4F882361F7A9
:102480005BCFF70126813781F90181939F01F70125
:10249000378326838D0150CFD70116968D919C915D
:1024A0001797FC0101900020E9F73197E81BF90B21
:1024B0008E0F9F1FF701978386833ECFCF91DF91C9
:1024C0001F910F91FF90EF90DF90CF9008950F93A1
:1024D0001F938C01FC01878160E00E94C45781E05A
:1024E00090E00E944057F801878161E00E94C45744
:1024F00081E090E00E944057F801878160E00E94EF
:10250000C45784E690E00E9440571F910F910895B0
:10251000CF92DF92EF92FF920F931F93CF93DF93AF
:102520007C01FC0184818823F9F48701C0E0D0E0BC
:10253000C62EDD24F801808561E00E948557B60132
:102540000C2E02C0759567950A94E2F76170F80148
:1025500080850E94C45721960F5F1F4FC430D1055C
:1025600049F7C7010E946712DF91CF911F910F9128
:10257000FF90EF90DF90CF9008951F93CF93DF935C
:10258000EC01162F8C818823C1F48D81642F0E9469
:10259000C4578E818F3F19F060E00E94C457612FAD
:1025A00070E084E0759567958A95E1F7CE010E9409
:1025B0008812CE01612F0E948812DF91CF911F9166
:1025C000089541E00E94BD1281E090E0089540E04E
:1025D0000E94BD120895EF92FF920F931F93CF9325
:1025E000DF938C017A016770660F660F660F606477
:1025F0000E94E712C0E0D0E0D801ED91FC91D70134
:10260000AC0FBD1F0190F081E02DC8016C910995C0
:102610002196C830D10581F7DF91CF911F910F919D
:10262000FF90EF900895FC0161896E7F618B686077
:102630000E94E7120895FC016189862F8460818BD6
:102640006C60CF010E94E7120895DF93CF93CDB75E
:10265000DEB728970FB6F894DEBF0FBECDBF9C0142
:10266000FE013196AAE2B2E088E00D90019281501D
:10267000E1F7F9018481882329F48489481710F04F
:10268000482F4150E42FF0E0EE0FFF1FEC0FFD1F2D
:102690008181680F6068C9010E94E71228960FB611
:1026A000F894DEBF0FBECDBFCF91DF91089561E0FA
:1026B0000E94E71280ED97E00E9440570895CF9363
:1026C000DF93EC018C81882309F061C088898860E0
:1026D000888B82E08C8B1D8A80E593EC0E944057AA
:1026E0008D8160E00E94C4578F8160E00E94C457D2
:1026F0008E818F3F19F060E00E94C457688964FDA5
:102700001DC0CE0163E00E94881284E991E10E941D
:102710004057CE0163E00E94881284E991E10E9453
:102720004057CE0163E00E94881286E990E00E9443
:102730004057CE0162E00E94881216C06062CE014E
:102740000E94E71284E991E10E9440576889606223
:10275000CE010E94E71286E990E00E944057688906
:102760006062CE010E94E71268896062CE010E9419
:10277000E71284E0898BCE010E941B13CE010E94D8
:10278000571382E08A8BCE0166E00E94E712DF9148
:10279000CF9108956F927F928F92AF92CF92EF92E6
:1027A0000F93DF93CF93CDB7DEB73C01FC01458398
:1027B00026830783E086C186A28683868C858487EC
:1027C0008D8585878E8586878F85878782EA9BE0C2
:1027D0000E94B45CF3011482858161E00E948557F8
:1027E000F30186818F3F19F061E00E948557F30164
:1027F000878161E00E94855788E0F301808BCF914B
:10280000DF910F91EF90CF90AF908F907F906F906E
:102810000895FC01A681B7816D93B783A68381E0FB
:1028200090E008951F920F920FB60F9211242F93EC
:102830003F934F935F936F937F938F939F93AF9348
:10284000BF93EF93FF938091F5068F5F8093F5061A
:102850008091F506803128F0E091F306F091F406BE
:102860000995FF91EF91BF91AF919F918F917F91CA
:102870006F915F914F913F912F910F900FBE0F90ED
:102880001F9018958091DA0790E023E0880F991F38
:102890002A95E1F78552984FEBEDF7E003C01582DA
:1028A00014823896E817F907D0F3089589E18093E8
:1028B000AF061092B2061092C6061092CD06109284
:1028C000CF061092EA061092E90686E392E0909312
:1028D000E8068093E7060895AF92BF92CF92DF9209
:1028E000EF92FF920F931F938091C101882309F407
:1028F00040C090911107892F829586958770C9F500
:102900008091100783FD35C090FF33C00E94DD50D9
:102910005B016C01809111078E7F8093110780917C
:10292000F606882329F48CE790E061E00E940323F7
:102930000E9487327B018C0161157105810591052B
:10294000C1F00E94B050C801B7010E94380E21E8C2
:10295000A21628ECB2062FE4C2062AE3D20648F4F7
:102960000E94DD506158784C8F449A4310F00E94C9
:10297000C0201F910F91FF90EF90DF90CF90BF90FC
:10298000AF900895EF92FF920F931F938091D4011F
:10299000823099F50E94D9569B01AC0180912D0798
:1029A00090912E07A0912F07B091300779018A01ED
:1029B000E81AF90A0A0B1B0BD801C701C297A10537
:1029C000B105D8F08091EF069091F006A091F10644
:1029D000B091F2060196A11DB11D8093EF06909370
:1029E000F006A093F106B093F20620932D073093E2
:1029F0002E0740932F07509330071F910F91FF90A0
:102A0000EF900895EF92FF920F931F93809110071C
:102A100083FD6AC08091110781FF66C08D7F80931E
:102A200011078091F606882359F48FEB97E06FE049
:102A300041E00E9425138FEB97E064E00E94E112D1
:102A40008AED92E00E94A94A0E94D9567B018C012E
:102A50000E946A0F0E94F64A8AED92E00E946B4D36
:102A6000882361F40E94D9566E197F09800B910B5F
:102A7000683C71058105910558F323C080911107C9
:102A80008F7102C08F71806C809311078091110744
:102A900082958695877090E08630910534F080911C
:102AA00010078064809310071FC00397ECF00E940A
:102AB000BC2D8823C9F0809111078F718093110775
:102AC00013C080911107982F9295969597709F5FEC
:102AD0009770292F2295220F207E8F71822B809351
:102AE0001107973079F2D2CF1F910F91FF90EF909D
:102AF0000895EF92FF920F931F938C018EEA96E058
:102B000060E071E040E00E94EB6934EBE32E37E0D7
:102B1000F32EC701B8010E9431080EE317E0C80187
:102B200068EB71E00E943108C801B7010E941B08E0
:102B3000C8016DEA70E00E94EC071F910F91FF90B1
:102B4000EF900895CF93DF93EC018091E301882308
:102B500061F18091100785FF28C0CE0162E071E02D
:102B600043E050E00E943808009771F48EEA96E046
:102B700068EB71E040E00E94EB698823B1F08DECD6
:102B800096E00E949D6211C0CE010E9479158EEAE6
:102B900096E06EE377E00E94E769882331F08EEAE1
:102BA00096E06EE377E00E94C469DF91CF910895CB
:102BB0007F928F929F92AF92BF92CF92DF92EF92CD
:102BC000FF920F931F93DF93CF93CDB7DEB76E972E
:102BD0000FB6F894DEBF0FBECDBF782E4A015B0161
:102BE0008091E301882309F44BC1CB01BA0120E8AD
:102BF00031E541E050E00E942F75CA01B9014EE372
:102C000057E02AE030E00E94CB088EE397E00E9474
:102C100079158091100785FF33C18EEA96E060E058
:102C200071E040E00E94EB698EEA96E068EB71E0AB
:102C300040E00E94EB69882351F48EEA96E068EB4D
:102C400071E041E00E94C869882309F419C11D821E
:102C50001F821C821B828BE792E09A8389838E01FC
:102C60000B5F1F4F4EE3C42E47E0D42EC801B601C0
:102C700042E40E943568F82E4F89588D698D7A8D0F
:102C8000C8010E94BC5DFF2009F4FAC0C6016BEACE
:102C900070E00E94F7077720E1F5F601019000202F
:102CA000E9F73197EC19FD09EC0DFD1D80918C09B8
:102CB00090E0BF014AE050E00E948D08C60169EA39
:102CC00070E00E94EC07F60101900020E9F73197CF
:102CD000EC19FD09EC0DFD1D80918B0990E0BF0101
:102CE0004AE050E00E948D08C60167EA70E00E9449
:102CF000EC07F60101900020E9F73197EC19FD0986
:102D000060918D0970918E0980E090E0EC0DFD1DC1
:102D10008DC084E07816A9F48091EF069091F006BA
:102D2000A091F106B091F206209125073091260777
:102D30004091270750912807281739074A075B0752
:102D400020F0CC24DD2476010CC0C090EF06D0909A
:102D5000F006E090F106F090F206C21AD30AE40AF7
:102D6000F50A0EE317E0F80101900020E9F731972A
:102D7000E01BF10BE00FF11FC701B601AF012AE024
:102D800030E00E94CB08C80164EA70E00E94EC07C2
:102D900063E0769EB001112465577F4FC8010E9401
:102DA000EC07C80161EA70E00E94EC0782E0781647
:102DB00099F0871510F081E004C083E0781601F1E6
:102DC00084E0781639F5609121077091220780918F
:102DD00023079091240708C0609131077091320752
:102DE0008091330790913407681579058A059B0512
:102DF00070F475016401C61AD70AE80AF90A0AC014
:102E00008091D601C82EDD24EE24FF2403C0CC24FB
:102E1000DD247601EEE3F7E001900020E9F7319739
:102E2000EE53F740E25CF84FC701B601AF012AE06C
:102E300030E00E94CB080EE317E0C8016FE970E0B4
:102E40000E94EC07F80101900020E9F73197E01BA0
:102E5000F10BE00FF11FC501B401AF012AE030E032
:102E60000E94CB08C8016BE970E00E94EC07CE011C
:102E70000196B8010E94906ACE0105960E942460D6
:102E80006E960FB6F894DEBF0FBECDBFCF91DF9127
:102E90001F910F91FF90EF90DF90CF90BF90AF9078
:102EA0009F908F907F9008950E94EE2A0E94312B70
:102EB0000E94963108952F923F924F925F926F92A7
:102EC0007F928F929F92AF92BF92CF92DF92EF92BA
:102ED000FF920F931F93DF93CF9300D000D0CDB715
:102EE000DEB72B013C014B015C010894811C911C55
:102EF000A11CB11C8091D0010E94705220919309B5
:102F000030919409409195095091960942165306C3
:102F10006406750618F07501640109C06C01EE24A1
:102F2000D7FCE094FE2CC20ED31EE41EF51E0091C9
:102F3000EA016BED262E67E0362E9C01442737FD13
:102F40004095542F29833A834B835C8361C0F10100
:102F500080819181A281B3810097A105B10509F01B
:102F600053C084819581892B09F44EC01681812F2D
:102F700086958695869590E08C53984F0E945121B6
:102F800090E0177002C0959587951A95E2F780FF3B
:102F90004EC0002309F04BC0F101C082D182E28211
:102FA000F38284819581A0E0B0E029813A814B8150
:102FB0005C81820F931FA41FB51FC80ED91EEA1E85
:102FC000FB1E8091100783FD1FC08860809310074F
:102FD0008091D4018230C1F48091EF069091F00687
:102FE000A091F106B091F2068093250790932607F1
:102FF000A0932707B09328074092210750922207F9
:10300000609223077092240748E050E0240E351E9A
:103010008091DA0790E053E0880F991F5A95E1F705
:103020008552984F2816390608F491CF0BC0F1014C
:1030300080829182A282B3820894811C911CA11C7F
:10304000B11CBFCF0F900F900F900F90CF91DF91D9
:103050001F910F91FF90EF90DF90CF90BF90AF90B6
:103060009F908F907F906F905F904F903F902F90A8
:1030700008956F927F928F929F92AF92BF92CF925C
:10308000DF92EF92FF920F931F93DF93CF93CDB711
:10309000DEB7C754D0400FB6F894DEBF0FBECDBF29
:1030A000A82E0E9454178A2D81508E3F28F4BE010D
:1030B0006F5F7F4F0E94DD309924BB24BEEF8B2EC3
:1030C000ACE06A2E712C6C0E7D1E41C0CB2CDD2431
:1030D0008FEFA81631F4F2E0EF2EF12C012D112D17
:1030E00012C0AA2009F43FC0F301EC0DFD1D808140
:1030F0000E9400520E942D527B018C0161157105C6
:103100008105910519F1E3E0D694C794EA95E1F7BA
:10311000C6018254984F0E94512190E02B2D2770B8
:1031200002C0959587952A95E2F780FD0FC00E9411
:10313000712EFC01009751F01082118212821382CD
:10314000F582E482B682878299249394B394809125
:103150001A07B81608F4BACF992059F00E94952B97
:103160000E945B1706C07CE3E72EF12C012D112D88
:10317000CACFC95BDF4F0FB6F894DEBF0FBECDBF1D
:10318000CF91DF911F910F91FF90EF90DF90CF9043
:10319000BF90AF909F908F907F906F900895CF9247
:1031A000DF92EF92FF920F931F93CF93DF93D82E6E
:1031B0007A018B0160E00E94B52ACD2DD0E0FE019E
:1031C000E55AF64FC0808091DA07C81608F041C072
:1031D000EC2DF0E083E0EE0FFF1F8A95E1F7E5525A
:1031E000F84F40815181628173814E155F05600700
:1031F000710740F59E012F5F3F4F8091120790E0CD
:1032000082179307F9F08091130790E082179307D4
:10321000C9F0D0928B09878180938C09C701841BE8
:10322000950B90938E0980938D09E0928F09F0920F
:103230009009009391091093920980E0B801A701C9
:103240000E94D8158C2D0E948C2EC55AD64F8FEF18
:103250008883DF91CF911F910F91FF90EF90DF90C6
:10326000CF9008958F929F92AF92BF92CF92DF92AC
:10327000EF92FF920F931F93CF93DF935B016C014B
:103280008091100788248394882281FD09C082FDE3
:1032900002C0EE2407C0EE248091D401813011F4E5
:1032A000EE24E394FF2449C00F2D10E0C8018E5492
:1032B000984F0E9451219F2C990C990C990CC0E0B9
:1032C000D0E0082F10E0492D4C0FE42FF0E09F01D3
:1032D0002F5F3F4F8091120790E08217930741F1D3
:1032E0008091130790E08217930711F1E55AF64F8A
:1032F000E081EF3FE9F0F0E093E0EE0FFF1F9A95D9
:10330000E1F7E552F84F8781833690F4882059F031
:10331000EE2071F0C8010C2E02C0959587950A9495
:10332000E2F780FD05C0842FB601A5010E94CF18E9
:103330002196C830D10539F6F39480911907F81613
:1033400008F4B2CFDF91CF911F910F91FF90EF90D2
:10335000DF90CF90BF90AF909F908F900895809115
:10336000110782958695877009F04FC080911007EC
:1033700083FD4BC08091EA01882309F046C00E947A
:10338000952B20913A0730913B0740913C07509193
:103390003D072115310541055105B9F02F553E4A2C
:1033A0004E4F5F4F261737074807590770F41092A2
:1033B0003A0710923B0710923C0710923D0780910C
:1033C000100780648093100708952091360730918C
:1033D00037074091380750913907211531054105CC
:1033E000510549F02F5E314F4F4F5F4F261737077A
:1033F0004807590750F46093360770933707809356
:103400003807909339070E949653089584B7877FB1
:1034100084BF0E944E2C0E944A270E94A9316CE36F
:1034200070E080E090E00E94A75088E59EE00E9456
:1034300050510E94952B0E94CF2B80916000886193
:103440008093600081E280936000809160008064DE
:10345000809360000E94BC2D882321F08091110789
:103460008F7104C0809111078F7180628093110762
:10347000809111078D7F8160809311070E94312B0D
:103480008FE0809335070895FF920F931F93DF938A
:10349000CF93CDB7DEB7C754D0400FB6F894DEBF98
:1034A0000FBECDBF80913507882321F40E9487216C
:1034B0001092F60682E00E94F321F82E082F10E009
:1034C00086FF24C18FE08093350781E00E94872129
:1034D0008091F606833020F4813008F0D3C004C018
:1034E000833009F013C1C2C0C8018F709070823060
:1034F000910509F45AC08430910509F494C00197EC
:1035000009F004C1F7FE30C08DE10E941858892BE4
:1035100021F48FEF0E943918F9C08EE10E941858EB
:10352000892B69F08091DA0790E023E0880F991FDA
:103530002A95E1F78552984FEBEDF7E011C08AED3F
:1035400092E060E00E9459258FEB97E060E041E057
:103550000E9425138FE091E022C0158214823896D4
:10356000E817F907D0F3D2C08EEC92E060E00E9439
:1035700059258FEB97E060E041E00E9425138DE034
:1035800091E00E94B1226091B6017091B7018FEB7A
:1035900097E04AE050E00E94735B85E091E00E9472
:1035A000B12281E08093F606B1C0F7FE32C08FE110
:1035B0000E941858892B71F48CE097E061E00E941A
:1035C00059258FEB97E060E041E00E9425138FEFD3
:1035D00090E0E5CF8DE10E941858892BB9F48FEB6C
:1035E00097E00E94571360913A0770913B078091D2
:1035F0003C0790913D070E94CF2B8FEB97E060E056
:1036000041E00E94251388EF90E0C9CF0E94C020BE
:103610007DC08FEB97E00E94571388EC92E00E94E8
:10362000C12282E0BFCFF7FE0CC089EE90E060E0DF
:103630000E94032388ED90E061E00E94032383E071
:10364000B1CF20911107822F86958695877090E0E3
:1036500060911907019670E00E941C758770880FB1
:10366000880F237E282B2093110750C00F701070F5
:103670000430110509F04AC0F7FE07C08091030726
:103680000E9439181092F60641C08091030790E01D
:103690006091D90770E06F5F7F4F01960E941C75A3
:1036A0008093030787EC90E060E00E940323809101
:1036B0000307882331F18150BE016F5F7F4F0E9465
:1036C000DD3085EC90E061E00E9403238FEB97E012
:1036D00060E041E00E942513609103078FEB97E0C3
:1036E00070E04AE050E00E94C45B82EC90E00E94EF
:1036F000B1228FEB97E0BE01645C7F4F0E94D75BE5
:1037000005C082EB90E061E00E940323C95BDF4FBC
:103710000FB6F894DEBF0FBECDBFCF91DF911F91E2
:103720000F91FF9008952F923F924F925F926F9268
:103730007F928F929F92AF92BF92CF92DF92EF9241
:10374000FF920F931F93DF93CF93CDB7DEB7CF5484
:10375000D0400FB6F894DEBF0FBECDBF8091D1012F
:10376000809312078091E401809313070E94952BA8
:103770004B015C010E946A0F0E94F64A009721F0FB
:1037800082519D4F0E94EB3DA8951092F5060E9434
:10379000441A8091FF0690910007A0910107B09113
:1037A000020788159905AA05BB0509F4BAC48092D9
:1037B000FF0690920007A0920107B0920207809145
:1037C0003507882319F08150809335078091F606DC
:1037D000882321F40E94952B0E94CF2B8091100703
:1037E00081FF10C08091080790910907A0910A07F6
:1037F000B0910B0788169906AA06BB0690F00E94A6
:10380000AE260FC08091080790910907A0910A0782
:10381000B0910B0788169906AA06BB0610F40E9401
:10382000BE26909110079695917080911407869509
:1038300081708917C9F0992349F0809231079092DD
:103840003207A0923307B092340705C082E0B50179
:10385000A4010E94D81590911007927080911407CE
:103860008D7F892B809314078091D4018130B9F525
:103870000E943C22909110079695969591708091A8
:103880001407869586958170891749F1992349F027
:103890008092210790922207A0922307B0922407DA
:1038A00015C08091210790912207A0912307B09124
:1038B00024070A96A11DB11D88159905AA05BB0507
:1038C00028F481E0B501A4010E94D8159091100759
:1038D0009470809114078B7F892B80931407C50106
:1038E000B4012CE330E040E050E00E942F757901F4
:1038F0008A018091FB069091FC06A091FD06B09193
:10390000FE06E816F9060A071B0709F49FC0E092B5
:10391000FB06F092FC060093FD061093FE0655246C
:1039200066241E010894211C311C85C0862DB1011E
:103930000E94DD30C101B501A4010E94313088230D
:1039400009F478C07724462C43946FC0272D30E0CB
:10395000A9014F5F5F4F8091120790E08417950790
:1039600009F462C08091130790E08417950709F469
:103970005BC00CE010E00C0F1D1F020F131FD801DD
:103980008C91882309F450C053E0369527955A95B9
:10399000E1F7C9018254984F0E94512190E0272DF0
:1039A000277002C0959587952A95E2F780FD3CC067
:1039B000F80180810E9400520E942D526B017C010F
:1039C000898181FF1DC01091D601212F30E040E098
:1039D00050E0C701B6010E94DD7424E630E040E00B
:1039E00050E00E942F75C901DA016C017D0114318C
:1039F00038F4FAE0CF16D104E104F104A8F005C0D0
:103A0000C114D104E104F10479F00E94712EFC018B
:103A1000009751F01082118212821382D582C482E3
:103A20007682478255245394739480911A077816AE
:103A300008F48CCF63948091D907681608F476CF88
:103A4000552021F0C501B4010E945B178091100739
:103A500083FF81C18091DA07E82EFF2443E0EE0C5A
:103A6000FF1C4A95E1F78BED97E0E80EF91E8C01FB
:103A7000DD2429C0D80116968C911697682F70E026
:103A8000FB01E55AF64FE081EF3FB1F0F0E033E0A3
:103A9000EE0FFF1F3A95E1F7E552F84F2081318193
:103AA000428153818D919D910D90BC91A02D28173D
:103AB00039074A075B0720F0655A764FFB01D08231
:103AC000085F1F4FD3940E151F05A0F2CC247EC0B3
:103AD0008C2D90E0FC01E55EF84F20815C2C550CAC
:103AE000550C550CEE24FF24622E7724D52CDE0CC9
:103AF000ED2DF0E09F012F5F3F4F8091120790E086
:103B00008217930709F459C08091130790E0821738
:103B1000930709F452C0E55AF64F80818F3F09F4AC
:103B20004CC0082F10E023E0000F111F2A95E1F789
:103B30000552184FD8012D913D914D915C911397ED
:103B40002115310541055105A1F014968D919C91E7
:103B50001597A0E0B0E0820F931FA41FB51F881631
:103B60009906AA06BB0628F08D2DB501A4010E9476
:103B7000CF18C3010E2C02C0959587950A94E2F7E1
:103B800080FD1BC0F8012081318142815381821662
:103B90009306A406B50688F084819581A0E0B0E084
:103BA000820F931FA41FB51F88169906AA06BB068D
:103BB00020F48D2D61E00E94B52A0894E11CF11CCF
:103BC000F8E0EF16F10409F091CFC3948091190742
:103BD000C81608F47DCF8091DA07082F10E0015055
:103BE0001040780193E0EE0CFF1C9A95E1F78BED05
:103BF00097E01EC0D70114968D919C911597009760
:103C000081F0A0E0B0E0F701208131814281538151
:103C1000820F931FA41FB51F88169906AA06BB061C
:103C200018F0802F0E948C2E0150104088EF9FEFDB
:103C3000E80EF91E9FEF0F3F1907E1F6C501B40129
:103C40000E9432190E94312B10929309109294090C
:103C500010929509109296096090EA018BEDC82E9A
:103C600087E0D82E4BC0D60116967C9016971496F6
:103C70008D919C9115977C0100E010E08D919D91B4
:103C80000D90BC91A02DE80EF91E0A1F1B1F8E146B
:103C90009F04A006B10670F5872D869586958695BA
:103CA00090E08C53984F0E94512190E0B7E07B2226
:103CB00002C0959587957A94E2F780FF1BC0662035
:103CC000C9F420919309309194094091950950913C
:103CD0009609D801C701E216F3060407150710F488
:103CE000DA01C9018093930990939409A0939509EF
:103CF000B0939609E8E0F0E0CE0EDF1E2091DA07DF
:103D0000822F90E003E0880F991F0A95E1F7855212
:103D1000984FC816D90608F4A6CF2223E1F40E94D2
:103D2000EE2A0E94312B0E94963180911007877FE6
:103D3000809310078091D401823029F484E0B5018A
:103D4000A4010E94D8158091D1018093120780911F
:103D5000E4018093130780911207882309F48CC033
:103D60001091D2010091D3018CEA97E06EE377E0E5
:103D70000E942D2730901A07E0901207CE2CDD24E8
:103D8000FF2461E070E0812F90E0A0E0B0E0609659
:103D90008CAF9DAFAEAFBFAF6097402E5524662469
:103DA000772462C02F2D30E0C616D70609F459C01B
:103DB000D90113E0B695A7951A95E1F74F2D4770F5
:103DC000FD01E55EF84F808190E0042E02C09595DC
:103DD00087950A94E2F780FF44C0A25CB84F8C91AB
:103DE000992787FD909502C0959587954A95E2F7AA
:103DF00080FF37C0255A364FD9018C91E82FF0E06B
:103E0000A3E0EE0FFF1FAA95E1F7E552F84F2081DE
:103E100031814281538160968CAD9DADAEADBFAD19
:103E20006097820F931FA41FB51F88169906AA06D4
:103E3000BB06B8F02C5330404040504084819581FF
:103E4000A0E0B0E0280F391F4A1F5B1F240D351D6D
:103E5000461D571D281539054A055B0510F061E020
:103E600007C0F3946F5F7F4FF31408F49BCF60E0BB
:103E70008E2D81500E94B52A80911307882309F462
:103E80008CC01091E5010091E60188EB97E06EE3AC
:103E900077E00E942D2730901A07E0901307CE2C70
:103EA000DD24FF2461E070E0812F90E0A0E0B0E02D
:103EB0002C968CAF9DAFAEAFBFAF2C97402E552444
:103EC0006624772462C02F2D30E0C616D70609F489
:103ED00059C0D90153E0B695A7955A95E1F74F2DF2
:103EE0004770FD01E55EF84F808190E0042E02C02E
:103EF000959587950A94E2F780FF44C0A25CB84F7D
:103F00008C91992787FD909502C0959587954A9544
:103F1000E2F780FF37C0255A364FD9018C91E82F40
:103F2000F0E043E0EE0FFF1F4A95E1F7E552F84F4E
:103F300020813181428153812C968CAD9DADAEADF7
:103F4000BFAD2C97820F931FA41FB51F881699062B
:103F5000AA06BB06B8F02C53304040405040848144
:103F60009581A0E0B0E0280F391F4A1F5B1F240D88
:103F7000351D461D571D281539054A055B0510F0EE
:103F800061E007C0F3946F5F7F4FF31408F49BCF99
:103F900060E08E2D81500E94B52AC501B4010E94B7
:103FA00032190E94312B8091F606882389F4C501CD
:103FB000B40123E030E040E050E00E942F759B0107
:103FC000AC01265C3D4F81E0F90160810E94A22492
:103FD0008091100786FF22C083FD20C010E03E01C3
:103FE0000894611C711C3CE3C32ED12CE12CF12CF4
:103FF000C80CD91CEA1CFB1C0CC0812FB3010E9409
:10400000DD30C301B701A6010E943130882331F4AD
:104010001F5F8091D907181780F380C08091D40169
:10402000823009F04BC0C501B4012EE130E040E020
:1040300050E00E942F756115710581059105F1F51C
:104040008091EF069091F006A091F106B091F206F2
:104050002091F7063091F8064091F9065091FA0642
:10406000281739074A075B0728F080E090E0A0E0B6
:10407000B0E00CC08091EF069091F006A091F1069F
:10408000B091F206821B930BA40BB50B809329070A
:1040900090932A07A0932B07B0932C078091EF06EB
:1040A0009091F006A091F106B091F2068093F70688
:1040B0009093F806A093F906B093FA06C501B401EF
:1040C00023E831E541E050E00E942F75611571054C
:1040D0008105910529F48091110781608093110772
:1040E0000E946C1481149104A104B10491F0C501E3
:1040F000B40129E532E040E050E00E942F756115DF
:1041000071058105910529F48091110782608093E2
:1041100011070E9402150E94AF1903C00E94C0201F
:104120007DCFC15BDF4F0FB6F894DEBF0FBECDBFB2
:10413000CF91DF911F910F91FF90EF90DF90CF9083
:10414000BF90AF909F908F907F906F905F904F90B7
:104150003F902F9008959C01F999FECF32BD21BD6B
:10416000F89A80B508959C01F999FECF1FBA32BD27
:1041700021BD60BD0FB6F894FA9AF99A0FBE089562
:10418000E091D507F091D60709950895EF92FF9237
:104190000F931F93FC0120E030E040E050E070E01E
:1041A00038C0908179018A0184E0EE0CFF1C001F69
:1041B000111F8A95D1F7892F80538A3030F4892FC7
:1041C000992787FD9095C09719C0892F8154863013
:1041D00030F4892F992787FD9095C7970FC0892FB5
:1041E0008156863028F020E030E040E050E013C0F7
:1041F000892F992787FD9095875590409C014427EA
:1042000037FD4095542F2E0D3F1D401F511F7F5FDE
:104210003196761730F2B901CA011F910F91FF90C4
:10422000EF900895EF92FF920F931F93CF93DF9338
:10423000EC018B017A0166E00E94C62061157105D0
:104240008105910521F10115110529F0F80160831F
:10425000718382839383CE01069666E00E94C62016
:10426000611571058105910591F0E114F10429F0C2
:10427000F7016083718382839383CE010C9664E09F
:104280000E94C620611571058105910511F460E059
:1042900070E0CB01DF91CF911F910F91FF90EF90D4
:1042A00008959C01F999FECF32BD21BDF89A80B5E1
:1042B0000895FC0120EF33E084E02431380711F445
:1042C00040E009C0F999FECFC901019632BD21BD78
:1042D000F89A40B59C019081442331F0992349F02C
:1042E000491739F43196E8CF80E0992319F481E039
:1042F000089580E0089508951092C2071092C107B2
:1043000086E292E09093C0078093BF0708951F93C1
:10431000182F8091C307882391F48CE061E00E94FC
:104320008557112319F08091DB0102C08091DC01D7
:104330006FEF70E0681B71098CE00E9431561F918D
:1043400008958091C307882351F48DE061E00E94B5
:1043500085576091DA018DE070E00E943156089532
:10436000EF92FF920F931F93CF93DF93E82E162FB8
:10437000042FF22E662321F0623081F4222371F0A3
:104380008E2D0E941858892B11F000E024C0FF20C8
:1043900011F480E001C080E8082B1DC0C0E0D0E02F
:1043A0008E2D0E941858892B81F4113031F0123073
:1043B00061F483E0C83ED80744F461E070E080E037
:1043C00090E00E94E7562196EBCFFF2019F4C85EDB
:1043D000D3400CF00068802FDF91CF911F910F9197
:1043E000FF90EF9008950F931F93082F1091D70718
:1043F000107861E070E080E090E00E94E7568FE185
:104400000E941858892B21F48FE1602F41E013C0DE
:104410008EE10E941858892B21F48EE1602F42E032
:104420000AC08DE10E941858892B11F040E007C0A6
:104430008DE1602F44E0212F0E94B021482F809110
:10444000D70790E08F709070242F30E0892B39F4DB
:104450002F703070232B71F0842F806406C02F7072
:104460003070232B39F4842F80624093D7071F913B
:104470000F910895842FF9CF8091D401813099F460
:104480008BE00E94185840E02091D50130E082175F
:10449000930709F041E0440F440F809110078B7F90
:1044A000842B8093100708951F93182F843690F063
:1044B00064E60E94FC74682F8FEB97E070E04AE09E
:1044C00050E00E94C45B8FEB97E066E071E00E94D1
:1044D000D75B02C08A30A0F0812F6AE00E94FC7492
:1044E0000E94FC74692F8FEB97E070E04AE050E087
:1044F0000E94C45B8FEB97E066E071E00E94D75B9F
:10450000812F6AE00E94FC74692F8FEB97E070E0C6
:104510004AE050E00E94C45B1F910895EF92FF9221
:104520000F931F938C019FEBE92E97E0F92EC801A2
:104530006AE070E00E941C75C7014AE050E00E94EA
:10454000C45BC8016AE070E00E941C75BC01C70131
:104550004AE050E00E94C45B1F910F91FF90EF90E2
:104560000895CF93DF93EC0104C08FEB97E00E9496
:10457000E45AFE01219664916623B9F7DF91CF9149
:1045800008950F931F93CF93DF93182F092F8FEB6D
:1045900097E060E040E00E942513212F302FC901F1
:1045A000EC0110E005C088E495E00E94B12221965C
:1045B000688170E024E0759567952A95E1F78FEBA7
:1045C00097E040E150E00E94C45B688170E06F704A
:1045D00070708FEB97E040E150E00E94C45B1430B4
:1045E00031F48FEB97E060E041E00E9425131F5FFC
:1045F0001630C9F681E495E00E94B122DF91CF9197
:104600001F910F9108950F931F93CF93DF938C0108
:10461000462F8FEB97E060E00E942513E80104C06D
:104620008FEB97E00E94E45A9E01201B822FFE012F
:10463000219664916623A1F7992787FD9095C0E1A3
:10464000D0E0C81BD90B05C082E795E00E94B122DB
:104650002197D7FFF9CFDF91CF911F910F91089547
:10466000EF92FF920F931F93CF93DF937C01BC01D6
:1046700054E0660F771F5A95E1F7645F7D4F8EE334
:1046800097E040E150E00E94B3518FEB97E060E08B
:1046900040E00E9425138FEB97E06EE377E00E94E5
:1046A000D75B87E295E061E00E9403238FEB97E000
:1046B00060E041E00E94251384E1E816F10409F46A
:1046C00097C085E1E816F1041CF58CE0E816F104CA
:1046D00009F4A2C08DE0E816F10454F4E114F104E9
:1046E00009F440C081E0E816F10409F0F1C041C0CE
:1046F00081E1E816F10409F4CBC083E1E816F10486
:1047000009F46DC08EE0E816F10409F0E1C024C0A0
:104710008EE1E816F10409F4D5C08FE1E816F10442
:104720005CF48BE1E816F10409F4BAC08CE1E816F8
:10473000F10409F0CDC0B9C087E2E816F10409F42C
:1047400057C089E2E816F10409F46EC086E2E81663
:10475000F10409F0BDC043C08FEB97E068E071E061
:104760000E94D75BF701E154FE4F80810E945422E2
:10477000CBC08091C001C82FD0E0E097D7FD05C025
:1047800085E295E00E94B12207C083E295E00E9495
:10479000B122D095C195DF4FCE0164E070E00E9458
:1047A0001C758FEB97E04AE050E00E94C45B81E209
:1047B00095E00E94B122CE0164E070E00E941C7579
:1047C000BC0144E0660F771F4A95E1F7681B790B3F
:1047D00009F063C08EE195E00E94B1229CC08CE19B
:1047E00095E00E94B122F701E154FE4F608185C03F
:1047F000F701E154FE4F80818C3320F08AE195E08F
:104800000E94B122F701E154FE4F608170E06C53C9
:1048100070408FEB97E074C07091CC0160E08091A4
:10482000CB01680F711D2DC01091E90100E080914E
:10483000E801080F111DC80164E670E00E940875C8
:104840008FEB97E04AE050E00E94735B88E195E0CF
:104850000E94B122C8016AE070E00E940875CB0195
:104860006AE070E00E940875BC018FEB97E04AE0B7
:1048700050E00E94735BC8016AE070E00E94087516
:10488000BC018FEB97E04AE050E00E94735B43C0AD
:104890008091D0010E947052BC018FEB97E00DC057
:1048A0000E94A1216091DA0105C081E00E94872168
:1048B0006091DB018FEB97E070E04AE050E00E94EE
:1048C000C45B29C08FEB97E06DE20E94E45A23C0DD
:1048D000F701E352FB4FE491D701A154BE4FE13001
:1048E00059F48C91882319F481E195E002C084E1A8
:1048F00095E00E94B12208C06C918FEB97E070E0C8
:104900004AE050E00E94C45B87E1E816F10419F424
:104910008FE095E00EC0C7014397029740F086E212
:10492000E816F10421F087E2E816F10421F48AE0A8
:1049300095E00E94B122DF91CF911F910F91FF90DE
:10494000EF900895FF920F931F93482FF62E8FEB51
:1049500097E060E00E942513809111078695869567
:10496000877019F48DE395E012C08BE395E00E9407
:10497000B122609111076695669567708FEB97E09D
:1049800070E04AE050E00E94C45B89E395E00E9439
:10499000B1228091100780FD06C08DE295E061E0B4
:1049A0000E9403232EC0E0911107E695E695E7707B
:1049B000F0E0E55EF84F008110E090911107990F4B
:1049C00098739F5F910F8091D101981721F400FD9A
:1049D0000EC06DE40DC08091E401981721F400FD34
:1049E00006C06EE405C000FD02C06FE501C06F2D7A
:1049F0008FEB97E00E94E45A1F5F183011F0069584
:104A0000DCCF88E295E00E94B1228FEB97E06CE06A
:104A100041E00E9425138091EA01882329F08FEB61
:104A200097E065E00E94E1128FEB97E06DE041E0D6
:104A30000E9425138091100781FD06C082FF09C0E6
:104A40008091D401813029F48FEB97E063E00E94DC
:104A5000E1128091D401823029F48FEB97E066E077
:104A60000E94E1128FEB97E06EE041E00E94251377
:104A70008091100785FF05C08FEB97E062E00E94F0
:104A8000E1128FEB97E06FE041E00E94251360E0B8
:104A90008091110782958695877090E003970CF0BE
:104AA00061E08FEB97E00E94E1121F910F91FF9060
:104AB0000895DF92EF92FF920F931F93CF93DF93AE
:104AC0007C01D62E8FEB97E00E9457138FEB97E077
:104AD00060E040E00E9425138701C0E0D0E0DD20C7
:104AE00019F0F801638104C0F701EC0FFD1F60812C
:104AF0008FEB97E070E04AE050E00E94C45BC33067
:104B000021F08AE495E00E94B122219601501040E4
:104B1000C430D10521F7DF91CF911F910F91FF9004
:104B2000EF90DF9008952CE230E0F901E25CF84F5D
:104B3000D901A154BE4F8C918083215030408FEF1A
:104B40002F3F380791F780ED97E06EE377E04DE275
:104B500050E023EB30E20E9471088091CE018F5F1C
:104B60008093190790E063E0880F991F6A95E1F739
:104B700080931A079091D7019170809110078E7FD2
:104B8000892B8093100708950F931F93CF93DF9382
:104B9000EC010AEA82E00E94F321482F50E09A01DA
:104BA0002F7030702230310589F12430310509F43D
:104BB00052C02130310509F09BC0209709F49BC0F9
:104BC000CE30D10509F497C0C832D10509F493C09D
:104BD000CC30D10509F48FC0CD30D10509F48BC09C
:104BE000C932D10509F487C0CA32D10509F483C09E
:104BF000FE01E352FB4FE491DE01A154BE4F8C91C4
:104C0000E81709F478C08F5F8C9375C0209709F47A
:104C10006FC0CE30D10509F46BC0C832D10509F49C
:104C200067C0CC30D10509F463C0CD30D10509F49B
:104C30005FC0C932D10509F45BC0CA32D10509F49D
:104C400057C0FE01E154FE4F9081992309F450C0F2
:104C5000915090834DC086FF4BC087FF0AC0809162
:104C6000EB01882311F00093EB010E94932511E0E2
:104C700043C0C330D10539F48091C201882319F1B2
:104C8000CCE0D0E038C0CC30D10519F4CEE0D0E093
:104C900032C0C932D10519F4CBE2D0E02CC0C53105
:104CA000D10539F48091D4018130A1F0C7E1D0E081
:104CB00022C0C231D10539F48091D101882351F449
:104CC000C5E1D0E018C0C532D10521F48091E401DE
:104CD000882309F1CE0101966DE270E00E941C75F7
:104CE000EC018031910539F410E0C1E1D0E004C05D
:104CF000882309F44FCF10E0CE010E943023112306
:104D000009F448CF8FEB97E00E941313DF91CF9106
:104D10001F910F910895C8E2D0E0EDCF8091100768
:104D20008E7F809310071092D7010E9493250895DB
:104D30008091100781608093100781E08093D701F4
:104D40000E949325089584EE93E064E077E04CE0C0
:104D500050E023EB30E20E94710808958091100723
:104D60008D7F809310071092080710920907109208
:104D70000A0710920B070E94A3260895809110073E
:104D80008260809310070E94A326089546E050E0B9
:104D900023EB30E20E9471080895FB01108A90E035
:104DA00074E0880F991F7A95E1F784559B4FBF01F6
:104DB00040E150E023EB30E20E94710808958EE359
:104DC00097E060ED77E04DE250E02BEA30E20E94A0
:104DD000550820E030E0F901E154FE4FD901A25C12
:104DE000B84F8C9180832F5F3F4F2D32310599F75B
:104DF0008091CE018F5F8093190790E0E3E0880FE8
:104E0000991FEA95E1F780931A079091D701917065
:104E1000809110078E7F892B8093100782E080930A
:104E2000E701089584E097E064EE73E04CE050E021
:104E30002BEA30E20E9455088091100790911107EB
:104E4000A0911207B0911307809314079093150750
:104E5000A0931607B093170708959C01CB01B901E1
:104E600046E050E02BEA30E20E9455080895FB012D
:104E7000108A682F70E0A4E0660F771FAA95E1F70B
:104E800064557B4FCF0140E150E02BEA30E20E94B5
:104E900055080895EF92FF920F931F93CF93DF93DE
:104EA0006AEF70E080E090E00E94E756F999FECF4B
:104EB00080ED97E092BD81BDF89A80B5883D59F4A8
:104EC000F999FECF8CEF97E092BD81BDF89A80B53D
:104ED0008A3A09F0DAC084ED95E060E00E9403238D
:104EE00085EC95E061E00E940323EEE3F7E0119288
:104EF00087E0EE3BF807D9F7C0E0D0E000E018E02B
:104F0000A8014C1B5D0B4138510514F040E850E0FE
:104F1000CE016EE377E023EB30E20E947108C058C7
:104F2000DF4F88E0C030D80759F70E94A32680EFF2
:104F300093E06AE071E049E050E023EB30E20E9448
:104F4000710884E194E063E171E04AE050E023EB12
:104F500030E20E94710884E494E06DE171E040E287
:104F600050E023EB30E20E9471088CE694E06DE3A0
:104F700071E04AE150E023EB30E20E94710884E9DD
:104F800094E067E571E041E050E023EB30E20E94FD
:104F9000710883E580933E07109241070CEA14E004
:104FA000C1E0D0E0BEE3EB2EB7E0FB2ECE016AE01D
:104FB00070E00E941C75605D60933F07CE016AE05F
:104FC00070E00E941C75805D80934007F70101909E
:104FD0000020E9F7EE53F740C8016EE377E0AF0138
:104FE00023EB30E20E947108005F1F4F219687E09B
:104FF0000C3A1807D9F610923E0780E380933F07DA
:1050000010924007C0E0D0E081E291E06EE377E0EB
:1050100048E150E09E0100E00E942C53689684E035
:10502000C038D80789F78FEF80933E0780933F07FA
:105030008093400780934107809342078093430702
:105040008CEA97E06EE377E046E050E023EB30E255
:105050000E94710884EC97E06EE377E046E050E050
:1050600023EB30E20E94710886E191E00E948552B4
:105070000E94932564EF71E080E090E00E94E75683
:10508000E091D507F091D60709950E94DF260E948E
:10509000122780E00E94F321182F90E08F7090700B
:1050A0008130910519F0049781F503C08CE290E0FE
:1050B00021C085EB95E060E00E94032360ED77E07E
:1050C00080E090E00E94E75684EA95E060E00E946C
:1050D000032384E995E061E00E94032380E00E94BD
:1050E000F321182F86FFFACF8FEB97E00E9457131A
:1050F00080E090E00E94C4258091EB01882329F094
:10510000E091D507F091D607099581E00E948721AB
:105110000E94A121112309F040C085E895E060E0DC
:105120000E9403238FEB97E062E041E00E94251389
:1051300080E895E00E94B1221091CD01812F6AE0B4
:105140000E94FC74682F605D8FEB97E00E94E45A28
:105150008FEB97E06EE20E94E45A812F6AE00E9492
:10516000FC74692F605D8FEB97E00E94E45A809198
:1051700018078A3129F08C3D31F48CE795E005C0A1
:1051800088E795E002C084E795E00E94B12268EECE
:1051900073E080E090E00E94E756DF91CF911F918D
:1051A0000F91FF90EF900895AF92BF92DF92EF9230
:1051B000FF920F931F93DF93CF93CDB7DEB728975E
:1051C0000FB6F894DEBF0FBECDBF8C01D62E68E0BF
:1051D0000E94C620292F3327442755272093E60213
:1051E0009C01442755272093E702272F382F492F6A
:1051F00055272093E8026093E902A090B601B09091
:10520000B701C801089664E00E94C6207093B701F8
:105210006093B60186E5E82E87E0F82E1C821B829B
:1052200086E392E09A838983FE82ED82F886EF829C
:10523000C8010C9662E00E94C6202DB73EB72C50E4
:1052400030400FB6F8943EBF0FBE2DBFEDB7FEB78E
:1052500031969E012F5F3F4FADB7BEB712963C937C
:105260002E93119727EE35E03383228320EF33E02E
:105270003583248377836683D086118680E690E029
:10528000938782870E948B112DB73EB7245F3F4FD3
:105290000FB6F8943EBF0FBE2DBF83EE95E0B70169
:1052A00041EE55E02BE731E20E94E04700E010E0DC
:1052B0000E946A0F0E94F64A0F5F1F4F04361105C5
:1052C000B9F7B092B701A092B60128960FB6F8943C
:1052D000DEBF0FBECDBFCF91DF911F910F91FF9029
:1052E000EF90DF90BF90AF9008950F931F93DF93DF
:1052F000CF930F92CDB7DEB7FC01162F018100517D
:1053000080812AE0829FC0011124080F928190536E
:10531000802F61E099830E9485579981112319F0AC
:10532000802F692F03C061E0691B802F0E94C45742
:105330000F90CF91DF911F910F910895EF92FF92FF
:105340000F931F93DC01CB0179018A01139A0E940C
:1053500040571398C7010E9440571F910F91FF902B
:10536000EF9008952F923F924F925F926F927F92AB
:105370008F929F92AF92BF92CF92DF92EF92FF9265
:105380000F931F93DF93CF9300D00F92CDB7DEB76B
:105390004B015C0179018A01DA01C901880F991F6B
:1053A000AA1FBB1F820F931FA41FB51F582E692E63
:1053B0007A2ECB2EDA01C90155E0880F991FAA1F5A
:1053C000BB1F5A95D1F78E199F09A00BB10B89838A
:1053D000292E3A2E4B2EDD242FC0D501C4010A8080
:1053E00004C0B695A795979587950A94D2F780FF44
:1053F00007C0652D762D872D9C2DA801970106C02D
:10540000C801B701252D362D472D5C2D0E949E2900
:105410008A819B8101979B838A838F5F9F4FE9F6E7
:10542000C801B7012981322D432D542D0E949E2998
:10543000D394FFE0DF1629F087E190E09B838A8315
:10544000CCCF0F900F900F90CF91DF911F910F91C4
:10545000FF90EF90DF90CF90BF90AF909F908F9094
:105460007F906F905F904F903F902F9008951F9383
:10547000DF93CF93CDB7DEB728970FB6F894DEBF92
:105480000FBECDBF162FBE016F5F7F4FAE014B5FCA
:105490005F4F0E9412219C01112329F069817A81BA
:1054A0008B819C8104C06D817E818F81988540E0D5
:1054B00050E00E94B22928960FB6F894DEBF0FBEC6
:1054C000CDBFCF91DF911F9108951F93162F482FC5
:1054D00050E0F999FECFCA01F3E095958795FA95CA
:1054E000E1F78653984F92BD81BDF89A80B590E060
:1054F0009A012770307002C0959587952A95E2F73A
:1055000080FF31C09A01220F331F240F351F73E033
:10551000220F331F7A95E1F781E291E06EE377E0A5
:1055200048E150E00E94BA5280913E07813041F438
:1055300060E0111161E08FE397E00E94372A13C009
:10554000823041F460E0111161E08FE397E00E9446
:10555000D42809C0833039F460E0111161E08FE391
:1055600097E00E9475291F910895782F282F30E029
:10557000F901A3E0F595E795AA95E1F7E55EF84F07
:105580002770307081E090E002C0880F991F2A9543
:10559000E2F7282F3081482F50E0662371F0832FE7
:1055A00090E084239523892BB9F4322B3083872F05
:1055B00061E00E94652A81E00895832F90E08423B2
:1055C0009523892B49F0209523232083872F60E0A2
:1055D0000E94652A8FEF089580E008951F9310E0E0
:1055E000812F60E00E94B52A1F5F1133C9F71F9118
:1055F000089584E00E940F569C0183E02A3B3807FF
:1056000018F020E030E02BC083E02D33380718F08D
:1056100021E030E024C082E02E3D380718F022E07F
:1056200030E01DC082E02239380718F023E030E076
:1056300016C082E02535380718F024E030E00FC0AE
:1056400082E02232380718F025E030E008C0275FFA
:10565000314018F026E030E002C02FEF3FEFC901E3
:105660000895EF92FF920F931F93CF93DF9383E000
:1056700060E00E94C45700E217E08091100780FDAF
:1056800002C060E002C0F8016081C7E0D0E0E62E11
:10569000FF2486E160E00E94C457B7010C2E02C0CF
:1056A000759567950A94E2F7617085E10E94C45789
:1056B00086E161E00E94C4572197FFEFCF3FDF07EB
:1056C00041F70150104087E00A311807B1F683E036
:1056D00061E00E94C4570E94DD5020E330E040E0CA
:1056E00050E00E942F75962F8091D8076817B1F06F
:1056F0006093D807E62FE695E695E695F0E0E55E3F
:10570000F84F608170E0892F877002C075956795AA
:105710008A95E2F76170892F0E94652ADF91CF9107
:105720001F910F91FF90EF900895EF92FF920F93CA
:105730001F930E94DD507B018C016091C00170E0DD
:1057400080E090E024E833E040E050E00E94DD7427
:105750009B01AC01205C384A404050402E0D3F1D5B
:10576000401F511FB901CA011F910F91FF90EF9087
:1057700008950E94952B20E831E541E050E00E9419
:105780002F752D5F3F4F4F4F5F4FCA01B90127E083
:1057900030E040E050E00E942F75862F0895EF9290
:1057A000FF920F931F937B018C018FEB97E060E0DA
:1057B00040E00E942513C801B7010E94CA4F0E9411
:1057C0008E2280E795E00E94B122C801B7010E94B5
:1057D000C44F0E948E228DE695E00E94B1220E9465
:1057E000B92B90E0880F991F880F991F845B9A4FFF
:1057F0000E94B1228BE695E00E94B122C801B70158
:105800000E94B24F0E948E2289E695E00E94B1224A
:10581000C801B7010E94BE4F0E948E221F910F91B6
:10582000FF90EF9008958F92AF92CF92EF920F93E7
:1058300000D000D0EDB7FEB73196ADB7BEB7119628
:105840001C921182128213828FEB97E061E043E198
:105850002FEF02E1E4E1EE2E75E1C72E56E1A52E11
:1058600037E1832E0E94CA130F900F900F900F9074
:105870008FEB97E00E945F138091C307882341F468
:1058800082E08093810081E00E9487210E94A12113
:105890000F91EF90CF90AF908F9008958F929F923D
:1058A000AF92BF92CF92DF92EF92FF920F931F932E
:1058B000DF93CF93CDB7DEB728970FB6F894DEBF4E
:1058C0000FBECDBF81E061E00E94855781E061E0BD
:1058D0000E94C45783E061E00E94855783E061E045
:1058E0000E94C45786E161E00E94855785E161E02E
:1058F0000E9485570E94EE2A0E94312B81E060E0D1
:105900000E94C4578BE060E00E9485578BE061E005
:105910000E94C45781E062EC74E142E050E00E94D2
:1059200056558091100781608F7B8093100780917E
:10593000100790911107A0911207B091130780935F
:10594000140790931507A0931607B093170788E6DE
:1059500091E0909305078093040788E394E0909387
:10596000070780930607FF24F394F092190748E095
:10597000B42EB0921A078CE161E00E9485578CE149
:1059800060E00E94C4578CEA8093180782EA9BE08B
:105990000E94B45C0E94132C198284E18A83BB822A
:1059A00035E1E32EEC82FD8225E0C22ECE82CF824D
:1059B000E8868FEB97E061E08E010F5F1F4FA80133
:1059C0000E94EB121A821B82FC828FEB97E060E050
:1059D000A8010E94EB121A829FE1F92EFB8281E15D
:1059E000D82EDC82FD82DE82B3E18B2E8F82AEE187
:1059F0009A2E98868FEB97E062E0A8010E94EB1246
:105A000086E08B83F9E0AF2EAC82FD821E82EF82AE
:105A1000E8868FEB97E063E0A8010E94EB1287E035
:105A20008B8383E08C83CD82BE8280E18F83188656
:105A30008FEB97E064E0A8010E94EB121B82DC82EE
:105A40008BE08D83CE82AF8298868FEB97E065E006
:105A5000A8010E94EB121B829AE19C8382E18D8354
:105A60009E838F8218868FEB97E066E0A8010E94E4
:105A7000EB1280E061E00E94855780E061E00E94C7
:105A8000C4578EEA96E060E044E00E94476A8823AB
:105A900029F0809110078062809310078FE160E009
:105AA0000E9485578EE160E00E9485578DE160E09D
:105AB0000E9485578FE161E00E94C4578EE161E04A
:105AC0000E94C4578DE161E00E94C4570E94850D79
:105AD00028960FB6F894DEBF0FBECDBFCF91DF91F1
:105AE0001F910F91FF90EF90DF90CF90BF90AF90FC
:105AF0009F908F900895CF93DF9382EA9BE060E5BB
:105B000070E00E94DA5B82EA9BE060E00E945C5CED
:105B100082EA9BE00E949F5C882311F080E029C00C
:105B200082EA9BE060E570E00E94DA5B82EA9BE03B
:105B30006AEF0E945C5C82EA9BE00E949F5C82EAC2
:105B40009BE060E570E046E050E00E94B05C82EAD5
:105B50009BE00E94E45B892BD1F3CEE3D7E082EA9D
:105B60009BE00E94ED5B899387E0C434D807B9F7C6
:105B700081E0DF91CF910895DF93CF93CDB7DEB76A
:105B800028970FB6F894DEBF0FBECDBF80E096E039
:105B900061E00E9403230E947B2D882391F41092E0
:105BA0003E0789E680933F07809340078DE280930C
:105BB000410781E3809342078091D9018093430795
:105BC00005C08091100780688093100780EC93E0F7
:105BD0006EE377E044E00E944811882309F461C035
:105BE0009091CC0180E02091CB01820F911D909388
:105BF000B7018093B6018091C201882349F10E94C8
:105C0000A60B882309F44DC08091CE028093C30176
:105C10008091CF028093C4018091D0028093C5010E
:105C20008091D1028093C6018091DA028093C701EE
:105C30008091DB028093C8018091DC028093C901CE
:105C40008091DD028093CA010E94932591E02AC0D1
:105C50008091C30189838091C4018A838091C501A9
:105C60008B838091C6018C838091C7018D83809145
:105C7000C8018E838091C9018F838091CA01888772
:105C8000AE014B5F5F4FCE010196BA0120E030E0DC
:105C90000E94121190E0882309F491E081E0982796
:105CA00001C090E0892F28960FB6F894DEBF0FBE92
:105CB000CDBFCF91DF9108959C01F999FECF32BD00
:105CC00021BDF89A80B508959C01F999FECF1FBABD
:105CD00032BD21BD60BD0FB6F894FA9AF99A0FBE95
:105CE00008952091DA07203318F020E030E012C048
:105CF0002F5F2093DA0781E090E0821B910923E077
:105D0000880F991F2A95E1F722273327281B390B83
:105D10002552384FC9010895CF93DF93582F4091F2
:105D2000DA07841798F5E82FF0E0242F30E02150AF
:105D30003040E217F3073CF5EF01A3E0CC0FDD1F85
:105D4000AA95E1F7D90173E0AA0FBB1F7A95E1F795
:105D5000C552D84FA552B84F88E00D900992815096
:105D6000E1F763E0EE0FFF1F6A95E1F7E552F84FA8
:105D70008681E82FF0E0E55AF64F808190E08217A7
:105D8000930709F4508341504093DA07DF91CF9194
:105D900008951092D907F999FECF1FBA81E090E0DB
:105DA00092BD81BD10BC0FB6F894FA9AF99A0FBE55
:105DB0000895982F8091D907981708F041C099232A
:105DC00009F43EC0892F90E0019727E430E0AC0150
:105DD000429FC001439F900D529F900D11249C0142
:105DE0002E5F3F4F875B9F4F24C0F999FECF32BD96
:105DF00021BDF89A50B5F999FECF72BD61BDF89AF0
:105E000040B5F999FECF1FBA32BD21BD40BD0FB6D6
:105E1000F894FA9AF99A0FBEF999FECF1FBA72BD9B
:105E200061BD50BD0FB6F894FA9AF99A0FBE2F5F74
:105E30003F4FB901695B7F4F2817390709F0D5CF6C
:105E4000089577FF03C06FEF7FEF22C0CB019770FB
:105E500074FF03C0909581959F4F76FF0BC06091B2
:105E6000040770910507680F791F77FF11C060E084
:105E700070E00EC075FF0CC06091060770910707B7
:105E8000680F791F85E0603A780714F06FE975E0D4
:105E9000CB010895BF92CF92DF92EF92FF920F93C2
:105EA0001F936C01FC01B080E1800E94952B20E8DB
:105EB00031E541E050E00E942F752B0D311D411D51
:105EC000511DFF2400E010E0CA01B901A8019701AB
:105ED0000E942F75F60160831F910F91FF90EF9044
:105EE000DF90CF90BF9008958F929F92AF92BF9214
:105EF000CF92DF92EF92FF920F931F934C01FC0120
:105F0000A180E080FF24EA0CF11C0027F7FC00953B
:105F1000102F0E94952BBB24CC24DD2420E831E5F2
:105F200041E050E00E942F75CA01B901A601950118
:105F30000E942F75E61AF70A080B190BC801B70162
:105F4000A60195010E942F75F40160831F910F91A6
:105F5000FF90EF90DF90CF90BF90AF909F908F9089
:105F60000895BF92CF92DF92EF92FF920F931F930B
:105F7000CF93DF93EC017A018B01CB01BA010E9430
:105F8000B84FC82EC801B7010E94BE4FD82EC80115
:105F9000B7010E94B24FB82E88818295837090E03D
:105FA00082309105B1F083309105E9F0892BA1F59C
:105FB000298130E08C2D90E0059667E070E00E942A
:105FC0001C7502C0359527958A95E2F720FD24C0FF
:105FD0003BC02D2D30E0898190E08F7190702817A3
:105FE000390791F519C0C801B70120E831E541E052
:105FF00050E00E942F75CA01B9012A8130E040E0CB
:1060000050E00E942F75298130E040E050E0621797
:10601000730784079507C1F48881869586958370F8
:10602000A9F0823019F48D2D80950CC0813071F467
:106030008FE1D81649F08DE1D81619F482E0B81630
:1060400019F08D2D817003C080E001C081E0DF91E7
:10605000CF911F910F91FF90EF90DF90CF90BF9065
:1060600008956F927F928F929F92AF92BF92CF923C
:10607000DF92EF92FF920F931F93CF93DF938C01E8
:106080006A017B01DC018C9180FF85C013966D91C4
:106090007C911497C8010E94212F4C01F801658062
:1060A0007680C781D085C701B60120E831E541E09F
:1060B00050E00E942F752CE330E040E050E00E9459
:1060C0002F755901C801B701A6010E94B12F88237D
:1060D000A9F1D8018C9186FF14C0E801B8E0EB2E3D
:1060E000F12CE00EF11E6B817C81C8010E94212FF2
:1060F000A816B90609F451C02296CE15DF0599F706
:106100004AC0A814B90409F448C08A149B04B0F426
:106110002097A1F0950128193909C901BE010E94F3
:1061200008756C9FC0016D9F900D7C9F900D112490
:106130008217930719F4661677067CF5F8018081BB
:1061400086FD29C0209739F180E89EEAAEEFBFEFC7
:10615000C80ED91EEA1EFB1EC801B701A6010E9487
:10616000B12F8823C1F095012819390920563A4FDB
:10617000C901BE010E9408756C9FC0016D9F900D02
:106180007C9F900D11248217930729F480E06616F6
:10619000770624F002C080E001C081E0DF91CF915A
:1061A0001F910F91FF90EF90DF90CF90BF90AF9035
:1061B0009F908F907F906F900895982F9B01809172
:1061C000D907981768F467E4969FB00111246E5FB1
:1061D0007F4FC90147E450E02CE53EE20E9455089C
:1061E0000895DF92EF92FF920F931F93DF93CF9367
:1061F000CDB7DEB7C754D0400FB6F894DEBF0FBEA0
:10620000CDBF2091D907821708F046C0222309F498
:1062100043C090E0019627E430E0829F8001839F95
:10622000100D929F100D11240E5F1F4F87E4D82E82
:106230007E010894E11CF11C14C0C701B80147E4B9
:1062400050E02CE53EE20E945508C801875490407A
:10625000B70147E450E024E63EE20E947108095B82
:106260001F4F2091D9072D9DC001112402960817B8
:10627000190718F321502093D907F999FECF1FBAB7
:1062800081E090E092BD81BD20BD0FB6F894FA9AEE
:10629000F99A0FBE81E001C080E0C95BDF4F0FB605
:1062A000F894DEBF0FBECDBFCF91DF911F910F914C
:1062B000FF90EF90DF900895982F8091D90798175D
:1062C00010F080E0089587E4989FC00111240296A1
:1062D00047E450E024E63EE20E94710881E0089520
:1062E000BC019091D9079E3010F080E0089587E4BA
:1062F000989FC0011124029647E450E024E63EE254
:106300000E9471082091D9072F5F2093D907F9992E
:10631000FECF1FBA81E090E092BD81BD20BD0FB6D7
:10632000F894FA9AF99A0FBE81E008958BE599E006
:106330006FEF70E040E350E00E9414081092DA071B
:10634000109293091092940910929509109296094F
:1063500008950E949631F999FECF81E090E092BDB8
:1063600081BDF89A80B58093D90708959C01F99969
:10637000FECF1FBA32BD21BD60BD0FB6F894FA9AA8
:10638000F99A0FBE0895EF92FF920F93CF93DF9388
:10639000DC01EB01722F532F002331F4822F932F56
:1063A0009C01F90160E03EC0822F932FFC0160E068
:1063B00019C08491332727FD309590E028173907BD
:1063C00069F431968491882361F411968C918D3310
:1063D00029F4872F952FFC0161E003C0872F952FAB
:1063E000FC0111962C91222339F1203229F12A3017
:1063F00019F16623F1F224C08081981771F4319667
:106400008081882371F411968C918D3331F4872F1C
:10641000952F9C01F90161E004C0872F952F9C0105
:10642000F90111969C91992339F0903229F09A3014
:1064300019F0662309F304C0613011F030E018C090
:106440007A2F50E04150504002C0299311963A2FC4
:10645000371B2C91222359F0203249F02A3039F091
:10646000263229F0832F90E08417950774F3188261
:10647000E114F10411F0F7016083832FDF91CF91D4
:106480000F91FF90EF900895CF93DF93FC01EC0103
:1064900037C08B3211F480E231C0853279F5DF01EB
:1064A00011969181392F30533A3070F0892F8156EF
:1064B000863010F4375208C0892F8154863010F08E
:1064C00030E002C0392F3753FD01319611962C91DF
:1064D000922F90539A3070F0822F8156863010F4AC
:1064E000975208C0822F8154863010F090E002C08D
:1064F000922F9753832F8295807F892B8993319692
:106500008081882331F61882DF91CF9108956F92B0
:106510007F928F929F92BF92CF92DF92EF92FF92E3
:106520000F931F93DF93CF93CDB7DEB728970FB6A6
:10653000F894DEBF0FBECDBF8091DF0189838091CB
:10654000E0018A838091E1018B838091E2018C8359
:10655000BB243E010894611C711C85E0882E912C9F
:106560008C0E9D1E609114026F5F60931402C30134
:106570000E94584A0E94D9566B017C0188EE93E034
:10658000A0E0B0E0C80ED91EEA1EFB1E0E946A0FF2
:106590008C010E94F64A012B71F1C4016091140232
:1065A0000E949447882339F12D813E814F8158857F
:1065B00020583E474A4A534808C0B39494E1B9165C
:1065C00089F620E030E040E050E0B901CA012896A9
:1065D0000FB6F894DEBF0FBECDBFCF91DF911F91F4
:1065E0000F91FF90EF90DF90CF90BF909F908F9092
:1065F0007F906F9008950E94D9566C157D058E0589
:106600009F0520F2DACF1F93CF93DF93182F8DB71A
:106610009EB70C970FB6F8949EBF0FBE8DBFEDB717
:10662000FEB73196C7EED6E0ADB7BEB71296DC9393
:10663000CE93119782E09DE09383828389E59CE06D
:10664000958384838BE69CE0978386838FE99CE027
:106650009187808780EC9CE0938782870E948B11D2
:10666000EDB7FEB73C960FB6F894FEBF0FBEEDBF78
:106670001123A1F000D000D0ADB7BEB71296DC93C5
:10668000CE93119780E09DE014969C938E93139780
:106690000E948B110F900F900F900F90DF91CF9170
:1066A0001F9108958DB79EB70C970FB6F8949EBFB3
:1066B0000FBE8DBFEDB7FEB7319687EE96E0ADB752
:1066C000BEB712969C938E93119787E29DE09383B9
:1066D000828389E59CE0958384838DE09DE09783A8
:1066E000868380EC9CE0918780878FE99CE093878C
:1066F00082870E948B118DB79EB70C960FB6F894C7
:106700009EBF0FBE8DBF08950F931F930E945233FB
:1067100000D000D000D0EDB7FEB7319607EE16E0FE
:10672000ADB7BEB712961C930E93119788E098E010
:10673000938382838CE497E0958384830E948B11FA
:1067400000D0EDB7FEB73196ADB7BEB712961C9329
:106750000E9311978AEE97E09383828388ED90E001
:10676000958384838091D801868317820E948B1140
:106770000F900F90EDB7FEB73196ADB7BEB712963A
:106780001C930E93119787EB97E09383828384E4A5
:1067900094E0958384830E948B118DB79EB70696F3
:1067A0000FB6F8949EBF0FBE8DBF80E01F910F9172
:1067B00008950E9452338DB79EB70C970FB6F89488
:1067C0009EBF0FBE8DBFEDB7FEB7319687EE96E048
:1067D000ADB7BEB712969C938E93119785E299E060
:1067E0009383828384E494E09583848388E591E0B5
:1067F000978386838CE694E09187808788E791E091
:10680000938782870E948B118DB79EB70C960FB627
:10681000F8949EBF0FBE8DBF80E00895AF92BF92E7
:10682000DF92EF92FF920F931F93CF93DF9300D0ED
:1068300000D007EE16E0ADB7BEB712961C930E93CC
:10684000119782E197E014969C938E9313970E9480
:106850008B11FF240F900F900F900F90D02EE12EF0
:106860002FE0A22E27E0B22ECDE0D7E04FC00F2DB3
:1068700010E000D000D000D0ADB7BEB71196EDB794
:10688000FEB7D182E2821396BC92AE921297F801C3
:1068900093E0F595E7959A95E1F7E55EF84F8081ED
:1068A00090E098012770307002C0959587952A95E1
:1068B000E2F78170907015969C938E9314970E94C6
:1068C0008B1180911A0790E001972DB73EB72A5F90
:1068D0003F4F0FB6F8943EBF0FBE2DBF08171907E4
:1068E000A1F000D000D0ADB7BEB71196DC921197E1
:1068F0001296EC9212971496DC93CE9313970E9403
:106900008B110F900F900F900F90F39420911A0716
:10691000F21608F4ACCF00D000D000D0EDB7FEB72F
:10692000319687EE96E0ADB7BEB712969C938E93E4
:1069300011978BEF96E093838283248315820E94C4
:106940008B11EDB7FEB736960FB6F894FEBF0FBEAB
:10695000EDBF61E070E080E090E00E94E756DF91DB
:10696000CF911F910F91FF90EF90DF90BF90AF906C
:10697000089581E00E9403330E940E3480E0089560
:10698000EF92FF920F936EE377E040E821ED36E05F
:1069900001E0EE24FF240E94C331882311F480E13A
:1069A00005C08EE397E00E94A21581E00F91FF9051
:1069B000EF900895CF93DF939C0110923E07FC0166
:1069C000A081B181C0E0D0E00FC09C919D3231F038
:1069D0009B3221F0892F80538A3068F4FE01E25CFB
:1069E000F84F908321961196F901808191810A9642
:1069F000A817B90750F3C25CD84F18821196F90155
:106A0000B183A0838EE397E00E94B907CB01DF91A9
:106A1000CF9108958F929F92AF92BF92CF92DF92C3
:106A2000EF92FF920F931F93CF93DF93EC016EE3EE
:106A300077E040E827EF36E001E0EE24FF240E94F3
:106A4000C331882309F475C08EE397E00E949B0749
:106A50006C0197FD6CC080911A0790E0C816D906AA
:106A60000CF065C0CE016EE377E040E824EF36E03D
:106A70000E94C331882309F45CC08EE397E00E9432
:106A80009B07182F0E94952B4B015C01112309F4E1
:106A900047C0CE016EE377E040E822EF36E00E9487
:106AA000C331882309F445C08EE397E00E94B907FB
:106AB000EB01CB01019780529D4FC8F596012F5FE6
:106AC0003F4F8091120790E082179307A1F18091C8
:106AD000130790E08217930771F1F601E55AF64F1C
:106AE00080818F3F51F0E82FF0E033E0EE0FFF1F81
:106AF0003A95E1F7E552F84F03C00E94712EFC0170
:106B00003097C9F01082118212821382D583C48318
:106B1000C68283E68783C501B4010E945B1705C066
:106B20008C2DB501A4010E94CF1881E005C081E140
:106B300003C080E101C080E3DF91CF911F910F91ED
:106B4000FF90EF90DF90CF90BF90AF909F908F908D
:106B50000895AF92BF92CF92DF92EF92FF920F9380
:106B6000DF93CF93CDB7DEB7C058D0400FB6F894BF
:106B7000DEBF0FBECDBF6C014EE3A42E47E0B42EA6
:106B8000B50140E82DE137E001E0EE24FF240E944A
:106B9000C331882311F480E12EC0C6016E01089430
:106BA000C11CD11CB60140E829E137E001E0EE2428
:106BB000FF240E94C3318823E9F0C501B60144E2F5
:106BC00050E00E9438080097A9F4C5010E944432A1
:106BD00010926107F50101900020E9F7EE53F740AC
:106BE00080EF93E0B501AF0126EB31E30E9471081D
:106BF00081E001C083E0C058DF4F0FB6F894DEBFDC
:106C00000FBECDBFCF91DF910F91FF90EF90DF903E
:106C1000CF90BF90AF900895EF92FF920F93CF93D4
:106C2000DF93EC016EE377E040E827E337E001E033
:106C3000EE24FF240E94C331882311F18EE397E0F4
:106C40000E94443210926607AEE3B7E0FD018081F6
:106C5000803209F08D938081882311F03196F7CF2F
:106C6000AEE3B7E0FD0101900020E9F7EA1BFB0B62
:106C700084E494E0BD01AF0126EB31E30E9471088A
:106C8000CE016EE377E040E823E337E001E0EE2455
:106C9000FF240E94C331882311F18EE397E00E9404
:106CA000443210926607AEE3B7E0FD018081803286
:106CB00009F08D938081882311F03196F7CFAEE3F0
:106CC000B7E0FD0101900020E9F7EA1BFB0B8CE621
:106CD00094E0BD01AF0126EB31E30E9471088FEF14
:106CE000DF91CF910F91FF90EF9008952F923F92F7
:106CF0004F925F926F927F928F929F92AF92BF92CC
:106D0000CF92DF92EF92FF920F931F93DF93CF9377
:106D1000CDB7DEB727970FB6F894DEBF0FBECDBF55
:106D20003C01FFEBAF2EF1E0BF2E552488241F82DB
:106D3000CC24DD24E2E02E2E312C2C0E3D1E1C2D09
:106D40001C3209F47BC0183109F478C0CC2009F456
:106D500075C01E3009F472C0183209F46FC01031CA
:106D600009F46CC01B3209F469C0C601F50140800A
:106D7000F601E352FB4F9490F1E09F1611F4F501F8
:106D80001082D101EDE3F2E025E001900D92215057
:106D9000E1F7BE016D5F7F4F4AE050E00E948D0831
:106DA000C3016EE377E040E8910100E0EE24FF24A8
:106DB0000E94C331882371F1F1E09F1619F4F501A7
:106DC000908228C08EE397E00E94B9079B01AC0136
:106DD000143111F0173221F4245C3F4F4F4F5F4FB5
:106DE000113141F4C9010E945B52282F30E040E08C
:106DF00050E002C057FD0CC0892D90E0A0E0B0E04B
:106E000082179307A407B5071CF0F501208302C081
:106E1000F1E0FF83F5018081841581F0812F81509D
:106E2000823010F455245394812F8052843010F412
:106E3000552453941F3111F4882483940894C11C61
:106E4000D11C0894A11CB11CFDE2CF16D10409F09D
:106E500076CF7EE3C72E77E0D72EC301B60140E898
:106E60002FE237E001E0EE24FF240E94C3318823A3
:106E7000E1F0C6010E94443210926D07C60164E140
:106E800074E00E94C351882381F0F6010190002034
:106E9000E9F7EC19FD0984E194E0B601AF0126EBB6
:106EA00031E30E9471088824839419826EE3C62E10
:106EB00067E0D62EC301B60140E829E237E001E0E1
:106EC0007E010894E11CF11C0E94C3318823E9F083
:106ED000C6010E94443210925507C60164E974E06D
:106EE0000E94C351882321F1F60101900020E9F7A7
:106EF000EC19FD0984E994E0B601AF0126EB31E31A
:106F00000E9471088824839413C08981882381F0AA
:106F100010923E07F60101900020E9F7EE53F7408A
:106F200084E994E0B601AF0126EB31E30E947108D9
:106F30008091C101882319F5C3016EE377E040E831
:106F400025E237E001E0EE24FF240E94C3318823CC
:106F5000B1F08EE397E00E94B907162F072FF82EA5
:106F6000E92E0E945417612F702F8F2D9E2D0E94A5
:106F7000B050612F702F8F2D9E2D0E94380E5EE332
:106F8000C52E57E0D52EC301B60140E821E237E017
:106F900001E0EE24FF240E94C3318823B1F0C60132
:106FA0000E9444321092BE07F60101900020E9F7DA
:106FB0003197EC19FD0986E191E0B601AF0120E0BF
:106FC00030E00E942C53882483942F81222311F0D7
:106FD00081E114C00E949325552029F0809111076A
:106FE000816080931107882041F01092360710923B
:106FF0003707109238071092390781E027960FB6AD
:10700000F894DEBF0FBECDBFCF91DF911F910F91DE
:10701000FF90EF90DF90CF90BF90AF909F908F90B8
:107020007F906F905F904F903F902F9008952F9298
:107030003F924F925F926F927F928F929F92AF9208
:10704000BF92DF92EF92FF920F931F93CF93DF9344
:107050008AE2A82E81E0B82EC0E0D0E00EE3202E18
:1070600007E0302E17EE812E16E0912EB5EB4B2E59
:10707000BBE05B2EA3EB6A2EABE07A2EFE01E1545F
:10708000FE4F8081E82EFF2400E010E0DC2E24E19A
:10709000C21719F037E2C31741F484EC9FEFAFEF4A
:1070A000BFEFE80EF91E0A1F1B1F91E1D91649F424
:1070B0008E2D0E9470527C010027F7FC0095102F46
:1070C0000FC0AEE1DA1609F44BC0B0E1DB1609F4EB
:1070D00047C0EAE1DE1621F48091100787FD40C029
:1070E0008EE397E0B50145E050E00E94B3512DB723
:1070F0003EB72A5030400FB6F8943EBF0FBE2DBFAA
:10710000EDB7FEB73196ADB7BEB712969C928E9290
:1071100011975382428235822482E682F782008769
:1071200011870E948B11EDB7FEB73A960FB6F8940F
:10713000FEBF0FBEEDBFFCE2DF1691F000D000D025
:10714000ADB7BEB712969C928E92119714967C9210
:107150006E9213970E948B110F900F900F900F90CB
:107160002196E5E0F0E0AE0EBF1ECD32D10509F06C
:1071700085CF0E94F92A2DB73EB72A5030400FB66E
:10718000F8943EBF0FBE2DBFEDB7FEB7319627EE88
:1071900036E0ADB7BEB712963C932E93119724E913
:1071A0003BE0338322839583848385E090E097835B
:1071B000868380911807808711860E948B11EDB716
:1071C000FEB73A960FB6F894FEBF0FBEEDBF61E072
:1071D00070E080E090E00E94E756DF91CF911F9130
:1071E0000F91FF90EF90DF90BF90AF909F908F90A6
:1071F0007F906F905F904F903F902F90089581E027
:107200000E9403330E94173880E00895AF92BF9226
:10721000CF92DF92EF92FF920F931F93DF93CF9362
:10722000CDB7DEB7CB54D0400FB6F894DEBF0FBE5B
:10723000CDBF6C016EE377E040E822EC3BE001E07B
:10724000EE24FF240E94C331882309F4E5C08EE3B5
:1072500097E00E949B075C018FEFA8168FEFB8069E
:107260000CF4DCC08091D90790E0A816B9060CF0A8
:10727000D5C0C6016EE377E040E82DEB3BE00E940D
:10728000C3318E01025C1F4F882361F08EE397E0CB
:107290000E944432C8016EE377E04CE050E00E9467
:1072A000460817C0C8016EE076E00E94F7079FEF1E
:1072B000A9169FEFB90621F48091D90790E001C08B
:1072C000C5010196BE016A5B7F4F4AE050E00E9413
:1072D0008D08C6010E944432DA82C98286010C59A7
:1072E0001F4F0EC0C70162E971E043E050E00E9409
:1072F0003808009781F00894E11CF11CFA82E982B9
:10730000E980FA80F7018081882309F485C0E016BE
:10731000F10640F381C083E090E0E80EF91EFA82A6
:10732000E9827E010894E11CF11CC7010E94DA3455
:107330008B83C7010E94DA348C83C7010E94DA3440
:107340008D8389819A8101969A838983C7010E94DE
:10735000DA349F838E83C7010E94DA349987888745
:10736000C7010E94DA349B878A87C7010E94DA34FA
:107370009D878C8789819A8102969A83898310E000
:107380002C96FFAEEEAE2C972B96DFAC2B972C965F
:107390000FAD2C979EE0E92EF12CEC0EFD1E0BC0DC
:1073A0008D2D902F0E94DA340E94DB51F701E10FFE
:1073B000F11D80831F5F80911A07181788F3898158
:1073C0009A8102969A838983CE010E9605C0FC01AC
:1073D000E10FF11D10821F5F1033C8F38B8182957E
:1073E0008370833039F48D81823020F0CE01049691
:1073F0000E944A2FBE016D5F7F4F9FEFA9169FEF3E
:10740000B90621F4CB010E94703103C08A2D0E947D
:107410005C31882329F402C080E103C081E101C00E
:1074200081E0C55BDF4F0FB6F894DEBF0FBECDBF66
:10743000CF91DF911F910F91FF90EF90DF90CF9050
:10744000BF90AF900895EF92FF920F936EE377E0B5
:1074500040E826EC3BE001E0EE24FF240E94C3312B
:10746000882311F480E114C08EE397E00E949B070B
:107470009C01181619065CF48091D90790E0281732
:1074800039072CF4822F0E94D92E81E001C081E1BE
:107490000F91FF90EF900895EF92FF920F936EE39C
:1074A00077E040E82AEC3BE001E0EE24FF240E9474
:1074B000C331882311F480E118C08EE397E00E9465
:1074C0009B079C018FEF2F3F380719F40E94C92EAC
:1074D0000BC08091D90790E02817390714F081E19B
:1074E00004C0822F0E94F13081E00F91FF90EF9055
:1074F00008958F929F92AF92BF92CF92DF92EF92B8
:10750000FF920F931F93CF93DF938091100785FD18
:1075100002C080E29BC081E00E940333AFE38A2E69
:10752000A7E09A2E10E000E0F7EEEF2EF6E0FF2E37
:10753000EAEDAE2EEBE0BE2E73EFC72E7BE0D72E2A
:1075400063C0C12FD0E0CE0163E0959587956A9521
:10755000E1F78653984F0E94512190E09E012770D9
:10756000307002C0959587952A95E2F780FF4BC051
:107570009E01220F331F2C0F3D1F43E0220F331FAC
:107580004A95E1F781E291E06EE377E048E150E06F
:107590000E94BA52002311F401E012C000D000D0C2
:1075A000ADB7BEB71296FC92EE9211971496DC928C
:1075B000CE9213970E948B110F900F900F900F9007
:1075C000EDB7FEB73A970FB6F894FEBF0FBEEDBF0A
:1075D0003196ADB7BEB71296FC92EE921197B38278
:1075E000A282D583C48380913E07868317829186C9
:1075F00080860E948B11EDB7FEB73A960FB6F894CD
:10760000FEBF0FBEEDBF1F5F80911A07181708F469
:1076100098CF00D000D087EE96E0ADB7BEB71296F7
:107620009C938E93119788ED9BE014969C938E9378
:1076300013970E948B110F900F900F900F9061E0A5
:1076400070E080E090E00E94E75680E0DF91CF910B
:107650001F910F91FF90EF90DF90CF90BF90AF9070
:107660009F908F9008959F92AF92BF92CF92DF929A
:10767000EF92FF920F931F93DF93CF9300D0CDB77C
:10768000DEB78C010E9444321A83098384E6C82E37
:10769000D12CC00ED11E0DC0C80166E971E043E0D7
:1076A00050E00E943808009779F00F5F1F4F1A834F
:1076B000098309811A81F8018081882309F44DC06A
:1076C0000C151D0548F349C00D5F1F4F1A83098330
:1076D0000E945417FF24EE245E010894A11CB11CE3
:1076E000BEEF9B2E2EC0C5010E94DA346C010097BC
:1076F00039F18F2D86958695869590E08254984F26
:107700000E94512190E02F2D277002C095958795FA
:107710002A95E2F780FD14C00E94712E8C0100971B
:1077200079F0FC011082118212821382C6010E943C
:107730002D52F801758364839782F682EE24E394D8
:10774000F39480911A07F81670F2EE2031F00E943F
:10775000952B0E945B1781E001C080E10F900F9094
:10776000CF91DF911F910F91FF90EF90DF90CF901D
:10777000BF90AF909F900895AF92BF92DF92EF922B
:10778000FF920F931F93CF93DF937C01CB016EE3A6
:1077900077E00E942D2700D000D000D0EDB7FEB7D3
:1077A000319607EE16E0ADB7BEB712961C930E9356
:1077B00011978FE49CE093838283F582E4820E9498
:1077C0008B11EE24EDB7FEB736960FB6F894FEBFD8
:1077D0000FBEEDBFD02EF12E9CE4A92E9CE0B92E59
:1077E000CAE4DCE040C000D000D000D0ADB7BEB7E6
:1077F0001196EDB7FEB7D182F2821396BC92AE928B
:1078000012970E2D10E0F801E25CF84F808114967B
:107810008C93149715961C920E948B1180911907D6
:1078200090E001972DB73EB72A5F3F4F0FB6F8940F
:107830003EBF0FBE2DBF08171907A1F000D000D022
:10784000ADB7BEB71196DC9211971296FC921297C3
:107850001496DC93CE9313970E948B110F900F9088
:107860000F900F90E39480911907E81608F4BBCFAE
:1078700000D000D087EE96E0EDB7FEB7928381830B
:1078800087E49CE0948383830E948B110F900F9078
:107890000F900F90DF91CF911F910F91FF90EF907C
:1078A000DF90BF90AF9008952F923F924F925F92DA
:1078B0006F927F928F929F92AF92BF92CF92DF9200
:1078C000EF92FF920F931F93DF93CF93CDB7DEB765
:1078D00029970FB6F894DEBF0FBECDBF4C01162F0F
:1078E0005A01CA01BE016C5F7F4F0E942D27DE0145
:1078F0001196E2E4F2E083E001900D928150E1F70D
:10790000198310E032E0232E312C2C0E3D1E2E0167
:107910000894411C511C24E0622E712C6C0E7D1EBB
:107920001DC0C12EDD24C601B1014AE050E00E9415
:107930008D08C4016EE377E040E8920100E0EE2498
:10794000FF240E94C331882341F08EE397E00E9418
:107950009B07C60CD71CF60180831F5F8091190717
:107960001817F8F2C501BE016C5F7F4F0E94C62652
:1079700029960FB6F894DEBF0FBECDBFCF91DF9131
:107980001F910F91FF90EF90DF90CF90BF90AF903D
:107990009F908F907F906F905F904F903F902F902F
:1079A00008958F929F92AF92BF92CF92DF92EF9203
:1079B000FF920F931F93DF93CF9300D000D0CDB7EA
:1079C000DEB76C0183E789831A821B821C8210E078
:1079D00052E0852E912C8C0E9D1E5E010894A11CF8
:1079E000B11C1DC0812F90E0B4014AE050E00E941C
:1079F0008D08C6016EE377E040E8950100E0EE24D3
:107A0000FF240E94C331882349F08EE397E00E944F
:107A10004432812F6EE377E00E94CD261F5F809174
:107A20001A071817F8F2C6016DE64CEA57E00E94F3
:107A3000543CC60169E642EB57E00E94543CC60143
:107A40006EE648EB57E00E94543CC60164E64EEBFC
:107A500057E00E94543CC60161E744EC57E00E94A5
:107A6000543C8091100785FF06C0C60160E74AECD0
:107A700057E00E94543C4EE3A42E47E0B42EC601CA
:107A8000B50140E824ED3BE001E0EE24FF240E9434
:107A9000C3318823E9F1C5010E949B07182F80910B
:107AA0001A07811710F481E136C0C601B50140E81C
:107AB00021ED3BE001E0EE24FF240E94C331882346
:107AC00049F1C601B5016F5F7F4F40E82EEC3BE006
:107AD0000E94C3318823F1F080913E078053809348
:107AE0003E0710925507833011F480E314C0F5016E
:107AF00001900020E9F7EE53F74028E1129F900132
:107B0000112481E291E0B501AF0100E00E942C5305
:107B100081E001C080E10F900F900F900F90CF9106
:107B2000DF911F910F91FF90EF90DF90CF90BF906A
:107B3000AF909F908F900895EF92FF920F939C01CA
:107B40008091D8018823B1F4C9016EE377E040E861
:107B500026E53CE001E0EE24FF240E94C3318823A7
:107B600051F08EE397E00E9444328EE397E00E944A
:107B70005921811181E00F91FF90EF9008958823A2
:107B800071F08091ED069091EE062091EB06309118
:107B9000EC06821B930B61E10E94D348089580910B
:107BA000ED069091EE062091EB063091EC06821BDB
:107BB000930B60E10E94D3481092EA061092E90606
:107BC00084E293E09093EC068093EB069093EE06AC
:107BD0008093ED060895DF92EF92FF920F931F932B
:107BE000CF93DF938C010E9456491092EA061092BF
:107BF000E90684E293E09093EC068093EB06909381
:107C0000EE068093ED0675E0E72EF12CE00EF11EF6
:107C1000D80115965C91503219F40E948433CAC081
:107C2000E7E1F6E0C0E0D0E0652F772767FD7095CB
:107C3000D8011696DC2E849190E08617970709F0FC
:107C4000C4C031962491319730E04C91842F99270C
:107C500087FD90952817390709F0B7C087010D5F98
:107C60001F4F533719F4453791F536C05A3679F519
:107C70004F3611F0413659F5C8010E949C3D8823CA
:107C800059F581E00E940333EDB7FEB738970FB680
:107C9000F894FEBF0FBEEDBF319687EE96E0ADB70C
:107CA000BEB712969C938E93119784E896E09383C7
:107CB00082838AE291E0958384838091BF018683E9
:107CC00017820E948B11EDB7FEB7389648C0C801E5
:107CD0000E949C3D882331F1CC0FDD1FC451DE4F43
:107CE000E881F981C8010995182F8823E9F18F3FB0
:107CF000D1F40E94523300D000D000D0EDB7FEB7CF
:107D0000319687EE96E0ADB7BEB712969C938E93F0
:107D1000119781E896E09383828380E496E09583CF
:107D2000848318C012E081E00E94033300D000D0A9
:107D300000D0EDB7FEB7319687EE96E0ADB7BEB78F
:107D400012969C938E93119784E796E09383828397
:107D5000148315820E948B11EDB7FEB736960FB6CD
:107D6000F894FEBF0FBEEDBFF4E1DF1619F581E018
:107D70000E94033300D000D000D0EDB7FEB731969B
:107D800087EE96E0ADB7BEB712969C938E9311978F
:107D900087E696E09383828380E290E095838483F4
:107DA0000E948B11EDB7FEB736960FB6F894FEBF62
:107DB0000FBEEDBF81E00E94BF3DDF91CF911F91CB
:107DC0000F91FF90EF90DF900895D3942196329613
:107DD000C431D10509F02ECFC7CF2F923F924F92D9
:107DE0005F926F927F928F929F92AF92BF92CF924B
:107DF000DF92EF92FF920F931F93DF93CF93CDB754
:107E0000DEB7A3970FB6F894DEBF0FBECDBF4C010F
:107E10008091100785FD02C080E274C1C4016EE349
:107E200077E040E82DEE36E001E0EE24FF240E94EA
:107E3000C3318823B9F08EE397E00E949B077C0151
:107E400021E08E36920708F05AC10E94952B20E857
:107E500031E541E050E00E942F7559016901CE18CB
:107E6000DF083EC0C4016EE377E040E827EE36E06D
:107E700001E0EE24FF240E94C331882309F441C1AC
:107E80008EE397E00E94B9075B016C01C4016EE3C9
:107E900077E040E823EE36E00E94C331882309F4FE
:107EA00030C1C601B50120E831E541E050E00E9453
:107EB000517569018EE397E00E94B90720E831E52A
:107EC00041E050E00E94517559012C153D0508F420
:107ED00016C1C9018C199D098E56914008F00FC139
:107EE00019821A821B821C82C4012E010894411C33
:107EF000511CB20144E02EED36E001E0EE24FF24F7
:107F00000E94C3318BA380E00E94033300D000D0D5
:107F100007EE16E0ADB7BEB712961C930E931197FD
:107F20008CED96E014969C938E9313970E948B1180
:107F300099240F900F900F900F90F9E06F2E712CF5
:107F40006C0E7D1E802E012FEAED2E2EE6E03E2ED9
:107F5000B4C0C6016EE377E04AE050E00E948D08AD
:107F60008EE397E00E9479158EEA96E06EE377E063
:107F70000E94E769882309F49DC019861B8618862C
:107F80001F82EBE7F2E0FE83ED83C3016EE377E04F
:107F900041E00E94356802C099249394C3016EE3C6
:107FA00077E040E850E020E030E00E943C631816A3
:107FB000190624F0C3010E9424607CC01092BD0702
:107FC000EEE3F7E001C0FB018081882339F3BF01B4
:107FD0006F5F7F4F8C32B9F77B010894E11CF11C75
:107FE000FBA1FF2349F0C201B70142E050E00E942B
:107FF0003808009799F613C08AE991E0B70142E08A
:1080000050E00E943808009749F28DE991E0B701ED
:1080100042E050E00E943808009709F4BFCF992051
:10802000A1F000D000D0ADB7BEB711968C921197D9
:1080300012960C93129714963C922E9213970E94CC
:108040008B110F900F900F900F9000D000D000D0A8
:10805000EDB7FEB73196ADB7BEB711968C921197BA
:1080600012960C9327ED36E0338322838EE397E05C
:10807000958384830E948B118091ED069091EE068A
:108080002091EB063091EC06821B930BA0ECB3E041
:10809000A81BB90BEDB7FEB736960FB6F894FEBF26
:1080A0000FBEEDBFA035B1050CF076CF80E00E9489
:1080B000BF3D72CF0894C11CD11CAC14BD0408F0A4
:1080C00048CF00D000D087EE96E0ADB7BEB712968D
:1080D0009C938E93119785ED96E014969C938E93C6
:1080E00013970E948B110F900F900F900F9061E0EB
:1080F00070E080E090E00E94E75680E003C081E1FC
:1081000001C080E1A3960FB6F894DEBF0FBECDBFCD
:10811000CF91DF911F910F91FF90EF90DF90CF9063
:10812000BF90AF909F908F907F906F905F904F9097
:108130003F902F900895CF92DF92EF92FF920F938E
:108140001F93CF93DF936C016EE377E040E828E460
:1081500037E001E0EE24FF240E94C331882311F0B0
:108160000E944214C6016EE377E040E824E437E061
:1081700001E0EE24FF240E94C331882371F08EE3D6
:1081800097E00E949B07181619063CF40E94523390
:1081900081E00E94BF3D0E94C020C6016EE377E0EF
:1081A00040E821E437E001E0EE24FF240E94C331DF
:1081B000882399F080913E07813339F4809110072C
:1081C00080FD0BC00E94982608C0803331F4809156
:1081D000100780FF02C00E948E26C6016EE377E082
:1081E00040E82EE337E001E0EE24FF240E94C33193
:1081F000882361F18EE397E00E949B07EC0118163B
:108200001906F4F40E94952B7B018C01BE0188278E
:1082100077FD8095982F20E13EE040E050E00E94FD
:10822000DD74E60EF71E081F191FE0920807F09292
:10823000090700930A0710930B070E94BE2606C089
:10824000009711F081E126C00E94AE26C6016EE3C0
:1082500077E040E82BE337E001E0EE24FF240E94C2
:10826000C3318823B1F080913E07813341F480917E
:10827000EA01882371F481E08093EA0108C0803329
:1082800041F48091EA01882321F01092EA010E94D2
:10829000932581E0DF91CF911F910F91FF90EF9097
:1082A000DF90CF9008952F923F924F925F927F92EE
:1082B0008F929F92AF92BF92CF92DF92EF92FF92F6
:1082C0000F931F93DF93CF9300D00F92CDB7DEB7FC
:1082D0000E94952B5B016C012DB73EB722533040B5
:1082E0000FB6F8943EBF0FBE2DBFEDB7FEB7319667
:1082F00007EE16E0ADB7BEB712961C930E9311971A
:108300008CE898E093838283A482B582C682D78268
:10831000809119078087118680911007817082876C
:1083200013868091100786958170848715868091C9
:108330001007869586958170868717868091080735
:1083400090910907A0910A07B0910B07808B918B40
:10835000A28BB38B84E194E0958B848B84E994E0C9
:10836000978B868B8091040790910507918F808F62
:108370008091060790910707938F828F80910C0759
:1083800090910D07A0910E07B0910F07848F958FE4
:10839000A68FB78F8091360790913707A091380745
:1083A000B091390780A391A3A2A3B3A380913A0708
:1083B00090913B07A0913C07B0913D0784A395A302
:1083C000A6A3B7A380918B0980A711A680918C09E1
:1083D00082A713A680918D0990918E0995A784A7F5
:1083E00080918F0990919009A0919109B091920983
:1083F00086A797A7A0ABB1AB0E948B11EDB7FEB7D4
:10840000F2960FB6F894FEBF0FBEEDBF8091D40177
:10841000823081F52DB73EB72A5030400FB6F89420
:108420003EBF0FBE2DBFEDB7FEB73196ADB7BEB79D
:1084300012961C930E93119785E798E0938382839D
:108440008091290790912A07A0912B07B0912C07C2
:1084500084839583A683B7838EE190E0918780879C
:108460000E948B11EDB7FEB73A960FB6F894FEBF97
:108470000FBEEDBF00D000D007EE16E0ADB7BEB71F
:1084800012961C930E9311978BE698E014969C938A
:108490008E9313970E948B1190E00F900F900F9086
:1084A0000F90780107E618E023C000D000D000D07C
:1084B000EDB7FEB73196ADB7BEB71196EC921197F6
:1084C0001296FC9213830283A92FB0E0A55EB84FE9
:1084D0008C918483158299830E948B1199819F5F6F
:1084E000EDB7FEB736960FB6F894FEBF0FBEEDBFE0
:1084F0008091190727EE422E26E0522E9817A8F2F7
:1085000000D000D0ADB7BEB712965C924E921197D4
:108510008DE598E014969C938E9313970E948B118F
:1085200099240F900F900F900F90C201742C892EF8
:1085300012E5212E18E0312EB0EC4B2EB3E05B2E6D
:108540009AC0E92DF0E0FB83EA83E55AF64FE0811B
:10855000EF3F61F1F0E0A3E0EE0FFF1FAA95E1F716
:10856000E552F84FE080F18002811381848195818A
:10857000AE14BF04C006D106A8F09C0140E050E054
:108580002E0D3F1D401F511F2A193B094C095D0943
:10859000203060E0360761E0460760E0560708F0EB
:1085A000CBC0CEC09C0140E050E0CAC0EE24FF2406
:1085B000870180E090E020E030E040E050E0ADB79F
:1085C000BEB71E970FB6F894BEBF0FBEADBFEDB7D6
:1085D000FEB7319611967C92119712968C92338247
:1085E0002282958384832683378340875187E2865E
:1085F000F386048715870E948B1180911A0790E0FB
:108600000197EDB7FEB73E960FB6F894FEBF0FBECA
:10861000EDBF2A813B81281739071CF08EE498E0D2
:1086200002C080E598E000D000D0ADB7BEB711968B
:108630007C92119712968C92129714969C938E931B
:1086400013970E948B118091ED069091EE06209178
:10865000EB063091EC06821B930BF201E81BF90B41
:108660000F900F900F900F90E035F1051CF480E013
:108670000E94BF3D939480911A07981608F461CF29
:108680000EE317E086E191E0B80140E850E020E019
:1086900030E00E94BA528823F1F000D000D000D020
:1086A000EDB7FEB7319687EE96E0ADB7BEB712963E
:1086B0009C938E93119782E498E093838283158331
:1086C00004830E948B11EDB7FEB736960FB6F8946F
:1086D000FEBF0FBEEDBF00D000D087EE96E0ADB775
:1086E000BEB712969C938E93119780E498E01496EF
:1086F0009C938E9313970E948B110F900F900F9065
:108700000F9061E070E080E090E00E94E7560F90EB
:108710000F900F90CF91DF911F910F91FF90EF90ED
:10872000DF90CF90BF90AF909F908F907F905F90A1
:108730004F903F902F90089520E030E040E050E0CF
:10874000878190E03CCF81E00E9403330E94534137
:1087500080E008952F923F924F925F926F927F92A6
:108760008F929F92AF92BF92CF92DF92EF92FF9241
:108770000F931F93DF93CF93CDB7DEB7C754D0408D
:108780000FB6F894DEBF0FBECDBF2DB73EB72E504B
:1087900030400FB6F8943EBF0FBE2DBFEDB7FEB709
:1087A000319607EE16E0ADB7BEB712961C930E9346
:1087B000119785E59BE0938382838091D907848319
:1087C000158280911907868317828EE090E0918749
:1087D000808784E090E0938782878CE090E09587A3
:1087E00084870E948B11EE24EDB7FEB73E960FB63C
:1087F000F894FEBF0FBEEDBFF02E012F75E4C72E1B
:108800007BE0D72E6CE0862E912C8C0E9D1EAF2C1B
:10881000B12E5BE2252E5BE0352E4EE2442E4BE07E
:10882000542E30EC632E33E0732E4AC18E2DBE01E0
:108830006F5F7F4F0E94DD30898182958370833026
:1088400039F48B81823020F0CE0102960E94742F81
:108850002DB73EB72A5030400FB6F8943EBF0FBE3A
:108860002DBFEDB7FEB73196ADB7BEB71196FC92EE
:10887000119712960C9329E43BE03383228389817C
:10888000848315828A81868317828B8180871186F3
:108890000E948B110F900F900F900F90EDB7FEB7C5
:1088A0003196ADB7BEB71196FC92119712960C9304
:1088B000D382C2828C819D81958384830E948B1197
:1088C000EDB7FEB73196ADB7BEB71196FC921197D2
:1088D00012960C93D382C2828E819F81958384836A
:1088E0000E948B11EDB7FEB73196ADB7BEB71196AA
:1088F000FC92119712960C93D382C2828885998537
:10890000958384830E948B11EDB7FEB73196ADB786
:10891000BEB71196FC92119712960C932FE33BE091
:10892000338322838A859B85958384830E948B1160
:1089300010E04DB75EB74A5F5F4F26C0E80DF91DE6
:1089400080810E940052ADB7BEB718970FB6F89459
:10895000BEBF0FBEADBFEDB7FEB731961196FC920C
:10896000119712960C932BE33BE033832283A0E014
:10897000B0E084839583A683B7830E948B111F5F29
:108980004DB75EB7485F5F4F0FB6F8945EBF0FBE3E
:108990004DBFE12FF0E080911A0790E00197E817B2
:1089A000F90764F2E80DF91D80810E940052ADB70D
:1089B000BEB718970FB6F894BEBF0FBEADBFEDB7E8
:1089C000FEB731961196AC9211971296BC9225E3A0
:1089D0003BE033832283A0E0B0E084839583A683C9
:1089E000B7830E948B114DB75EB7485F5F4F0FB6DC
:1089F000F8945EBF0FBE4DBF8EE397E0BE01645C8E
:108A00007F4F4CE050E00E94460810924A0700D089
:108A100000D000D0EDB7FEB73196ADB7BEB7119616
:108A2000AC9211971296BC9222E33BE033832283EF
:108A30004EE357E0558344830E948B112E2D30E086
:108A40008091D90790E00197ADB7BEB716960FB6E3
:108A5000F894BEBF0FBEADBF2817390749F000D04C
:108A600000D0EDB7FEB7F1820283548243820EC07C
:108A700000D000D0ADB7BEB71196FC9211971296F8
:108A80000C93129714963C922E9213970E948B117E
:108A90000F900F900F900F908091ED069091EE0641
:108AA0002091EB063091EC06821B930BF301E81B3F
:108AB000F90BEA3FF1051CF480E00E94BF3DE3940E
:108AC0008091D907E81608F4B1CE00D000D087EE27
:108AD00096E0ADB7BEB712969C938E93119788E23D
:108AE0009BE014969C938E9313970E948B110F908A
:108AF0000F900F900F9061E070E080E090E00E9496
:108B0000E756C95BDF4F0FB6F894DEBF0FBECDBF8F
:108B1000CF91DF911F910F91FF90EF90DF90CF9059
:108B2000BF90AF909F908F907F906F905F904F908D
:108B30003F902F90089581E00E9403330E94AA4342
:108B400080E008958F929F92AF92BF92CF92DF9272
:108B5000EF92FF920F931F93CF93DF9381E49CE0FA
:108B60006CEA77E00E94BC3B85E39CE062EB77E037
:108B70000E94BC3B8EE29CE068EB77E00E94BC3B2D
:108B800086E29CE06EEB77E00E94BC3B8EE19CE0CD
:108B900064EC77E00E94BC3B8091100785FF06C023
:108BA00086E19CE06AEC77E00E94BC3B00D000D0FC
:108BB00007EE16E0ADB7BEB712961C930E93119751
:108BC0008BE09CE014969C938E9313970E948B11DC
:108BD000FF240F900F900F900F90E02E012FAEE327
:108BE0008A2EA7E09A2EF6E0AF2EFCE0BF2EE4E03E
:108BF000CE2EECE0DE2EC0ECD3E051C08F2D6EE324
:108C000077E00E94372700D000D000D0EDB7FEB744
:108C10003196ADB7BEB71196EC92119712960C93A0
:108C2000B382A282958284820E948B112F2D30E024
:108C300080911A0790E00197EDB7FEB736960FB610
:108C4000F894FEBF0FBEEDBF28173907A1F000D082
:108C500000D0ADB7BEB71196EC92119712960C9357
:108C600012971496DC92CE9213970E948B110F905C
:108C70000F900F900F908091ED069091EE0620914D
:108C8000EB063091EC06821B930BFE01E81BF90BFF
:108C9000E035F1051CF480E00E94BF3DF394809123
:108CA0001A07F81608F4AACF00D000D000D0EDB70C
:108CB000FEB7319687EE96E0ADB7BEB712969C939D
:108CC0008E93119785EF9BE09383828380E190E000
:108CD000958384830E948B11EDB7FEB736960FB64D
:108CE000F894FEBF0FBEEDBF61E070E080E090E061
:108CF0000E94E756DF91CF911F910F91FF90EF9067
:108D0000DF90CF90BF90AF909F908F90089581E0BB
:108D10000E9403330E94A24580E008950F931F93A1
:108D200081E00E94033300D000D007EE16E0EDB7DB
:108D3000FEB71283018384EC96E0948383830E94C0
:108D40008B110F900F900F900F900E94534180E075
:108D50000E94BF3D00D000D0EDB7FEB71283018363
:108D600086EB96E0948383830E948B110F900F9083
:108D70000F900F900E94AA4380E00E94BF3D00D058
:108D800000D0EDB7FEB71283018389EA96E09483A1
:108D900083830E948B110F900F900F900F900E9471
:108DA000173880E00E94BF3D00D000D0EDB7FEB77D
:108DB000128301838DE996E0948383830E948B1153
:108DC0000F900F900F900F900E940E3480E00E9441
:108DD000BF3D00D000D0EDB7FEB7128301838FE80E
:108DE00096E0948383830E948B110F900F900F90D5
:108DF0000F900E94A24500D000D0EDB7FEB71283BD
:108E000001838DE896E0948383830E948B110F90F9
:108E10000F900F900F9061E070E080E090E00E9472
:108E2000E75680E01F910F910895DF92EF92FF9235
:108E30000F931F93CF93DF93D82E862FBA01213043
:108E400041F4675F7F4F9B0140E050E06950704004
:108E50000EC0223029F020E030E040E050E007C0B2
:108E6000625070409B0140E050E06E5F7F4FE82E03
:108E7000FF248EEE92E0E80EF91E8B01E7010FC091
:108E8000F881E0E0898190E08E2B9F2BA0E0B0E09C
:108E9000280F391F4A1F5B1F2296025010400230D4
:108EA000110570F7CB018E7FD701A80FB91F681786
:108EB000790779F08C9190E0A0E0B0E0BA2FA92F6B
:108EC000982F882702C040E050E0280F391F4A1F22
:108ED0005B1FCA01AA27BB270097A105B10599F717
:108EE000C90180959095ED2DF0E0E251FD4F908302
:108EF0008183DF91CF911F910F91FF90EF90DF90D1
:108F00000895109206031092070380E480930203F1
:108F1000109203038093040388E16EE044E150E083
:108F200020E00E9415470895282F662321F08091A4
:108F300013038617E1F4809114038823C1F4809110
:108F400015038833A1F4809111038B3781F4E22F4C
:108F5000F92F809140038383809141038283809124
:108F60004203818380914303808381E0089580E000
:108F700008958091970986958095817008958091D4
:108F8000D20280959091CE02892B8093D602809157
:108F9000D30280959091CF02892B8093D702809144
:108FA000D40280959091D002892B8093D802809131
:108FB000D50280959091D102892B8093D902089592
:108FC0009093AC098093AB097093B6096093B5098F
:108FD0005093AE094093AD098FED9DE09093B00999
:108FE0008093AF091092B2091092B1093093B4097D
:108FF0002093B3093091B6012091B70186E49EE435
:1090000090939F0980939E0986E89DE49093A1091F
:109010008093A00920939A0930939B0981E0809363
:109020009809809199098F5F87708093990980933F
:10903000AA0908950F931F93BC010EEE12E0C80118
:109040000E943C55C801069668EC72E00E943C55AF
:109050001F910F910895EF92FF920F931F937B0141
:109060000E941A480CE013E0C801B7010E94445561
:10907000C80104976EEC72E00E9444551F910F9155
:10908000FF90EF900895EF92FF920F931F93CF936D
:10909000DF937C01EB018A0182EA99E00E942B4870
:1090A0008881807F803E49F088819981AA81BB8137
:1090B0008F5F9F4FAF4FBF4F31F48EEE92E065E46C
:1090C00072E00E943C5588E08093FA021092FB0205
:1090D0008CEF92E06AE37DE049E050E00E94E30714
:1090E0001092FE0281E18093050310931203009316
:1090F0001303F0921003E0921103109214031092E4
:10910000160310921703DF91CF911F910F91FF90DB
:10911000EF900895EF92FF920F931F9304EF12E0E8
:10912000C8010E941A4874E1E72EF12CE00EF11EEE
:10913000C8014896B7010E944455C7016EEC72E021
:109140000E9444550E9481471F910F91FF90EF901C
:109150000895BC011092ED021092EC0281E0809320
:1091600097098AED92E00E94445508950F931F934A
:109170008C0188969093FE028093FF020E948147A3
:109180001092200310922103045E1F4F82E36AE1D4
:10919000A80122E00E941547C8014A960E94F30FD9
:1091A0001F910F910895EF92FF920F931F937C01EF
:1091B0008091B7099091B809A091B909B091BA0905
:1091C0002B2F33274427552720931403A0931503EF
:1091D000909316038093170360931D03C7010E94A9
:1091E000B64800E010E08091B7099091B809A091CD
:1091F000B909B091BA098E0D9F1DA01FB11F8093B0
:10920000B7099093B809A093B909B093BA091F910F
:109210000F91FF90EF900895CF93DF939C01862FDD
:10922000806180931D03643029F02115310511F40C
:1092300021E030E09091120380911003809312039B
:109240009093100390911303809111038093130363
:1092500090931103C7E1D3E08881A901480F511D04
:109260002C814C832883252F3327219753E0C3314A
:10927000D50791F71D861E8680E589871092FE022C
:1092800088E28093FF020E948A4884E08B871C86D4
:1092900082E36AE14CE150E022E00E94154786E358
:1092A00090E00E94F30FDF91CF9108958091A8097B
:1092B0009091A90960E00E940C498091140390E00C
:1092C000A0E0B0E0BA2FA92F982F8827209115038E
:1092D000820F911DA11DB11DBA2FA92F982F88278C
:1092E00020911603820F911DA11DB11DBA2FA92F28
:1092F000982F882720911703820F911DA11DB11D62
:109300008093B7099093B809A093B909B093BA09AB
:109310000895E82F4091120350E0292F30E04217C2
:10932000530709F092C0809113038E1709F08DC086
:1093300080911D03E82F81FF4EC01092FE028CE247
:109340008093FF020E948A4882E180931D039091DE
:109350001203809110038093120390931003909155
:109360001303809111038093130390931103E7E19A
:10937000F3E021E030E08081A901480F511D4483D2
:109380001082252F3327319753E0E331F50799F702
:1093900015861686118212828091160283831482AA
:1093A0008D5F8093160282E0818B84E0828B95E052
:1093B000938B148A80E68187938788E7848782E38A
:1093C0006AE140E250E022E00E9415478AE390E023
:1093D0000E94F30F3AC084FF38C09091FE0280E0F3
:1093E0002091FF0230E0282B392B80911C03482F5D
:1093F00050E0A4E055954795AA95E1F7CA01880F7A
:10940000991F880F991F281B390B2451304037FFB3
:1094100002C020E030E03093A9092093A809232B53
:1094200069F09A01220F331F220F331F2E5D3F4F29
:10943000685070406217730740F009C0E0FF05C034
:1094400080E090E060E00E940C4920E030E0C9013B
:1094500008950F931F93DF93CF930F92CDB7DEB78D
:109460008C01045E1F4F1093FE020C511040802FA0
:10947000845E8093FF0289830E948147085F1F4FAB
:10948000109314038981845180931503085F1F4F43
:1094900088E26AE1A80121E00E941547C8014A96C6
:1094A0000E94F30F0F90CF91DF911F910F910895BC
:1094B000FF920F931F939C01F62E82EA99E0B90167
:1094C0000E942B480AEF12E088E08093FA02109283
:1094D000FB02C80102966AE37DE049E050E00E9489
:1094E000E3078CE48093FF0281E1809305030E94EF
:1094F0008147109212038BE7809313038AE08093D5
:109500001003F09211031092140388E38093150363
:109510001092160310921703025E1F4F80E3F801AA
:1095200011928A95E9F7C80161EF7DE04AE050E0C9
:109530000E94E30788E26AE140E450E021E00E94F3
:1095400015478AE590E00E94F30F1F910F91FF905D
:109550000895EF92FF920F931F93BC0182EA99E066
:109560000E942B480AEF12E088E0F82EF092FA02EF
:109570001092FB02C80102966AE37DE049E050E0E8
:109580000E94E30784E58093FF02EE24E394E092D7
:1095900005030E948147F09210031092110310926C
:1095A00012031092130385E0809314038091D1027B
:1095B0008093150310921603E0921703C8014E968C
:1095C00062E470E048E350E00E94140884E262E242
:1095D00040E450E020E00E94154782E690E00E94BF
:1095E000F30F1F910F91FF90EF900895DF92EF928C
:1095F000FF920F931F93CF93DF93EC018091EA02C8
:10960000882319F0CE010E94100A209709F0BFC0EC
:10961000809197098570F1F18091EC029091ED02B3
:10962000892BC1F50E942B0F8823A1F185E492E0DC
:109630000E941A4888E08093FA02E6E0FE2EF0923B
:10964000FB028CEF92E062E37DE048E050E00E9494
:10965000E3070EE013E0D8011D92FA94E9F7C80180
:109660000A9768EC72E00E943C55C80106966AEDC4
:1096700072E00E944455C80104976EEC72E00E94AB
:109680004455809197098860809397098AE290E019
:109690000E94F30F8091EC029091ED02019690935D
:1096A000ED028093EC0280919809813009F003C2A9
:1096B0008091970981FFFFC102E000939809809192
:1096C00015028F5F809315028F7110919909129581
:1096D000110F107E182BE0909A09D0909B0982EA16
:1096E00099E066EE72E00E942B4878E0F72EF09247
:1096F000FA021092FB028CEF92E06AE37DE049E00F
:1097000050E00E94E3078CE28093FF0286E08093A2
:1097100005030E948147E0921203D09213038BE06D
:109720008093100310931103E4E1F3E0DF011D9235
:10973000FA94E9F780911602809316038D5F809367
:10974000160280E680931C0300931D0383E0809340
:109750001E0310921F0310922003109221031092F7
:109760002203109223030093240384E080932503B3
:109770000093260386E28093270382E36AE140E2B6
:1097800050E022E00E9415478AE390E0AFC0C93262
:10979000D10508F490C11091FA02183009F096C171
:1097A0008091FB02863009F091C184E193E06EEC78
:1097B00072E044E050E00E94FE07009709F086C185
:1097C00080910303813029F584EF92E00E941A48CA
:1097D0001092020382E0809303038EE093E064E042
:1097E00073E00E943C5584E093E068EC72E00E94D4
:1097F0003C5584E193E06AE073E00E9444558AE0BE
:1098000093E06EEC72E00E9444558AE290E00E9480
:10981000F30F8091970983FF4EC11091030312301B
:1098200009F049C18AE093E06AED72E044E050E05B
:109830000E94FE07009709F03EC182EA99E064E0C9
:1098400073E00E943C551093970935C1183009F018
:1098500032C18091FB02882309F02DC18091FC0266
:10986000853409F028C18CE093E06EEC72E044E0AE
:1098700050E00E94FE070097A9F08CE093E066EDAF
:1098800072E044E050E00E94FE07009759F08CE03F
:1098900093E065E472E044E050E00E94FE07009728
:1098A00009F009C180910503813019F580911003F9
:1098B0008830F9F4E0919C09F0919D09309719F0F6
:1098C00088E093E009950E948A48109210038091E5
:1098D0001203883F28F0809113038F5F8093130356
:1098E00080911203885F80931203CE010E94F30FD0
:1098F000E2C00E946751882351F0809105038131B5
:1099000031F4CE010E946C51882309F0D4C0C633D3
:10991000D10528F480910503863009F0CCC08091F0
:1099200012038B3009F0BEC088E093E066EE72E06F
:1099300044E050E00E94FE07009709F0BCC080910F
:109940001D03382F82FF13C0E0919E09F0919F09FB
:10995000309759F08091130382958695877063E064
:1099600040E050E020E030E0099585E090C0909123
:10997000FE0280E02091FF02022F10E0082B192B3D
:1099800080911C03482F50E064E0559547956A95F7
:10999000E1F7CA01880F991F880F991F081B190B3F
:1099A0000451104017FF02C000E010E080919809B8
:1099B000823079F531FF21C034FF1FC080E090E094
:1099C00060E00E940C4988E180931D03E091A009AA
:1099D000F091A109309719F420E030E007C08091A0
:1099E000110382958695877009959C0183E0809389
:1099F0009809C9010E94B6485EC081E08093980929
:109A000034FF03C080E090E002C0C801019664E02A
:109A100046C0833081F50115110579F1E0919E0969
:109A2000F0919F09309749F1440F551F440F551F7E
:109A3000CE0108974E5D5F4F8417950708F4AC017F
:109A4000C801840F951FC817D90710F0980103C0EB
:109A50009E01241B350B8091130382958695877098
:109A600060E009958091EB02882319F0C80168E055
:109A700016C0C80108C08530F1F030FF0BC083303C
:109A8000D1F0C801019669E00E940C4986E08093FC
:109A9000980911C00115110571F0C80160E00E941C
:109AA0000C4909C08091B6019091B701BE010E9496
:109AB00089499C0102C020E030E0C901DF91CF91CB
:109AC0001F910F91FF90EF90DF900895CA32D1055A
:109AD00008F0BCCEF0CFBC01809105038130A1F429
:109AE00080911003882381F480911803823461F4FB
:109AF00088E093E044E050E00E94FE079C0180E093
:109B0000232B19F481E0089580E00895CF92DF922D
:109B1000EF92FF920F931F93DF93CF93CDB7DEB7F2
:109B200028970FB6F894DEBF0FBECDBF24E233E016
:109B30003E832D8338872F839091AA09891709F0D6
:109B40008FC01C821B8286E392E09A8389834091B6
:109B5000B1095091B20941155105A9F58DB79EB7CC
:109B60000C970FB6F8949EBF0FBE8DBFEDB7FEB732
:109B70003196CE010196ADB7BEB712969C938E93E7
:109B800011978BEB9DE0938382838091AB09909139
:109B9000AC09958384838091B5099091B609978328
:109BA00086838091AD099091AE09918780878091DD
:109BB000AF099091B009938782870E948B118DB76E
:109BC0009EB70C9648C02091AF093091B009E09043
:109BD000AB09F090AC090091AD091091AE092115C7
:109BE000310519F060EA71E004C063EA71E023E432
:109BF0003DE0DA010D900020E9F76D010894C108FD
:109C0000D108C41AD50A8DB79EB740970FB6F894FD
:109C10009EBF0FBE8DBFEDB7FEB73196CE01019648
:109C2000ADB7BEB712969C938E93119784E49DE0D6
:109C300093838283F582E4821783068331872087AA
:109C400073876287D586C486578746870E948B11A3
:109C50008DB79EB740960FB6F8949EBF0FBE8DBFCE
:109C60002F8138858D819E81281B390BC90128964B
:109C70000FB6F894DEBF0FBECDBFCF91DF911F911D
:109C80000F91FF90EF90DF90CF9008950F931F9367
:109C9000CF93DF9389019091AA09891759F0E09138
:109CA000B309F091B40984E060E070E040E050E076
:109CB00009952AC0662341F52D30310528F1C09160
:109CC000B309D091B4092097F9F049505D4F84EA67
:109CD00091E0BA0143E050E00E9438089C0180E026
:109CE000232B09F081E060911C0370E0B4E07595CE
:109CF0006795BA95E1F7660F771F660F771F6E5D60
:109D00007F4FA801FE01099580E0DF91CF911F915F
:109D10000F9108958F929F92AF92BF92CF92DF9250
:109D2000EF92FF920F931F93CF93DF937B018C01F0
:109D3000EA012CE330E040E050E00E942F75688398
:109D4000C801B7012CE330E040E050E00E942F75DD
:109D5000122F032FF42EE52E622F732F842F952FB1
:109D60002CE330E040E050E00E942F756983612FC2
:109D7000702F8F2D9E2D2CE330E040E050E00E94AC
:109D80002F75122F032FF42EE52E622F732F842FA1
:109D9000952F28E130E040E050E00E942F756A8363
:109DA000612F702F8F2D9E2D28E130E040E050E094
:109DB0000E942F7579018A01C801B7016C5F7F4F3E
:109DC0008F4F9F4F27E030E040E050E00E942F751A
:109DD0006F5F6B8320E0AA24BB24650101C02F5F65
:109DE000822E9924F401EE54F84FCF0183709070C5
:109DF000892B99F4CF0164E670E00E941C75892BD1
:109E000039F4CF0160E971E00E941C75892B29F4B7
:109E10008EE691E0A0E0B0E004C08DE691E0A0E025
:109E2000B0E0A80EB91ECA1EDB1EC501A0E0B0E05E
:109E3000E816F9060A071B0790F62E83F401EE5484
:109E4000F84F83E0882E912C8E229F22811491045A
:109E500099F4CF0164E670E00E941C75892B39F4F7
:109E6000CF0160E971E00E941C75892B29F48EE610
:109E700091E0A0E0B0E004C08DE691E0A0E0B0E0A9
:109E8000A81AB90ACA0ADB0A980187010A191B092C
:109E90002C093D09CF0164E670E00E941C757C012D
:109EA000CF0160E971E00E941C75AC01EBE4F2E0C7
:109EB00060E0613051F48114910449F4E114F1043B
:109EC00041F44115510529F002C0808103C08CE1A5
:109ED00001C08DE190E0A0E0B0E0081719072A0763
:109EE0003B0740F0081B190B2A0B3B0B6F5F3196A9
:109EF0006C30F9F66F5F6D83802F8F5F8C83DF91FD
:109F0000CF911F910F91FF90EF90DF90CF90BF9076
:109F1000AF909F908F900895EF92FF920F931F93B1
:109F20007B018C018091D2099091D309A091D40931
:109F3000B091D509E816F9060A071B0771F0C801A8
:109F4000B70147EC59E00E948A4EE092D209F092A4
:109F5000D3090093D4091093D5091F910F91FF9055
:109F6000EF9008950E948C4F8091CC0990E0089565
:109F70000E948C4F8091CA0990E008950E948C4FF6
:109F80008091CB0990E008950E948C4F8091C80980
:109F900090E008950E948C4F8091C90990E0089547
:109FA0004F925F926F927F928F929F92AF92BF92E9
:109FB000CF92DF92EF92FF920F931F93CF93DF9395
:109FC0004C01DC0116961C91612F70E080E090E05E
:109FD00020E833E341EE51E00E94DD745B016C0147
:109FE00022EB37E0E12FF0E0EE54F84F1DC0C9013D
:109FF00083709070892BB1F4C90164E670E00E940F
:10A000001C75892B39F4C90160E971E00E941C7547
:10A01000892B41F480E891E5A1E0B0E0A80EB91EDB
:10A02000CA1EDB1E2F5F3F4F2E173F0701F7D401DB
:10A0300015968C91482E5524C90164E670E00E9463
:10A040001C757C01C90160E971E00E941C758C01DE
:10A05000C1E0D0E093E0692E712C6222732227C008
:10A06000C230D10591F46114710479F4E114F10462
:10A0700019F40115110549F480E89BE3A6E2B0E06C
:10A08000A80EB91ECA1EDB1E11C0FE01E65BFD4F05
:10A09000608170E080E090E020E831E541E050E050
:10A0A0000E94DD74A60EB71EC81ED91E2196C415C7
:10A0B000D505B4F2D40112966C9170E080E090E086
:10A0C00020E13EE040E050E00E94DD747B018C0125
:10A0D000F401618170E080E090E02CE330E040E04A
:10A0E00050E00E94DD74E60EF71E081F191FD40110
:10A0F0008C91E80EF11C011D111D14966C9170E0FD
:10A1000061507040882777FD8095982F20E831E5D1
:10A1100041E050E00E94DD74E60EF71E081F191F93
:10A12000EA0CFB1C0C1D1D1DB701C801DF91CF916E
:10A130001F910F91FF90EF90DF90CF90BF90AF9065
:10A140009F908F907F906F905F904F900895609355
:10A150001702709318028093190290931A020895BF
:10A160006093BD097093BE098093BF099093C009A5
:10A1700020911702309118024091190250911A0251
:10A18000260F371F481F591F2093C1093093C2095A
:10A190004093C3095093C40982E090E09093C609AC
:10A1A0008093C5090E94D9566093CE097093CF0958
:10A1B0008093D0099093D1090895EF92FF920F9365
:10A1C0001F931CC02F5F3F4F4F4F5F4F2093BD0920
:10A1D0003093BE094093BF095093C00988EE93E0C5
:10A1E000A0E0B0E0E80EF91E0A1F1B1FE092CE09A6
:10A1F000F092CF090093D0091093D1090E94D9564B
:10A20000E090CE09F090CF090091D0091091D109CA
:10A210006E197F09800B910B2091BD093091BE0909
:10A220004091BF095091C009685E734080409040E2
:10A2300048F68091C1099091C209A091C309B091DB
:10A24000C409281739074A075B07E8F0E091BB0902
:10A25000F091BC093097B9F0099561157105810538
:10A26000910519F00E94B0500EC020E030E08091BE
:10A27000C5099091C609892B11F021E030E0309397
:10A28000C6092093C5096091BD097091BE098091EE
:10A29000BF099091C0091F910F91FF90EF90089511
:10A2A0009093BC098093BB098091BD099091BE0930
:10A2B000A091BF09B091C0098093C1099093C209D0
:10A2C000A093C309B093C4090E94DD500895809102
:10A2D000FE09811181E00895CF92DF92EF92FF9203
:10A2E0000F931F93CF93DF93C6EDD9E0CC24DD24E9
:10A2F00030E029C02A814B818091120390E0042F25
:10A3000010E080179107D9F4909113039217B9F4D4
:10A310008C818823A1F02091150330E02850304033
:10A32000F0901403EE242E0D3F1DE881F981892F52
:10A33000942F68E073E048E153E0099531E0089418
:10A34000C11CD11C25968091FE0990E0C816D90643
:10A350008CF2832FDF91CF911F910F91FF90EF909F
:10A36000DF90CF900895DC019B0105C0F9012F5FBC
:10A370003F4FE491ED93822F861B90E08417950761
:10A38000ACF31C920895FC01CB01F999FECF92BD6C
:10A3900081BDF89A30B52081332349F0222339F06A
:10A3A0000196321711F081E008953196EECF80E0EA
:10A3B000321381E008958C33910510F4682F1EC08C
:10A3C0002AE28033920730F46CE370E00E94087553
:10A3D000655C14C021EE8130920730F460E17EE0CC
:10A3E0000E94087564510AC02FEF8E3F920729F032
:10A3F0008F5F9F4F11F46FEF01C06EEF862F0895AE
:10A40000282F30E08C3338F18F3E68F48CE390E0F5
:10A41000A901489F9001499F300D589F300D11248C
:10A42000245D3D4018C08D3F68F480E19EE0A901A5
:10A43000489F9001499F300D589F300D1124205C9A
:10A44000364F09C08E3F29F08F3F19F42FEF3FEFB1
:10A4500002C02EEF3FEFC90108952FEF8E3F920704
:10A4600049F4609106077091070720910407309125
:10A4700005070EC02FEF8F3F9207B9F460910407D4
:10A480007091050760567A4F2091060730910707B3
:10A49000621B730B80E090E02CE330E040E050E082
:10A4A0000E94DD749B01AC0103C09C0140E050E0C0
:10A4B000B901CA010895CF93DF93EC01D7FF04C01F
:10A4C000882799278C1B9D0B0E94DB51982FD7FD65
:10A4D00002C0805802C080E8891BDF91CF910895A7
:10A4E0001F93182F90E08058904097FF03C09095DD
:10A4F00081959F4F0E9400529C0117FD03C030952B
:10A5000021953F4FC9011F9108950F931F93DF932A
:10A51000CF93CDB7DEB72C970FB6F894DEBF0FBE42
:10A52000CDBFBC018091100785FF19C08E010F5F60
:10A530001F4FC8010E94F7078EEA96E068EA71E0B3
:10A5400040E00E94EB698EEA96E0B8010E94E7695C
:10A55000882329F08EEA96E0B8010E94C4692C96FF
:10A560000FB6F894DEBF0FBECDBFCF91DF911F9124
:10A570000F9108958F929F92AF92BF92CF92DF92E8
:10A58000EF92FF920F931F93DF93CF93CDB7DEB778
:10A59000AA970FB6F894DEBF0FBECDBFFC017B01BA
:10A5A0005A0149018091100785FD04C0FB0110820A
:10A5B00080E03FC08E010F5F1F4FC801BF010E94A6
:10A5C000F7078EEA96E068EA71E040E00E94EB69E6
:10A5D000198A1B8A188A1F868BE792E09E878D87CF
:10A5E00081E1C82ED12CCC0EDD1EC601B80141E0A0
:10A5F0000E943568882319F4F701108219C0A4015C
:10A60000662757FD6095762FC6010E94BC5DC60186
:10A61000B701A50120E030E00E943C63EA0CFB1C7E
:10A620000894E108F108F7011082C6010E94246035
:10A6300081E0AA960FB6F894DEBF0FBECDBFCF91D2
:10A64000DF911F910F91FF90EF90DF90CF90BF901F
:10A65000AF909F908F900895AF92BF92CF92DF926C
:10A66000EF92FF920F931F93DF93CF93CDB7DEB797
:10A67000AA970FB6F894DEBF0FBECDBFFC016B01E9
:10A680005A0179018091100785FF37C0CE010196EC
:10A69000BF010E94F7078EEA96E068EA71E040E0A9
:10A6A0000E94EB69002319F042E550E002C042E449
:10A6B00050E08BE792E09E878D87188A1F861B8A61
:10A6C000198A8E010F5E1F4FC801BE016F5F7F4F59
:10A6D0000E943568882389F0A701662757FD609599
:10A6E000762FC8010E94BC5DCE010D96B601A50172
:10A6F0000E948C6AC8010E942460AA960FB6F89442
:10A70000DEBF0FBECDBFCF91DF911F910F91FF90A4
:10A71000EF90DF90CF90BF90AF9008959C01F99992
:10A72000FECF32BD21BDF89A80B50895EF92FF9219
:10A730000F931F93DF93CF93CDB7DEB7C454D040B0
:10A740000FB6F894DEBF0FBECDBF0EE317E0C80111
:10A750006CE674E048E250E02EE833E50E945508CC
:10A76000C80161E00E94E10B89E0E82EF12CEC0EBB
:10A77000FD1E86E191E0B7014CE350E020E030E0BF
:10A780000E94BA521C821B8286E392E09A838983DC
:10A790001E830D8318870F838DB79EB70E970FB654
:10A7A000F8949EBF0FBE8DBFEDB7FEB73196CE01B8
:10A7B0000196ADB7BEB712969C938E93119786E023
:10A7C0009EE0938382838091DE018483158284E1FD
:10A7D00094E09783868384E994E0918780878091D1
:10A7E000BF0182871386F586E4860E948B11D8010B
:10A7F0000D900020E9F71197A01BB10BA00FB11F1E
:10A8000022EB37E0EDB7FEB73E960FB6F894FEBFE9
:10A810000FBEEDBF50E342E395E213C08C91B90146
:10A8200061507040803249F4F9015083FB0140834C
:10A8300092939F012150304003C0F90180839B0116
:10A840001197F7E0AE33BF0749F78C91D9018C938C
:10A850000091B6011091B70180E590E09093B701A7
:10A860008093B6018DEF9DE0B9014BEF5DE02DE4E3
:10A8700034E50E94E0471093B7010093B601CC5B2A
:10A88000DF4F0FB6F894DEBF0FBECDBFCF91DF9183
:10A890001F910F91FF90EF900895EF92FF920F9309
:10A8A0001F93CF93DF93EB01C251DD4F01C021967F
:10A8B0008881882309F4D9C08632C9F7C7C08EE3DE
:10A8C00097E00E949B079C0185E0213A380720F41D
:10A8D0003093050720930407CE016EE377E040E84C
:10A8E00028E33EE001E0EE24FF240E94C3318823E8
:10A8F00069F08EE397E00E949B079C0185E0213A76
:10A90000380720F43093070720930607CE016EE343
:10A9100077E040E824E33EE001E0EE24FF240E94DB
:10A92000C331882361F08EE397E00E94B9076093FA
:10A930000C0770930D0780930E0790930F070E94EA
:10A94000A326CE016EE377E040E82EE23EE001E090
:10A95000EE24FF240E94C331882391F08EE397E018
:10A960000E949B079C018B3F910550F48091D6017A
:10A9700090E02817390721F02093D6010E949325F3
:10A98000CE016EE377E040E82BE23EE001E0EE240A
:10A99000FF240E94C331882391F08EE397E00E9448
:10A9A0009B079C018D36910550F48091C00190E089
:10A9B0002817390721F02093C0010E949325CE016A
:10A9C0006EE377E040E828E23EE001E0EE24FF2479
:10A9D0000E94C331882351F18EE397E00E949B07C8
:10A9E000EC0118161906F4F40E94952B7B018C01DA
:10A9F000BE01882777FD8095982F20E13EE040E05A
:10AA000050E00E94DD74E60EF71E081F191FE09249
:10AA10000807F092090700930A0710930B070E949A
:10AA2000BE2604C0009711F40E94AE260E94952B0A
:10AA3000AB01BC0140933A0750933B0760933C073E
:10AA400070933D0783E00E94D8150FC0CE016EE3DE
:10AA500077E040E82FE33EE001E0EE24FF240E948F
:10AA6000C331882309F438CF2ACFDF91CF911F91CA
:10AA70000F91FF90EF900895DC01FB0186E00190BB
:10AA80000D928150E1F708959C01FB018081918135
:10AA9000A281B381F90180839183A283B383089556
:10AAA0000E94931B08950E94061A0895833078F53A
:10AAB000E82FF0E0EE0FFF1FE150F64F7183608347
:10AAC000813069F0813018F0823009F514C080912E
:10AAD00069008C7F842B80936900E89A08958091A7
:10AAE0006900440F551F440F551F837F842B8093AB
:10AAF0006900E99A08958091690094E0440F551F18
:10AB00009A95E1F78F7C842B80936900EA9A0895E7
:10AB10001F920F920FB60F9211242F933F934F93D2
:10AB20005F936F937F938F939F93AF93BF93EF93B5
:10AB3000FF938091FF099091000A892B29F0E09101
:10AB4000FF09F091000A0995FF91EF91BF91AF9134
:10AB50009F918F917F916F915F914F913F912F9135
:10AB60000F900FBE0F901F9018951F920F920FB667
:10AB70000F9211242F933F934F935F936F937F9383
:10AB80008F939F93AF93BF93EF93FF938091010AAD
:10AB90009091020A892B29F0E091010AF091020AB2
:10ABA0000995FF91EF91BF91AF919F918F917F9107
:10ABB0006F915F914F913F912F910F900FBE0F902A
:10ABC0001F9018951F920F920FB60F9211242F937A
:10ABD0003F934F935F936F937F938F939F93AF9325
:10ABE000BF93EF93FF938091030A9091040A892BFE
:10ABF00029F0E091030AF091040A0995FF91EF9181
:10AC0000BF91AF919F918F917F916F915F914F9184
:10AC10003F912F910F900FBE0F901F901895982F76
:10AC20008E3008F09E50977080911B028295880F9D
:10AC3000880F807C892B80937C0080917A008064CF
:10AC400080937A0080917A0086FDFCCF2091780075
:10AC500040917900942F80E030E0282B392BC901F6
:10AC600008951F93CF93DF93182FEB0161E00E94AB
:10AC70008557209709F44AC0CF3FD10509F449C050
:10AC8000E12FF0E0EB55F14F84918330C1F0843037
:10AC900028F4813051F08230B1F50CC0863019F1C2
:10ACA000873049F1843079F514C084B5806884BD5B
:10ACB000C7BD33C084B5806284BDC8BD2EC080913D
:10ACC0008000806880938000D0938900C0938800C2
:10ACD00024C080918000806280938000D0938B009C
:10ACE000C0938A001AC08091B00080688093B00041
:10ACF000C093B30012C08091B00080628093B00016
:10AD0000C093B4000AC0C038D1051CF4812F60E0A4
:10AD100002C0812F61E00E94C457DF91CF911F9143
:10AD200008951F920F920FB60F9211242F933F9305
:10AD30008F939F93AF93BF938091090A90910A0AD2
:10AD4000A0910B0AB0910C0A30910D0A0196A11D39
:10AD5000B11D232F2D5F2D3720F02D570196A11DFA
:10AD6000B11D20930D0A8093090A90930A0AA093BB
:10AD70000B0AB0930C0A8091050A9091060AA091E3
:10AD8000070AB091080A0196A11DB11D8093050A1A
:10AD90009093060AA093070AB093080ABF91AF9157
:10ADA0009F918F913F912F910F900FBE0F901F9009
:10ADB00018958FB7F8942091090A30910A0A4091AA
:10ADC0000B0A50910C0A8FBFB901CA0108959B016B
:10ADD000AC017FB7F8948091050A9091060AA09182
:10ADE000070AB091080A66B5A89B05C06F3F19F025
:10ADF0000196A11DB11D7FBFBA2FA92F982F8827BB
:10AE0000860F911DA11DB11D62E0880F991FAA1F19
:10AE1000BB1F6A95D1F7BC012DC0FFB7F894809194
:10AE2000050A9091060AA091070AB091080AE6B5B2
:10AE3000A89B05C0EF3F19F00196A11DB11DFFBFF2
:10AE4000BA2FA92F982F88278E0F911DA11DB11DF4
:10AE5000E2E0880F991FAA1FBB1FEA95D1F7861B56
:10AE6000970B885E9340C8F22150304040405040DC
:10AE700068517C4F211531054105510571F6089542
:10AE8000019739F0880F991F880F991F0297019732
:10AE9000F1F70895789484B5826084BD84B58160AB
:10AEA00084BD85B5826085BD85B5816085BDEEE6D2
:10AEB000F0E0808181608083E1E8F0E010828081B1
:10AEC00082608083808181608083E0E8F0E080811F
:10AED00081608083E1EBF0E0808184608083E0EB3F
:10AEE000F0E0808181608083EAE7F0E08081846027
:10AEF0008083808182608083808181608083808183
:10AF0000806880831092C1000895CF93DF93482F0B
:10AF100050E0CA018B57914FFC0134914B59514F6E
:10AF2000FA018491882369F190E0880F991FFC0150
:10AF3000E95BF14FA591B491FC01EF5AF14FC59136
:10AF4000D491662351F42FB7F8948C91932F909558
:10AF500089238C93888189230BC0623061F42FB7D9
:10AF6000F8948C91932F909589238C938881832BCF
:10AF700088832FBF06C09FB7F8948C91832B8C9346
:10AF80009FBFDF91CF910895482F50E0CA018B55A4
:10AF9000914FFC012491CA018B57914FFC01949170
:10AFA0004B59514FFA013491332309F440C0222305
:10AFB00051F1233071F0243028F42130A1F02230F7
:10AFC00011F514C02630B1F02730C1F02430D9F487
:10AFD00004C0809180008F7703C0809180008F7DB6
:10AFE0008093800010C084B58F7702C084B58F7DB8
:10AFF00084BD09C08091B0008F7703C08091B000FC
:10B000008F7D8093B000E32FF0E0EE0FFF1FEF5A2B
:10B01000F14FA591B4912FB7F894662321F48C9148
:10B020009095892302C08C91892B8C932FBF089512
:10B03000682F70E0CB018B55914FFC012491CB011F
:10B040008B57914FFC0144916B59714FFB019491C7
:10B05000992319F420E030E03CC0222351F1233041
:10B0600071F0243028F42130A1F0223011F514C001
:10B070002630B1F02730C1F02430D9F404C08091DB
:10B0800080008F7703C0809180008F7D8093800047
:10B0900010C084B58F7702C084B58F7D84BD09C090
:10B0A0008091B0008F7703C08091B0008F7D809336
:10B0B000B000892F90E0880F991F855A914FFC01AD
:10B0C000A591B4918C9120E030E0842311F021E02F
:10B0D00030E0C901089508951F920F920FB60F92A4
:10B0E00011242F933F934F938F939F93EF93FF934D
:10B0F0004091C60020914E0A30914F0A2F5F3F4F7A
:10B100002F7330708091500A9091510A2817390797
:10B1100059F0E0914E0AF0914F0AE25FF54F4083FB
:10B1200030934F0A20934E0AFF91EF919F918F9198
:10B130004F913F912F910F900FBE0F901F90189538
:10B1400008951F920F920FB60F9211242F933F93E1
:10B150004F938F939F93EF93FF934091CE00209155
:10B16000D60A3091D70A2F5F3F4F2F7330708091EE
:10B17000D80A9091D90A2817390759F0E091D60AD0
:10B18000F091D70AEA56F54F40833093D70A2093BF
:10B19000D60AFF91EF919F918F914F913F912F91FF
:10B1A0000F900FBE0F901F901895E0912A0BF09111
:10B1B0002B0BE05CFF4F8191919120813181821BAB
:10B1C000930B8F739070892B11F00E946B58E09154
:10B1D000490BF0914A0BE05CFF4F819191912081E6
:10B1E0003181821B930B8F739070892B11F00E9419
:10B1F000A05808951F920F920FB60F9211242F930B
:10B200003F938F939F93EF93FF932091920A3091F6
:10B21000930A8091940A9091950A2817390731F47E
:10B220008091C1008F7D8093C10014C0E091940A89
:10B23000F091950AEE5AF54F20818091940A9091F1
:10B24000950A01968F7390709093950A8093940A53
:10B250002093C600FF91EF919F918F913F912F9185
:10B260000F900FBE0F901F9018951F920F920FB660
:10B270000F9211242F933F938F939F93EF93FF93FC
:10B2800020911A0B30911B0B80911C0B90911D0B80
:10B290002817390731F48091C9008F7D8093C90048
:10B2A00014C0E0911C0BF0911D0BE652F54F20816C
:10B2B00080911C0B90911D0B01968F739070909351
:10B2C0001D0B80931C0B2093CE00FF91EF919F915B
:10B2D0008F913F912F910F900FBE0F901F90189557
:10B2E000DC011C96ED91FC911D97E05CFF4F2191D4
:10B2F000319180819181281B390B2F733070C901E6
:10B300000895DC011C96ED91FC911D97E05CFF4FC8
:10B3100020813181E054F040DF01AE5BBF4F8D9161
:10B320009C9111972817390719F42FEF3FEF07C0A9
:10B330008D919C91E80FF91F8081282F30E0C90181
:10B340000895DC011C96ED91FC911D97E05CFF4F88
:10B3500020813181E054F040DF01AE5BBF4F8D9121
:10B360009C9111972817390719F42FEF3FEF10C060
:10B370008D919C911197E80FF91F20818D919C91DF
:10B38000119701968F73907011969C938E9330E075
:10B39000C9010895FC0186859785DC01A05CBF4F3B
:10B3A000FC01EE5BFF4F2D913C91119780819181C3
:10B3B00028173907C1F70895CF93DF93EC01EE8585
:10B3C000FF85E05CFF4F20813181E054F0402F5F2A
:10B3D0003F4F2F733070DF01AE5BBF4F8D919C915B
:10B3E000119728173907D1F3E05CFF4F80819181D5
:10B3F000E054F040E80FF91F6083EE85FF85E05CC4
:10B40000FF4F31832083EE89FF89208181E090E026
:10B410000D8C02C0880F991F0A94E2F7282B208315
:10B4200081E090E0DF91CF9108951F931092210B5E
:10B430001092200B28EE33E040E050E02093220BE6
:10B440003093230B4093240B5093250B6BE572E054
:10B4500070931F0B60931E0B8EE09AE090932B0B62
:10B4600080932A0B82E59AE090932D0B80932C0B0E
:10B4700085EC90E090932F0B80932E0B84EC90E062
:10B480009093310B8093300B80EC90E09093330BD2
:10B490008093320B81EC90E09093350B8093340BCA
:10B4A00086EC90E09093370B8093360B14E010936A
:10B4B000380BB3E0B093390BA7E0A0933A0BF5E05B
:10B4C000F0933B0BE1E0E0933C0B1092400B1092A9
:10B4D0003F0B2093410B3093420B4093430B50930F
:10B4E000440B70933E0B60933D0B86E99AE090937A
:10B4F0004A0B8093490B8AED9AE090934C0B809312
:10B500004B0B8DEC90E090934E0B80934D0B8CEC9D
:10B5100090E09093500B80934F0B88EC90E09093C9
:10B52000520B8093510B89EC90E09093540B8093D5
:10B53000530B8EEC90E09093560B8093550B109329
:10B54000570BB093580BA093590BF0935A0BE09301
:10B550005B0B1F910895CF93DF930E944A570E947F
:10B560005355C5EDD8E50E9450552097E1F30E9450
:10B57000D558F9CFCF92DF92EF92FF920F931F939E
:10B58000CF93DF937C016B018A01C0E0D0E00FC054
:10B59000D6016D916D01D701ED91FC910190F08183
:10B5A000E02DC7010995C80FD91F015010400115A2
:10B5B000110571F7CE01DF91CF911F910F91FF908F
:10B5C000EF90DF90CF900895DC01ED91FC91019018
:10B5D000F081E02D09950895CF93DF93DB010D9065
:10B5E0000020E9F71197A61BB70BEC01E881F98160
:10B5F0000280F381E02DAD010995DF91CF9108958F
:10B600004F925F927F928F929F92AF92BF92CF9212
:10B61000DF92EF92FF920F931F93DF93CF93CDB7FB
:10B62000DEB7A1970FB6F894DEBF0FBECDBF2C01D9
:10B63000742ECB01223008F42AE019A231E2C32E85
:10B64000D12CCC0EDD1E822E9924AA24BB24672D7A
:10B65000752FA50194010E942F7579018A01C801F7
:10B66000B701A50194010E94DD74472D461B089483
:10B67000C108D1084A3014F4405D01C0495CF601AC
:10B680004083E114F1040105110521F07E2C5F2DAA
:10B69000C801DDCFC201B6010E94EC5AA1960FB6D7
:10B6A000F894DEBF0FBECDBFCF91DF911F910F91F8
:10B6B000FF90EF90DF90CF90BF90AF909F908F90D2
:10B6C0007F905F904F900895DC012115310541F482
:10B6D000ED91FC910190F081E02D642F0995089582
:10B6E0000E94005B0895EF92FF920F931F939A01BF
:10B6F0007B0100E010E0B801A7010E94645B1F918C
:10B700000F91FF90EF900895CF92DF92EF92FF920A
:10B710000F931F93CF93DF93EC016A017B012115F7
:10B72000310541F4E881F9810190F081E02D642F29
:10B7300009951FC02A303105D1F477FF17C0E88181
:10B74000F9810190F081E02D6DE209958C0144278B
:10B750005527BA014C195D096E097F09CE012AE00F
:10B760000E94005B9801280F391F04C02AE00E9444
:10B77000005B9C01C901DF91CF911F910F91FF9058
:10B78000EF90DF90CF900895EF92FF920F931F9369
:10B790007B019A010027F7FC0095102FB801A70143
:10B7A0000E94845B1F910F91FF90EF9008950E947B
:10B7B000EC5A089581E08093A10B60937E0B109268
:10B7C0009F0B1092A00B089520917D0B30E080918B
:10B7D0007C0B281B3109C901089540917C0B809195
:10B7E0007D0B481718F02FEF3FEF0AC0E42FF0E071
:10B7F000E45AF44F8081282F30E04F5F40937C0B58
:10B80000C9010895E0917C0B80917D0BE81718F039
:10B81000EFEFFFEF06C0F0E0E45AF44F8081E82F2D
:10B82000F0E0CF01089508951092A50B1092A40B9B
:10B8300088EE93E0A0E0B0E08093A60B9093A70B76
:10B84000A093A80BB093A90B8BE692E09093A30B67
:10B850008093A20B0895CF92DF92EF92FF920F9305
:10B860001F93CF93DF937C016B018A018091A10B21
:10B870008823A1F0C0E0D0E00DC0D701ED91FC918C
:10B88000D601AC0FBD1F0190F081E02DC7016C9176
:10B8900009952196C017D10780F304C0CB01642F0E
:10B8A0000E941373C801DF91CF911F910F91FF90F8
:10B8B000EF90DF90CF900895DF93CF930F92CDB7A5
:10B8C000DEB7FC0169838091A10B8823C9F08091C8
:10B8D000A00B803238F081E090E09383828320E0F7
:10B8E00030E015C080919F0BE82FF0E0E158F44F55
:10B8F000998190838F5F80939F0B8093A00B05C0ED
:10B90000CE01019661E00E94137321E030E0C9018D
:10B910000F90CF91DF9108950F93062F80917E0BAA
:10B920006FE77BE04091A00B21E00E94BE72109275
:10B930009F0B1092A00B1092A10B0F91089561E044
:10B940000E948C5C0895413208F040E2862F6CE53D
:10B950007BE00E94757210927C0B80937D0B0895A2
:10B9600021E00E94A35C089510927C0B10927D0B45
:10B9700010929F0B1092A00B0E94BF7408950F931A
:10B980001F93CF93DF93DC01EB018A0180E090E00D
:10B9900020E2FE01E80FF91F208301968B3091050C
:10B9A000C1F757E040E024C0622F2E3219F085EC39
:10B9B0009EE007C05A3051F15AE048E018C03217F3
:10B9C00029F1FC01019634913323C9F75417F0F0A3
:10B9D0002132E0F02F37D0F4822F81568A3110F4D3
:10B9E000622F6052FE01E40FF11D60834F5F1196DC
:10B9F0002C91222311F02F32B9F6F801B183A083E4
:10BA000090E08881803219F091E001C090E0892FA8
:10BA1000DF91CF911F910F910895CF92DF92EF9216
:10BA2000FF920F931F93DF93CF9300D000D0CDB739
:10BA3000DEB77C01FC0186899789A08DB18D898351
:10BA40009A83AB83BC8300E010E06E010894C11CB4
:10BA5000D11C49815A816B817C81D70114968D91CB
:10BA60009C91159796010E94FA6C882379F1D70171
:10BA70001496ED91FC9115978481080F111DB0E18A
:10BA800000301B0718F529813A814B815C8183893D
:10BA9000803131F4285F3F4F40405040D0F205C024
:10BAA000285F3F4F4F4F5F40A0F2C801A0E0B0E0D9
:10BAB00029E0880F991FAA1FBB1F2A95D1F7F7010C
:10BAC000828B938BA48BB58B81E001C080E00F90BB
:10BAD0000F900F900F90CF91DF911F910F91FF90DA
:10BAE000EF90DF90CF900895CF93DF93EC01FB01AF
:10BAF0008A818823D1F57D836C8383898031C9F560
:10BB000082E08A831E8A1F8A188E198E84899589FD
:10BB1000A0E0B0E035E0880F991FAA1FBB1F3A953F
:10BB2000D1F78A8B9B8BAC8BBD8B0FC083E08A8354
:10BB300086899789A08DB18D8E8B9F8BA88FB98FA9
:10BB4000CE010E940D5D882381F081E089831E82F1
:10BB50001F82188619861A861B861C861D861E86DD
:10BB60001F86188A198A1B8201C080E0DF91CF915D
:10BB700008958032D1F7DACF6F927F928F929F92A1
:10BB8000AF92BF92CF92DF92EF92FF920F931F93EB
:10BB9000CF93DF93EC017A018B012A81222309F4F0
:10BBA00080C08A899B89AC89BD8984179507A607BF
:10BBB000B70708F476C085C0E114F104010511054A
:10BBC00051F41E821F82188619861A861B861C86CF
:10BBD0001D8681E067C02A853B854C855D85EC81AB
:10BBE000FD81828590E009962150304040405040D0
:10BBF00039014A01082E04C096948794779467947B
:10BC00000A94D2F72F5F3F4F4F4F5F4F0894E108E0
:10BC1000F108010911095701680104C0D694C794BD
:10BC2000B794A7948A95D2F70894E11CF11C011DE2
:10BC3000111DA614B704C804D90428F02115310534
:10BC40004105510549F48E899F89A88DB98D8E8350
:10BC50009F83A887B98716C0A618B708C808D9084F
:10BC600011C04E815F81688579858C819D819401A9
:10BC70000E94FA6C0894A108B108C108D108882371
:10BC800031F40FC046E0842E912C8C0E9D1EA11421
:10BC9000B104C104D10429F7EA86FB860C871D870D
:10BCA00098CF80E0DF91CF911F910F91FF90EF909F
:10BCB000DF90CF90BF90AF909F908F907F906F90CC
:10BCC0000895223009F078CFE7CFCF93DF93EC01CE
:10BCD000462F6E857F85888999890E940D6BAC01FE
:10BCE000009719F420E030E00AC08B81282F30E063
:10BCF00065E0220F331F6A95E1F7240F351FC90154
:10BD0000DF91CF9108950F931F93CF93DF938C0111
:10BD1000FC0182818823F1F1818187FF38C0C8014D
:10BD200061E00E94655EEC010097A1F18881853E8B
:10BD300089F1F8018281823040F482899389A48953
:10BD4000B5898C8F9D8FAE8FBF8FF80186899789BB
:10BD50009B8F8A8F86899789A08DB18DCD01AA2767
:10BD6000BB279D8B8C8BE091B00BF091B10B309782
:10BD700051F0BE016A5E7F4FCE0148960995888DCD
:10BD8000998D9B8B8A8BF80181818F7781830E94AB
:10BD9000C56A04C081E0F801808380E0DF91CF9123
:10BDA0001F910F9108956F927F928F929F92AF9201
:10BDB000BF92CF92DF92EF92FF920F931F93DF9388
:10BDC000CF9300D000D0CDB7DEB77C015A016B0114
:10BDD000DC0112968C911297813009F091C0119676
:10BDE0008C9181FF8DC0A0C00097A105B10511F411
:10BDF00081E087C0F7016284738484849584C701DD
:10BE0000B601A5010E94BC5D882309F479C0D70161
:10BE100014968D919C911597A114B104C104D1047D
:10BE200089F456964D915D916D917C9159970E9440
:10BE3000696D882309F464C0F701168A178A108E89
:10BE4000118E44C0D70116964D915D916D917C91F4
:10BE500019979E012F5F3F4F0E94FA6C882309F4C7
:10BE60004FC0D7011496ED91FC91159749815A81E5
:10BE70006B817C818389803149F4483FBFEF5B0748
:10BE8000B0E06B07B0E07B0748F020C0483F8FEF81
:10BE900058078FEF68078FE07807C0F4CF010E9442
:10BEA000696D882369F1D70116964D915D916D9169
:10BEB0007C91199714968D919C9115970FEF1FEF18
:10BEC0002FEF3FE00E948A6C8823D1F0F701A28A0D
:10BED000B38AC48AD58A818180688183C7010E9420
:10BEE000835E882369F0B601A5016A147B048C0483
:10BEF0009D0410F4B401A301C7010E94BC5D01C000
:10BF000080E00F900F900F900F90CF91DF911F91D5
:10BF10000F91FF90EF90DF90CF90BF90AF909F90E8
:10BF20008F907F906F900895F70182899389A489FB
:10BF3000B58984179507A607B70708F055CFE0CF56
:10BF40001F93CF93DF93EC01142F262F30E0F901DC
:10BF500085E0EE0FFF1F8A95E1F7E954F44F8385E2
:10BF6000817121F0842F827109F064C08091B70D36
:10BF70009091B80DA091B90DB091BA0D8E879F87A1
:10BF8000A88BB98B6B83F901B5E0EE0FFF1FBA9553
:10BF9000E1F7E954F44F2489358940E050E0A901E4
:10BFA000332722272E8B3F8B488F598F828D938D7D
:10BFB000A0E0B0E0282B392B4A2B5B2B2E8B3F8B3C
:10BFC000488F598F838590E088719070009751F465
:10BFD000848D958DA68DB78D8A8B9B8BAC8BBD8BFD
:10BFE00081E008C0409731F5CE010E940D5D8823A5
:10BFF00009F184E08A83812F8F7089831E821F82DA
:10C00000188619861A861B861C861D8614FF18C082
:10C01000CE0140E050E060E070E00E94D35E8823F3
:10C0200079F408C04A895B896C897D89CE010E94B8
:10C03000BC5D02C01A8280E0DF91CF911F9108950C
:10C0400015FDF0CF81E0F8CF0F931F938C010E9474
:10C05000835EF80112821F910F910895CF93DF93B1
:10C06000EC0140E050E060E070E00E94D35E882385
:10C0700069F0CE0161E00E94655EFC01009731F03D
:10C0800085EE80831A820E94C56A01C080E0DF913C
:10C09000CF9108953F924F925F926F927F928F92CD
:10C0A0009F92AF92BF92CF92DF92EF92FF920F9347
:10C0B0001F93DF93CF93CDB7DEB728970FB6F894D1
:10C0C000DEBF0FBECDBF98878F835E834D83DC01BB
:10C0D00012968C911297882309F41DC111968C91A8
:10C0E00080FF19C133C1F501EE19FF09FE83ED830D
:10C0F0007A8369838F81988506969C838B836D8074
:10C100007E8002C1AF81B8851A962D913D914D91E7
:10C110005C911D978FEF482E81E0582E42225322CA
:10C120001496ED91FC91159759016A0109E0D69496
:10C13000C794B794A7940A95D1F735803A20129600
:10C140008C91823049F4E688F788008D118DEA0CD5
:10C15000FB1C0C1D1D1D35C04114510411F533206D
:10C1600001F5211531054105510559F4EF81F88597
:10C1700086899789A08DB18D86839783A087B187A3
:10C1800010C0AF81B88516964D915D916D917C91EF
:10C190001997CF012B813C810E94FA6C882309F406
:10C1A000BAC0EF81F88546815781608571858481A9
:10C1B00095810E94AB6A7B018C01E30CF11C011D8F
:10C1C000111D4114510499F4F0E06F16F2E07F065E
:10C1D00070F02091B70D3091B80D4091B90D50918C
:10C1E000BA0DE216F3060407150709F0CFC0C8011F
:10C1F000B70140E00E940D6B009709F48CC040E04D
:10C2000052E04419550943014615570508F44A01FF
:10C210009C01240D351D89819A81B901A4010E94D8
:10C220000B0859C08091BC0D9091BD0DB801A701BC
:10C2300029813A810E944E71882309F46CC0812CB7
:10C2400012E0912E48C0D72CD694AF81B8851296B3
:10C250008C911297823049F01496ED91FC911597CC
:10C26000848183198D1508F4D82EE216F30604078D
:10C27000150770F02D0D311D411D511DE216F306FD
:10C280000407150728F40E94C56A882309F443C0EF
:10C290008091BC0D9091BD0DB801A7010E94B270B4
:10C2A0008823C9F109811A81FF2408C0B8010E94BE
:10C2B0003B7100501E4F882371F1F3948091BC0DA7
:10C2C0009091BD0DFD1490F30E949870882319F190
:10C2D0009D2C990C8824E981FA81E80DF91DFA83D7
:10C2E000E983940140E050E0EF81F88582859385F1
:10C2F000A485B585820F931FA41FB51F82879387DE
:10C30000A487B587681879086114710409F0FACE1A
:10C310004D815E8102C04FEF5FEFCA0128960FB6D4
:10C32000F894DEBF0FBECDBFCF91DF911F910F916B
:10C33000FF90EF90DF90CF90BF90AF909F908F9045
:10C340007F906F905F904F903F900895AF81B88538
:10C350005296AD90BD90CD90DC9055971A96ED9089
:10C36000FD900D911C911D97ED81FE819F0140E094
:10C3700050E0D601C5018E199F09A00BB10B2817FB
:10C3800039074A075B0708F0AECEB2CEF0E06F1671
:10C39000F4E07F0608F057CF45CFDF93CF930F929D
:10C3A000CDB7DEB7BE016F5F7F4F41E050E00E9426
:10C3B0004A60019719F02FEF3FEF03C08981282FC2
:10C3C00030E0C9010F90CF91DF910895EF92FF9275
:10C3D0000F931F93CF93DF93EC018A81823038F162
:10C3E000EA84FB840C851D85CE010E94CD6197FDFA
:10C3F0001EC08A859B85AC85BD854F96A11DB11D4C
:10C400008A879B87AC87BD8725E016950795F794AB
:10C41000E7942A95D1F72E2D30E02F70307095E0FB
:10C42000220F331F9A95E1F72954344F02C020E0C0
:10C4300030E0C901DF91CF911F910F91FF90EF90F4
:10C440000895CF93DF93EC018A81843071F5CE019A
:10C4500040E050E060E070E00E94BC5D10C0CE01A2
:10C460000E94E661FC01009701F180818823A1F020
:10C47000853E29F08E3219F0838583FF16C02A8508
:10C480003B854C855D858A899B89AC89BD89281748
:10C4900039074A075B0718F381E08A838981826044
:10C4A0008983CE010E942E6001C080E0DF91CF9190
:10C4B0000895DF92EF92FF920F931F93CF93DF9334
:10C4C0008C01EB017A01D22E8C819D81F80195833C
:10C4D00084838281882329F56115710559F521C06E
:10C4E000A70165E0440F551F6A95E1F760E070E031
:10C4F000CE010E94BC5D8823A1F0CE010E94E661BE
:10C50000FC01009771F08081882359F0853E49F045
:10C510008E3239F06E2D6F70C8014D2D0E94A05FD4
:10C5200001C080E0DF91CF911F910F91FF90EF90BC
:10C53000DF90089527FFD4CFF4CFAF92BF92CF9270
:10C54000DF92EF92FF920F931F93DF93CF93CDB7BC
:10C55000DEB76A970FB6F894DEBF0FBECDBF8C0171
:10C5600019821B8240E050E060E070E00E94BC5DF8
:10C570005E010894A11CB11C52C0C8010E94E66172
:10C58000FC01009709F466C08081882309F456C035
:10C59000853E09F444C08E3209F441C0838583FD91
:10C5A0003EC0A7019601F5E056954795379527952A
:10C5B000FA95D1F77901C501B801A90121E00E94DE
:10C5C0005962882309F446C08B81843021F4C50167
:10C5D0000E949D6206C08A8182608A83C5010E9492
:10C5E0002E608823B9F10894E11CF11CA70160E0DA
:10C5F00070E0E5E0440F551F661F771FEA95D1F7FD
:10C60000F80182859385A485B58584179507A607CB
:10C61000B70729F0C8010E94BC5D8823D9F0F80152
:10C62000C284D384E484F58482899389A489B589FA
:10C63000C816D906EA06FB0608F49FCFF8018281E6
:10C640008250823028F0C8010E942162882319F0AC
:10C6500081E001C080E06A960FB6F894DEBF0FBE9D
:10C66000CDBFCF91DF911F910F91FF90EF90DF90A1
:10C67000CF90BF90AF9008952F923F924F925F92CC
:10C680006F927F928F929F92AF92BF92CF92DF92E2
:10C69000EF92FF920F931F93DF93CF930F92CDB73B
:10C6A000DEB72C015B013A01490100E010E0EE2405
:10C6B000EA94FE2C1E010894211C311C13C00A0DA3
:10C6C0001B1DF80160838114910419F46A3049F448
:10C6D0001EC0772767FD7095C4010E942608009749
:10C6E000B1F4860168010894C11CD11CC614D7049A
:10C6F00044F5C201B10141E050E00E944A607C0172
:10C7000081309105F1F469816D30C9F6EBCF860176
:10C71000A00EB11EF5011082C8010F90CF91DF91DC
:10C720001F910F91FF90EF90DF90CF90BF90AF904F
:10C730009F908F907F906F905F904F903F902F9041
:10C740000895F7FEE5CF0FEF1FEFE6CFCF93DF930E
:10C75000EC019C012A5F3F4F8C819D8141E050E0BC
:10C7600060E070E00E94D06D8823A1F08E899F89DF
:10C77000A88DB98D0097A105B10559F48E819F81CF
:10C78000A885B9858E8B9F8BA88FB98F898180688A
:10C79000898381E0DF91CF9108952F923F924F924C
:10C7A0005F926F927F928F929F92AF92BF92CF9241
:10C7B000DF92EF92FF920F931F93DF93CF93CDB74A
:10C7C000DEB729970FB6F894DEBF0FBECDBF4C0180
:10C7D000162F072F59874887DC0112968C911297E4
:10C7E000813009F0BDC111968C9181FFB9C1D7C1CB
:10C7F000F401428953896489758982859385A4856A
:10C80000B58584179507A607B70731F0C4010E94C4
:10C81000BC5D882309F4A4C1888599859C0140E00A
:10C8200050E0F40182859385A485B5858095909527
:10C83000A095B09582179307A407B50708F490C197
:10C84000812F902F9C013F832E83288439844CC1F3
:10C85000D4011496ED91FC911597DA01C90119E004
:10C86000B695A795979587951A95D1F715811823B1
:10C87000AFEFEA2EA1E0FA2EE222F322112309F013
:10C8800052C0E114F10409F04EC0D40116964D9146
:10C890005D916D917C911997411551056105710567
:10C8A00071F1CF019E012F5F3F4F0E94FA6C8823E8
:10C8B00009F456C129813A814B815C81D4011496D7
:10C8C000ED91FC9115978389803149F4283FBFEFA2
:10C8D0003B07B0E04B07B0E05B0748F019C0283FCA
:10C8E000EFEF3E07EFEF4E07EFE05E0788F4D4016D
:10C8F00016962D933D934D935C93199714C0F401B4
:10C9000086899789A08DB18D0097A105B10531F475
:10C91000C4010E94A663882331F422C1F4018683F6
:10C920009783A087B187D40116964D915D916D9143
:10C930007C91199714968D919C9115970E94AB6AE2
:10C940005B016C01A10EB11CC11CD11CE114F104EE
:10C95000A9F4B0E02B16B2E03B06A0F5F401228565
:10C9600033854485558582899389A489B58928179B
:10C9700039074A075B0710F045E001C041E0C601F6
:10C98000B5010E940D6B009709F4EAC000E012E0C7
:10C990000E191F0921010215130508F428019C0135
:10C9A0002E0D3F1DC9016E817F81A2010E940B08DF
:10C9B0004016510609F080C00E940A6B882309F0D6
:10C9C0007BC0CEC0F0E02F16F4E03F0600F580916A
:10C9D000B70D9091B80DA091B90DB091BA0D8A150F
:10C9E0009B05AC05BD0511F40E949C6A8091BC0DAD
:10C9F0009091BD0DB601A5012E813F810E945E7010
:10CA0000882309F4ADC0412CF2E05F2E55C0D4015B
:10CA10001496ED91FC9115978481811BB32DB695E9
:10CA2000BD838B1708F48D83ED810E2F10E020E07D
:10CA300030E08091BC0D9091BD0DB601A5010E9422
:10CA4000B16F882309F48CC06E807F8086017501E8
:10CA500022C08091B70D9091B80DA091B90DB09101
:10CA6000BA0DE816F9060A071B0711F40E949C6A22
:10CA70008091BC0D9091BD0DB3010E94387020E0F3
:10CA800032E0620E731E0894E11CF11C011D111DA1
:10CA9000882309F465C08E2D8A193D818317C8F259
:10CAA0008091BC0D9091BD0D0E948B6F882309F47D
:10CAB00057C05D80550C4424920140E050E0F401E1
:10CAC00082859385A485B585820F931FA41FB51F0A
:10CAD00082879387A487B5872E813F81240D351DDA
:10CAE0003F832E8324183508D4011A962D913D9149
:10CAF0004D915C911D972114310409F0A9CE5296F5
:10CB00008D919D910D90BC91A02D82179307A40744
:10CB1000B50748F4F401228B338B448B558B81810C
:10CB20008068818311C08091B00B9091B10B892BEB
:10CB300059F028853985232B39F0D40111968C9131
:10CB40001197806811968C93F401818183FF05C051
:10CB5000C4010E94835E882319F04885598505C069
:10CB600081E0D4018C934FEF5FEFCA0129960FB695
:10CB7000F894DEBF0FBECDBFCF91DF911F910F9113
:10CB8000FF90EF90DF90CF90BF90AF909F908F90ED
:10CB90007F906F905F904F903F902F90089582FD0F
:10CBA00027CE3ACE9F92AF92BF92CF92DF92EF9272
:10CBB000FF920F931F93CF93DF938C01FC01828927
:10CBC0009389A489B589805E9F4FAF41B04008F03A
:10CBD0005CC0C8010E94A663882309F456C0D8012E
:10CBE00016964D915D916D917C91199714968D914A
:10CBF0009C9115970E94AB6A5B016C0145E00E9415
:10CC00000D6BEC01009709F442C080E092E0FE0158
:10CC10009C01119221503040E1F79C2EED2EFF2413
:10CC2000F39411C0B601A5014F0D511D611D711D79
:10CC30008091BC0D9091BD0D292D3E2D0E945E70FE
:10CC4000882319F1F394D8011496ED91FC9115976E
:10CC50002481F21638F330E040E050E089E0220F02
:10CC6000331F441F551F8A95D1F752968D919D9180
:10CC70000D90BC91A02D820F931FA41FB51FF8012A
:10CC8000828B938BA48BB58B02C0C0E0D0E0CE0129
:10CC9000DF91CF911F910F91FF90EF90DF90CF9098
:10CCA000BF90AF909F9008953F924F925F926F9286
:10CCB0007F928F929F92AF92BF92CF92DF92EF922C
:10CCC000FF920F931F93CF93DF934C01EB01442E00
:10CCD000352E522E8C819D81F40195838483CB0166
:10CCE00040E050E060E070E00E94BC5D77244FC0FF
:10CCF000CE010E94CD6197FDABC08A859B85AC8536
:10CD0000BD8581509E4FAF4FBF4F8A879B87AC87B1
:10CD1000BD87A090B70DB090B80DC090B90DD09060
:10CD2000BA0D27EBE22E2BE0F22E00E010E0602E91
:10CD3000F7018081882311F0853E79F4772041F452
:10CD4000F401A686B786C08AD18A63827724739459
:10CD5000F7018081882391F428C0B80195E0660F1F
:10CD6000771F9A95E1F76954744F842D932D4BE00A
:10CD700050E00E94FE07009709F47DC00F5F1F4F2F
:10CD800080E290E0E80EF91E0031110581F62A8557
:10CD90003B854C855D858A899B89AC89BD8928172F
:10CDA00039074A075B0708F4A3CF56FE51C051FE6E
:10CDB0004FC0772051F0F4016380C40161E00E940C
:10CDC000655EEC01009761F443C08A81823009F40A
:10CDD0003FC0CE010E94D2650097D1F1EC016624DC
:10CDE00080E2FE0111928A95E9F7DE01242D332DB0
:10CDF000C901FC018BE001900D928150E1F7E091B7
:10CE0000B00BF091B10B309739F0BE01625F7F4FEC
:10CE1000CE014096099508C081E298E2998B888BF3
:10CE200080E098E09F878E87888999899B8B8A8B81
:10CE3000998F888F8E859F859F8B8E8B0E94C56A68
:10CE4000882331F0C401662D452D0E94A05F01C0EA
:10CE500080E0DF91CF911F910F91FF90EF90DF90D5
:10CE6000CF90BF90AF909F908F907F906F905F908A
:10CE70004F903F90089557FEE5CFEACF2F923F9213
:10CE80004F925F926F927F928F929F92AF92BF92DA
:10CE9000CF92DF92EF92FF920F931F93DF93CF9386
:10CEA000CDB7DEB7C454D0400FB6F894DEBF0FBE86
:10CEB000CDBF4C016B01DE01A05CBF4F11965C93AE
:10CEC0004E9323962FAF23976115710509F48AC0FD
:10CED0001E8618A6FC018281882309F083C01C8667
:10CEE0001EA2FA0180818F32F1F086015CE0E52E0E
:10CEF000F12CEC0EFD1E40E4A42EB12CAC0EBD1E98
:10CF00003E010894611C711C2596FFAEEEAE25977C
:10CF100036E2232E312C2C0E3D1E27012BC01196FC
:10CF2000B183A08301C0FD01A081B1818C918F32BA
:10CF3000B1F3882349F4D60114966D917C9115972D
:10CF4000C4010E94745D4FC0F6018281825082301C
:10CF500060F28E010A5D1F4F64817581C8010E94D5
:10CF6000745D882319F63EC0342D252D8701832F4B
:10CF7000922F7C01D5018D919C91B301A5010E9456
:10CF8000BF5C882329F42EC03196D501ED93FC9324
:10CF9000D501ED91FC9180818F32B1F38823C9F0E6
:10CFA000C701B801A30121E00E9454668823D1F093
:10CFB0000C151D0519F0C8010E9424602596EEADE0
:10CFC000FFAD2597EE16FF0679F6C101322D292F08
:10CFD000CDCFC401B801A30123962FAD23970E94A2
:10CFE000546601C080E0CC5BDF4F0FB6F894DEBF23
:10CFF0000FBECDBFCF91DF911F910F91FF90EF90AA
:10D00000DF90CF90BF90AF909F908F907F906F9068
:10D010005F904F903F902F9008950F931F93DF9351
:10D02000CF93CDB7DEB76A970FB6F894DEBF0FBEC9
:10D03000CDBF9C01AB0119821B828E010F5F1F4F78
:10D04000C801B90122E00E943E67882319F0C80197
:10D050000E942E606A960FB6F894DEBF0FBECDBF59
:10D06000CF91DF911F910F910895FB01242F6091C3
:10D07000AE0B7091AF0BAF010E943E670895DF9336
:10D08000CF93CDB7DEB76A970FB6F894DEBF0FBE69
:10D09000CDBF9C01AB0119821B82CE010196B90163
:10D0A00021E00E943E676A960FB6F894DEBF0FBE7D
:10D0B000CDBFCF91DF910895EF92FF920F931F9311
:10D0C000DF93CF93CDB7DEB7A0970FB6F894DEBF4E
:10D0D0000FBECDBF8C017B01FB018281823008F441
:10D0E0006FC0C80123EC0E945466882309F468C00D
:10D0F00081E0F801818384E08283C8010E94D265C7
:10D10000892B09F45DC0C8010E94835E882309F45D
:10D1100057C0C80161E00E94655EFC01009709F4F8
:10D120004FC080E18387DE01119680E201900D926D
:10D130008150E1F78EE28983FE01329620E2CE0132
:10D140000C962193E817F907E1F7F801468957890A
:10D15000608D718D848195810E94AB6A41E00E944F
:10D160000D6B9C01009761F1DC01FE01319680E2BC
:10D1700001900D928150E1F78EE28A83F70182815E
:10D180008250823028F41C8E1B8E1E8A1D8A0CC091
:10D19000F70186899789A08DB18D9C8F8B8FCD01EA
:10D1A000AA27BB279E8B8D8BD9019096FE013196C5
:10D1B00080E201900D928150E1F70E94C56A01C0A2
:10D1C00080E0A0960FB6F894DEBF0FBECDBFCF9122
:10D1D000DF911F910F91FF90EF9008952F923F9252
:10D1E0004F925F926F927F928F929F92AF92BF9277
:10D1F000CF92DF92EF92FF920F931F93DF93CF9323
:10D20000CDB7DEB7C454D0400FB6F894DEBF0FBE22
:10D21000CDBF3C016B01DE01A05CBF4F11965C935A
:10D220004E9323962FAF23976115710509F487C09C
:10D230001E8618A6FC018281882309F080C09AC04E
:10D240008601FCE0EF2EF12CEC0EFD1EE0E4AE2E8C
:10D25000B12CAC0EBD1E4E010894811C911C25966C
:10D26000FFAEEEAE259776E2272E312C2C0E3D1E1A
:10D27000270124C01196B183A08301C0FD01A081C4
:10D28000B1818C918F32B1F3D60112968C911297A5
:10D2900082508230A8F28E010A5D1F4F14966D9164
:10D2A0007C911597C8010E94745D882351F647C090
:10D2B000342D252D8701832F922F7C01F50180814C
:10D2C0009181B401A5010E94BF5C882329F437C075
:10D2D0003196D501ED93FC93D501ED91FC918081C0
:10D2E0008F32B1F3882329F1C701B801A40121E0ED
:10D2F0000E945466882361F42396BFAD2397BB2315
:10D30000F1F0C701B801A4010E945C688823B9F05C
:10D310000C151D0519F0C8010E9424602596EEAD7C
:10D32000FFAD2597EE16FF0619F6C101322D292F04
:10D33000C1CFC301B801A4010E945C6801C080E0B4
:10D34000CC5BDF4F0FB6F894DEBF0FBECDBFCF91E1
:10D35000DF911F910F91FF90EF90DF90CF90BF90E2
:10D36000AF909F908F907F906F905F904F903F9085
:10D370002F9008951C861EA2ED91FC91119780813B
:10D380008F3209F05DCF7ACF4F960E940D680895D5
:10D39000DF93CF93CDB7DEB76A970FB6F894DEBFB1
:10D3A0000FBECDBFFB01242F19821B82BC01615E21
:10D3B0007F4FCE010196AF010E94EE686A960FB6CC
:10D3C000F894DEBF0FBECDBFCF91DF9108954F9689
:10D3D0000E943F680895DF92EF92FF920F931F9390
:10D3E000DF93CF93CDB7DEB76A970FB6F894DEBF61
:10D3F0000FBECDBF9B01D42E19821B828C01015E12
:10D400001F4F7E010894E11CF11CC701B801A9015E
:10D4100021E00E943E678B81823010F480E00EC0D4
:10D42000D801F7018AE101900D928150E1F7DD20EA
:10D4300021F01093AF0B0093AE0B81E06A960FB60C
:10D44000F894DEBF0FBECDBFCF91DF911F910F913A
:10D45000FF90EF90DF900895CF93DF93EC01662368
:10D4600031F06F96D093AF0BC093AE0B6F9789A13D
:10D47000882321F0CE014F960E942460CE014F9662
:10D480002596BE010E94745DDF91CF9108950F93A0
:10D490001F93CF93DF93EC010E9482718823C9F020
:10D4A0008E010B5F1F4FC801BE0141E00E94516B0E
:10D4B000882339F4C801BE0140E00E94516B8823E3
:10D4C00041F0CE0161E00E942C6A882319F081E0CE
:10D4D00001C080E0DF91CF911F910F9108950496D4
:10D4E0000E94CD630895DF93CF930F92CDB7DEB73F
:10D4F00069830496BE016F5F7F4F41E050E00E9458
:10D50000CD6320E030E0019711F421E030E0C90163
:10D510000F90CF91DF91089504960E94CD630895F6
:10D52000DB010D900020E9F71197A61BB70B0496BD
:10D53000AD010E94CD6308958FEF9FEFAFEFBFEF76
:10D540008093B70D9093B80DA093B90DB093BA0D19
:10D550001092BB0D0895FC019A01AB01225030409E
:10D5600040405040028404C0220F331F441F551F07
:10D570000A94D2F783859485A585B685280F391F2F
:10D580004A1F5B1FB901CA0108958091BB0D80FF3E
:10D590003DC04091B70D5091B80D6091B90D70919B
:10D5A000BA0D8091BC0D9091BD0D27EB3BE00E9420
:10D5B0005E70882369F18091BB0D81FF22C080914C
:10D5C000B20B8230F0F04091B30B5091B40B6091EC
:10D5D000B50B7091B60B8091B70D9091B80DA091DD
:10D5E000B90DB091BA0D480F591F6A1F7B1F80916A
:10D5F000BC0D9091BD0D27EB3BE00E945E7088232F
:10D6000039F08091BB0D8E7F8093BB0D81E0089532
:10D6100080E008950E94C56A0895DF92EF92FF921C
:10D620000F931F937B018C01D42E8091B70D9091A5
:10D63000B80DA091B90DB091BA0D8E159F05A00738
:10D64000B107E1F00E94C56A882311F1D2FC0CC039
:10D650008091BC0D9091BD0DB801A70127EB3BE077
:10D660000E944E718823A1F01092BB0DE092B70D7D
:10D67000F092B80D0093B90D1093BA0D83E0D82243
:10D680008091BB0D8D298093BB0D27EB3BE002C041
:10D6900020E030E0C9011F910F91FF90EF90DF90E3
:10D6A00008956F927F928F929F92AF92BF92CF9286
:10D6B000DF92EF92FF920F931F93CF93DF93EC01D2
:10D6C000142F7093BD0D6093BC0D1B8A82E090E017
:10D6D000A0E0B0E088839983AA83BB831092BB0D3E
:10D6E0008FEF9FEFAFEFBFEF8093B70D9093B80D23
:10D6F000A093B90DB093BA0D442321F46624772486
:10D70000430136C0453008F0F1C060E070E080E0D1
:10D7100090E040E00E940D6BDC01009709F4E6C048
:10D72000412F50E041505040FA0174E0EE0FFF1FCE
:10D730007A95E1F7E80FF91FE254FE4F808190E0FF
:10D740008F779070892B09F0D1C064E0440F551F8A
:10D750006A95E1F7A40FB51FAA53BE4F6D907D9057
:10D760008D909C90611471048104910409F4BEC0F1
:10D77000C401B30140E00E940D6B5C01009709F405
:10D78000B5C0FC01838594858050924009F0AEC0FD
:10D79000F5012089222309F4A9C046855785411542
:10D7A000510509F4A3C02093B20B85858C83815069
:10D7B0008D831A8691E060E070E00AC0990F6F5F78
:10D7C0007F4F6830710509F491C08A858F5F8A8721
:10D7D0008C81891799F7F50166897789611571053B
:10D7E00019F080E090E005C0F50164A175A186A163
:10D7F00097A16093B30B7093B40B8093B50B909388
:10D80000B60B6A01EE24FF24C60CD71CE81CF91CD9
:10D81000CF86D88AE98AFA8AF501018912891D8B97
:10D820000C8B30E040E050E00E94DD746C0D7D1DFB
:10D830008E1D9F1D6E8B7F8B888F998F35E0000F1B
:10D84000111F3A95E1F701501E4F012F1127069540
:10D85000980140E050E0260F371F481F591F2B87C3
:10D860003C874D875E87F50183899489009721F075
:10D870007C0100E010E005C0F501E0A0F1A002A1EC
:10D8800013A1C401B301621B730B840B950B6E0DC6
:10D890007F1D801F911F0A8404C0969587957795F8
:10D8A00067950A94D2F76E837F8388879987653F4F
:10D8B000FFE07F07F0E08F07F0E09F0718F48CE0AF
:10D8C0008B8B14C0655F7F4F8040904010F480E1E7
:10D8D0000AC0F50184A595A5A6A5B7A58E8B9F8B3B
:10D8E000A88FB98F80E28B8B81E001C080E0DF914F
:10D8F000CF911F910F91FF90EF90DF90CF90BF904D
:10D90000AF909F908F907F906F90089542600E949B
:10D910000D6B08958F929F92AF92BF92CF92DF923C
:10D92000EF92FF920F931F93CF93DF93EC016A0165
:10D930007B0148015901423051056105710508F428
:10D940004BC08E819F81A885B9850196A11DB11D0F
:10D9500084179507A607B70708F43EC08B89803166
:10D9600029F4252F362F472F55270BC08032A1F5DC
:10D970009A01AB0117E056954795379527951A956B
:10D98000D1F78F859889A989BA89280F391F4A1F2D
:10D990005B1FCA01B90141E00E94866C9C0100979F
:10D9A000D9F08B89803149F4F601F070EE0FFF1F3A
:10D9B000E20FF31F918280820DC0F601EF77F070C5
:10D9C000EE0FFF1FEE0FFF1FE20FF31F8082918209
:10D9D000A282B38281E001C080E0DF91CF911F91EC
:10D9E0000F91FF90EF90DF90CF90BF90AF909F90FE
:10D9F0008F900895CF92DF92EF92FF920F931F9333
:10DA0000CF93DF93EC017A018B016901423051051C
:10DA10006105710508F453C08E819F81A885B98581
:10DA20000196A11DB11D84179507A607B70708F435
:10DA300046C08B89803129F45527412F302F2F2D57
:10DA40000BC08032E1F59A01AB0167E0569547952E
:10DA5000379527956A95D1F78F859889A989BA89CD
:10DA6000280F391F4A1F5B1FCA01B90140E00E94FD
:10DA7000866C9C01009719F18B89803159F4F7016C
:10DA8000F070EE0FFF1FE20FF31F80819181A0E085
:10DA9000B0E00EC0F701EF77F070EE0FFF1FEE0F52
:10DAA000FF1FE20FF31F80819181A281B381BF70BC
:10DAB000F60180839183A283B38381E001C080E07B
:10DAC000DF91CF911F910F91FF90EF90DF90CF905A
:10DAD00008958F929F92AF92BF92CF92DF92EF9272
:10DAE000FF920F931F93DF93CF9300D000D0CDB759
:10DAF000DEB75C016A017B014E010894811C911C18
:10DB0000C501B701A60194010E94FA6C8823B1F106
:10DB1000C501B701A60100E010E020E030E00E945E
:10DB20008A6C882359F1F50180819181A281B381AA
:10DB3000C816D906EA06FB0620F4C082D182E2822A
:10DB4000F382C980DA80EB80FC80F5018389803123
:10DB500051F4F8EFCF16FFEFDF06F0E0EF06F0E04C
:10DB6000FF0670F209C088EFC8168FEFD8068FEF56
:10DB7000E8068FE0F80620F281E001C080E00F9017
:10DB80000F900F900F90CF91DF911F910F91FF9009
:10DB9000EF90DF90CF90BF90AF909F908F900895BF
:10DBA0002F923F924F925F926F927F928F929F92AD
:10DBB000AF92BF92CF92DF92EF92FF920F931F939B
:10DBC000DF93CF93CDB7DEB766970FB6F894DEBF7D
:10DBD0000FBECDBF1C0149875A876B877C873E8764
:10DBE0002D87DC0116962D913D914D915C911997F1
:10DBF0002F5F3F4F4F4F5F4F2D833E834F8358879B
:10DC0000ED85FE8500811181228133810115110589
:10DC10002105310549F0480159010894811C911CE6
:10DC2000A11CB11C10E006C0DC018D909D90AD9050
:10DC3000BC9011E075016401442455243201F101C6
:10DC400086819781A085B185481659066A067B06AC
:10DC500008F09DC02D813E814F8158852C153D05D2
:10DC60004E055F0550F4F2E08F2E912CA12CB12CC3
:10DC7000E2E0CE2ED12CE12CF12CC101B701A6019E
:10DC80009E012F5F3F4F0E94FA6C882309F47FC0EA
:10DC900089819A81AB81BC810097A105B10571F0A2
:10DCA0008C149D04AE04BF0409F010E04601570136
:10DCB0000894811C911CA11CB11C16C0D701C6017F
:10DCC0000196A11DB11D8B8B9C8BAD8BBE8B8819D2
:10DCD0009909AA09BB0929853A854B855C85821774
:10DCE0009307A407B50759F00894411C511C611C07
:10DCF000711C0894C11CD11CE11CF11CA0CF112384
:10DD000049F08B899C89AD89BE89F101808391831B
:10DD1000A283B383C101B701A6010FEF1FEF2FEF5D
:10DD20003FE00E948A6C882399F431C026013701B4
:10DD300008944108510861087108C101B301A201AA
:10DD4000970186010E948A6C882309F173016201A0
:10DD50008C149D04AE04BF0448F3AD85BE854D917F
:10DD60005D916D917C91411551056105710539F009
:10DD7000C101950184010E948A6C882341F0ED85E0
:10DD8000FE8580829182A282B38281E001C080E020
:10DD900066960FB6F894DEBF0FBECDBFCF91DF9170
:10DDA0001F910F91FF90EF90DF90CF90BF90AF90B9
:10DDB0009F908F907F906F905F904F903F902F90AB
:10DDC00008958091C10085FDFCCF8091C00085FF42
:10DDD000F8CF6093C60081E090E008951092C10DE5
:10DDE0001092C00D83E892E09093BF0D8093BE0D1A
:10DDF0000895FF920F931F93CF93DF938B010E949F
:10DE0000D956EB01FF24FA9409C00E94D9566C1B25
:10DE10007D0B6017710710F080E008C0FEBC0DB4E8
:10DE200007FEFDCF8EB58F3F81F781E0DF91CF9167
:10DE30001F910F91FF9008950F931F938C0182EC17
:10DE40009DE0F80162810E944672F801808160E0E5
:10DE50000E94C4571F910F910895FF920F931F9333
:10DE6000DF93CF9300D000D0CDB7DEB78C01F62E74
:10DE700029833A834B835C830E941C6FC80168E549
:10DE800072E00E94F96E8F2D80648EBD0DB407FE86
:10DE9000FDCFFE0131969E012350304083818EBD1F
:10DEA0000DB407FEFDCF3197E217F307B9F7FF2056
:10DEB00011F087E801C085E98EBD0DB407FEFDCFE6
:10DEC0008CE0F81631F48FEF8EBD0DB407FEFDCF58
:10DED0008EB590E02FEF2EBD0DB407FEFDCF8EB5B1
:10DEE00087FF02C09150B9F7F80183830F900F901C
:10DEF0000F900F90CF91DF911F910F91FF90089598
:10DF0000FC01808161E00E94C4578FEF8EBD0DB48B
:10DF100007FEFDCF0895CF93DF93EC010E941C6FA5
:10DF2000CE0168E572E00E94F96E882389F08DEFDA
:10DF30008EBD0DB407FEFDCFCE0168E572E00E94F4
:10DF4000F96E882329F0CE010E94806F81E006C01F
:10DF500082E18983CE010E94806F80E0DF91CF91C2
:10DF60000895AF92BF92CF92DF92EF92FF920F93FC
:10DF70001F93CF93DF93EC015A016B017801890164
:10DF800067E320E030E040E050E00E942D6FCE01DA
:10DF900067E1A80197010E942D6F882311F089E0A5
:10DFA00013C08C81833039F089E0AA0CBB1CCC1CD7
:10DFB000DD1C8A95D1F7CE0169E1A60195010E9489
:10DFC0002D6F882339F087E08983CE010E94806F0E
:10DFD00080E004C0CE010E94806F81E0DF91CF918C
:10DFE0001F910F91FF90EF90DF90CF90BF90AF9077
:10DFF0000895CF93DF93EC01DA016EBD0DB407FEF7
:10E00000FDCF8C918EBD1196EC91119782E090E03E
:10E010000DB407FEFDCFEEBD22E08030920731F057
:10E02000FD01E80FF91FE0810196F2CF0DB407FE64
:10E03000FDCF8FEF8EBD0DB407FEFDCF8FEF8EBDF0
:10E040000DB407FEFDCF8FEF8EBD0DB407FEFDCFE3
:10E050008EB58B838F71853011F481E006C083E12A
:10E060008983CE010E94806F80E0DF91CF91089577
:10E070000F931F93CF93DF93EC018B010E941C6FD2
:10E08000CE0168E572E00E94F96E882361F0CE014E
:10E090006CEFA8010E94F96F882329F0CE010E943D
:10E0A000806F81E006C085E18983CE010E94806F88
:10E0B00080E0DF91CF911F910F910895CF92DF9271
:10E0C000EF92FF920F931F93CF93DF93EC017A01AE
:10E0D0008B0169018C81833039F099E0EE0CFF1CD3
:10E0E000001F111F9A95D1F7CE0168E1A801970191
:10E0F0000E942D6F882319F086E089830CC0CE0121
:10E100006EEFA6010E94F96F882329F0CE010E94CC
:10E11000806F81E004C0CE010E94806F80E0DF91BB
:10E12000CF911F910F91FF90EF90DF90CF900895C6
:10E13000CF93DF93EC016CE020E030E040E050E072
:10E140000E942D6F882339F083E08983CE010E94DD
:10E15000806F80E004C0CE010E94806F81E0DF917B
:10E16000CF910895CF93DF93EC019A01AB018C819D
:10E17000833039F069E0220F331F441F551F6A9521
:10E18000D1F7CE0162E10E942D6F882339F085E03E
:10E190008983CE010E94806F80E004C0CE010E947E
:10E1A000806F81E0DF91CF910895BF92CF92DF928F
:10E1B000EF92FF920F931F93CF93DF93EC016B01CC
:10E1C0007A010E94D9568B01BB24BA9409C00E94DF
:10E1D000D956601B710B6D52714010F081E10BC07C
:10E1E000BEBC0DB407FEFDCF8EB58B838F3F79F398
:10E1F0008E3F39F08FE08983CE010E94806F80E0EE
:10E2000030C0D7011197EF28D9F08FEF8EBD20E0F5
:10E2100030E09FEF0BC00DB407FEFDCF8EB59EBD65
:10E22000F601E20FF31F80832F5F3F4F2A173B0752
:10E2300090F30DB407FEFDCF8EB5AC0DBD1D8C93D4
:10E240001B828FEF8EBD0DB407FEFDCF8EB58FEF15
:10E250008EBD0DB407FEFDCF8EB5CE010E94806F3E
:10E2600081E0DF91CF911F910F91FF90EF90DF90B0
:10E27000CF90BF900895EF92FF920F931F938C0160
:10E280007B010E941C6FC801B70140E052E00E9470
:10E29000D5701F910F91FF90EF900895CF92DF926C
:10E2A000EF92FF920F931F93CF93DF93EC017A01CC
:10E2B0008B0169018C81833039F0B9E0EE0CFF1CD1
:10E2C000001F111FBA95D1F7CE0161E1A801970196
:10E2D0000E942D6F882339F084E08983CE010E944B
:10E2E000806F80E006C0CE01B60140E052E00E949F
:10E2F000D570DF91CF911F910F91FF90EF90DF903C
:10E30000CF900895BF92CF92DF92EF92FF920F933A
:10E310001F93CF93DF93EC01B42E1C821982688384
:10E320000E94D9566B01888161E00E9485578881DF
:10E3300061E00E94C45782EC9DE00E94607280E41C
:10E340008A8382EC9DE060E40E94467280E09FEF49
:10E350009EBD0DB407FEFDCF8F5F8A30C9F709C09F
:10E360000E94D9566C197D09615D774010F081E0FB
:10E3700063C0CE0160E020E030E040E050E00E9469
:10E380002D6F813069F71FEFCE0168E02AEA31E096
:10E3900040E050E00E942D6F853011F481E00DC007
:10E3A00080E01EBD0DB407FEFDCF9EB58F5F8430AB
:10E3B000C1F79B839A3A31F482E08C838C8182305E
:10E3C00051F40DC00E94D9566C197D09615D7740EA
:10E3D000D8F282E031C0EE24FF2487010FC0E12C87
:10E3E000F12C012D80E4182F09C00E94D9566C1918
:10E3F0007D09615D774010F08AE01EC0CE0167E3C1
:10E4000020E030E040E050E00E942D6FCE0169E254
:10E41000A80197010E942D6F882339F78C818230E3
:10E4200031F5CE016AE320E030E040E050E00E94A8
:10E430002D6F882339F088E08983CE010E94806F98
:10E4400080E01AC08FEF8EBD0DB407FEFDCF8EB5F4
:10E45000807C803C11F483E08C8380E09FEF9EBD44
:10E460000DB407FEFDCF2EB58F5F8330C1F7CE010F
:10E470000E94806FBA8281E0DF91CF911F910F914E
:10E48000FF90EF90DF90CF90BF90089540E082E042
:10E4900002C0880F4F5F861710F44630D1F7242F43
:10E4A00030E0C9019595879580658CBD40FF02C01D
:10E4B00080E004C080E0463009F081E08DBD089521
:10E4C00084E061E00E94C45784E061E00E948557C7
:10E4D00086E060E00E94855785E061E00E948557F4
:10E4E00087E061E00E9485570895382F413210F08F
:10E4F00040E042C08091C30D8823E1F791E0909302
:10E50000C30D2093C50D8FEF8093300E1092EB0D4D
:10E5100041504093EC0D4F5F9093C40D8091C40D1A
:10E52000330F832B8093C40D8091C60D813041F44D
:10E530001092C60D8091C40D8093BB0085EC01C084
:10E5400085EE8093BC008091C30D8130E1F3809112
:10E55000EB0D841710F44091EB0D20E030E00AC081
:10E56000FB01E20FF31FD901A553B24F8C918083B9
:10E570002F5F3F4F2417A0F3842F08950F931F930D
:10E58000582F122F413210F081E04AC08091C30D04
:10E590008823E1F782E08093C30D0093C50D8FEFD0
:10E5A0008093300E1092EB0D4093EC0DABECBDE080
:10E5B000FB0102C081918D938E2F861B8417D0F3AF
:10E5C0001092C40D8091C40D550F852B8093C40DFE
:10E5D0008091C60D813041F41092C60D8091C40D1A
:10E5E0008093BB0085EC01C085EE8093BC001123B5
:10E5F00021F08091C30D8230E1F38091300E8F3F86
:10E6000011F480E00DC08091300E803211F482E070
:10E6100007C08091300E803311F084E001C083E0A8
:10E620001F910F910895482F613210F081E00895F5
:10E630008091C30D843011F082E0089560930E0E36
:10E64000ADEEBDE0842F9C01F90102C081918D9354
:10E650008E2F841B8617D0F380E008951F920F92AF
:10E660000FB60F9211242F933F934F935F936F93A5
:10E670007F938F939F93AF93BF93EF93FF9380917B
:10E68000B90090E0887F90708036910509F4F2C05F
:10E6900081369105CCF58832910509F47BC0893229
:10E6A0009105B4F48031910509F46FC08131910571
:10E6B0003CF4009709F447C1089709F04FC165C0C1
:10E6C0008831910509F466C0809709F047C182C07E
:10E6D0008034910509F4A4C08134910544F4803359
:10E6E000910509F482C0C89709F038C189C0803506
:10E6F000910509F489C08835910509F496C08834DC
:10E70000910509F02BC1AEC08839910509F413C1F8
:10E7100089399105ECF48837910509F4ABC0893744
:10E7200091054CF48836910509F4A4C08037910511
:10E7300009F014C19FC08838910509F4FCC08039E4
:10E74000910509F49DC08038910509F007C198C072
:10E75000803B910509F4C6C0813B91054CF4803A99
:10E76000910509F49FC0883A910509F0F7C0BAC035
:10E77000803C910509F4E3C0883C910509F4DFC0B1
:10E78000883B910509F0EAC0C2C08091C40D809316
:10E79000BB00CFC09091EB0D8091EC0D981768F401
:10E7A0009091EB0DE92FF0E0E553F24F80818093DB
:10E7B000BB009F5F9093EB0DBCC08091C50D88237B
:10E7C00009F44BC085ED8093BC008091BC0084FDB2
:10E7D000FCCFC2C080E28093300E85ED8093BC00F8
:10E7E0008091BC0084FDFCCFB7C080E38093300EE5
:10E7F00085ED8093BC008091BC0084FDFCCFACC053
:10E8000088E38093300E9BC08091EB0D9091BB000C
:10E81000E82FF0E0E553F24F90838F5F8093EB0D8C
:10E820009091EB0D8091EC0D82C08091EB0D909159
:10E83000BB00E82FF0E0E553F24F90838F5F8093A9
:10E84000EB0D8091C50D882341F085ED8093BC00D0
:10E850008091BC0084FDFCCF7FC081E08093C60D19
:10E8600084EA6EC085ED8093BC008091BC0084FD7D
:10E87000FCCF72C083E08093C30D10922F0E59C05D
:10E8800080912F0E803208F056C080912F0E90910B
:10E89000BB00E82FF0E0E15FF14F90838F5F809342
:10E8A0002F0E47C080912F0E803230F4E0912F0E52
:10E8B000F0E0E15FF14F108285ED8093BC00809124
:10E8C000BC0084FDFCCF1092C30D60912F0EE0912F
:10E8D000C90DF091CA0D8FE09EE070E0099510928D
:10E8E0002F0E2DC084E08093C30D10920D0E109258
:10E8F0000E0EE091C70DF091C80D099580910E0E96
:10E90000882329F481E080930E0E1092ED0D9091F2
:10E910000D0EE92FF0E0E351F24F80818093BB00B0
:10E920009F5F90930D0E90910D0E80910E0E981793
:10E9300010F485EC01C085E88093BC000FC085EC25
:10E940008093BC0009C01092300E85ED8093BC000E
:10E950008091BC0084FDFCCF1092C30DFF91EF911C
:10E96000BF91AF919F918F917F916F915F914F91E7
:10E970003F912F910F900FBE0F901F9018951092FE
:10E98000C30D81E08093C50D1092C60D81E161E059
:10E990000E94C45780E161E00E94C457E9EBF0E0B7
:10E9A00080818E7F808380818D7F808388E48093C7
:10E9B000B80085E48093BC000895629FD001739FE6
:10E9C000F001829FE00DF11D649FE00DF11D929F0B
:10E9D000F00D839FF00D749FF00D659FF00D99274A
:10E9E000729FB00DE11DF91F639FB00DE11DF91F6E
:10E9F000BD01CF0111240895991B79E004C0991F2E
:10EA0000961708F0961B881F7A95C9F78095089588
:10EA1000AA1BBB1B51E107C0AA1FBB1FA617B70744
:10EA200010F0A61BB70B881F991F5A95A9F7809560
:10EA30009095BC01CD01089597FB092E07260AD0B9
:10EA400077FD04D0E5DF06D000201AF470956195BB
:10EA50007F4F0895F6F7909581959F4F0895A1E215
:10EA60001A2EAA1BBB1BFD010DC0AA1FBB1FEE1F48
:10EA7000FF1FA217B307E407F50720F0A21BB30B93
:10EA8000E40BF50B661F771F881F991F1A9469F70F
:10EA900060957095809590959B01AC01BD01CF016B
:10EAA000089597FB092E05260ED057FD04D0D7DF19
:10EAB0000AD0001C38F450954095309521953F4F71
:10EAC0004F4F5F4F0895F6F790958095709561953B
:10EAD0007F4F8F4F9F4F08952F923F924F925F929B
:10EAE0006F927F928F929F92AF92BF92CF92DF925E
:10EAF000EF92FF920F931F93CF93DF93CDB7DEB7C3
:10EB0000CA1BDB0B0FB6F894DEBF0FBECDBF099456
:10EB10002A88398848885F846E847D848C849B84AD
:10EB2000AA84B984C884DF80EE80FD800C811B81BB
:10EB3000AA81B981CE0FD11D0FB6F894DEBF0FBEEA
:10EB4000CDBFED010895EE0FFF1F0590F491E02D6C
:06EB50000994F894FFCFC8
:10EB56002F00616C6C002E0076006F70656E646F1E
:10EB66006F7200426F73746F6E2C4D41006874743F
:10EB760070733A2F2F75692E6F70656E7370726998
:10EB86006E6B6C65722E636F6D2F6A7300776561AD
:10EB9600746865722E6F70656E737072696E6B6CD9
:10EBA60065722E636F6D000068747470733A2F2F50
:10EBB60075692E6F70656E737072696E6B6C6572B7
:10EBC6002E636F6D2F6A7300776561746865722EA8
:10EBD6006F70656E737072696E6B6C65722E636FA3
:10EBE6006D00763D5B00743D5B00776C00666C00E3
:10EBF6000D0A0000323030002F004F532D30300008
:10EC060063825363350150002F6C6F67732F00D8F2
:10EC16001C01010000000000000000500016000169
:10EC26008000003C00006401000096640F50003232
:10EC360061D2A90100003C02640000009B40A3438E
:10EC46004C3A0639333B233A9B457636FF38A9358D
:10EC5600B9340A35D13C8746793AED3EC034D933CA
:10EC66000C368E467B010A100E000001FFFFFFFFE7
:10EC7600FFFF00000000E112BA5A00004000140035
:10EC86005400000000000914BA5A2E6F4F6F00009E
:10EC96000000000000FFFFFFFFFFFF1F1C1F1E1FDD
:10ECA6001E1F1F1E1F1E1F00000000DC59BA5A70CF
:10ECB60059A1598159CA59000000005C5C2B5CE4DB
:10ECC6005BED5B025C135C00000000736A6F6A0018
:08ECD600000000E16EBA5A00D3
:00000001FF
